:04070000F6EFE9F037
:08070800056ED8CF06F0E0CF2A
:1007100007F00001E9CF0DF0EACF08F0E1CF09F0D2
:10072000E2CF0AF0D9CF0BF0DACF0CF0F3CF14F010
:10073000F4CF15F0FACF16F0FBCF17F000C00FF092
:1007400001C010F002C011F003C012F004C013F099
:10075000F2AAAEEF03F0F2B4EDEF25F09DA0B4EFF6
:1007600003F09EB0E0EF24F0A0A2BAEF03F0A1B234
:10077000F8EF26F0F2A8C0EF03F0F2B286EF24F013
:10078000F0A6C6EF03F0F0B0A8EF24F0F0A8CCEF8D
:1007900003F0F0B297EF24F09DAAD2EF03F09EBAD7
:1007A00087EF28F0A3AAD8EF03F0A4BAAEEF28F0A1
:1007B000F0AADEEF03F0F0B4B9EF24F00FC000F0C0
:1007C00010C001F011C002F012C003F013C004F019
:1007D0000DC0E9FF08C0EAFF088E09C0E1FF0AC0AA
:1007E000E2FF0BC0D9FF0CC0DAFF14C0F3FF15C045
:1007F000F4FF16C0FAFF17C0FBFF055007C0E0FF6B
:1008000006C0D8FF1000F2CF0EF0F29EF76A240F58
:10081000F66E080EF722000EF86E0900F5500EBEB7
:10082000F28E1200280C0106F2CF0EF0F29EF76A4B
:10083000460FF66E080EF722000EF86E0900F5500E
:100840000EBEF28E1200536F6E79204556492D442C
:1008500033302020202020202000F2CF0EF0F29E06
:10086000F76A780FF66E080EF722000EF86E090090
:10087000F5500EBEF28E1200536F6E792045564928
:100880002D4433302F44333120202000F2CF0EF09E
:10089000F29EF76AAA0FF66E080EF722000EF86EA7
:1008A0000900F5500EBEF28E120056616464696F45
:1008B000204164642D612D43616D20202000F2CF22
:1008C0000EF0F29EF76ADC0FF66E080EF722000EAD
:1008D000F86E0900F5500EBEF28E1200536F6E795D
:1008E000204556492D443130302020202020200042
:1008F000F2CF0EF0F29EF76A0E0FF66E090EF72297
:10090000000EF86E0900F5500EBEF28E1200536F05
:100910006E79204556492D44373020202020202054
:100920002000F2CF0EF0F29EF76A400FF66E090E2D
:10093000F722000EF86E0900F5500EBEF28E12007E
:10094000536F6E79204252432D33303020202020C7
:1009500020202000F2CF0EF0F29EF76A720FF66EA2
:10096000090EF722000EF86E0900F5500EBEF28E49
:100970001200536F6E79204252432D483730302099
:10098000202020202000F2CF0EF0F29EF76AA40F64
:10099000F66E090EF722000EF86E0900F5500EBE35
:1009A000F28E1200536F6E79204252432D5A373027
:1009B0003020202020202000F2CF0EF0F29EF76A97
:1009C000D60FF66E090EF722000EF86E0900F550EC
:1009D0000EBEF28E1200536F6E79204556492D4897
:1009E00044312020202020202000F2CF0EF0F29E63
:1009F000F76A080FF66E0A0EF722000EF86E09006D
:100A0000F5500EBEF28E120056616464696F204884
:100A1000442D31382020202020202000F2CF0EF05D
:100A2000F29EF76A3A0FF66E0A0EF722000EF86E83
:100A30000900F5500EBEF28E120056616464696FB3
:100A4000204365696C696E67564945572000F2CFAF
:100A50000EF0F29EF76A6C0FF66E0A0EF722000E89
:100A6000F86E0900F5500EBEF28E120043616E6EF4
:100A70006F6E2056432D4335306920202020200002
:100A8000F2CF0EF0F29EF76A9E0FF66E0A0EF72274
:100A9000000EF86E0900F5500EBEF28E12004E6F79
:100AA0007420466F756E6420202020202020202096
:100AB0002000F2CF0EF0F29EF76AD00FF66E0A0E0B
:100AC000F722000EF86E0900F5500EBEF28E1200ED
:100AD00045787420507265736574733A2043616D74
:100AE0003120312D31322C2043616D32204E6F6E1A
:100AF0006500F2CF0EF0F29EF76A100FF66E0B0E45
:100B0000F722000EF86E0900F5500EBEF28E1200AC
:100B100045787420507265736574733A2043616D33
:100B20003120312D362C2043616D3220312D36009D
:100B3000F2CF0EF0F29EF76A4E0FF66E0B0EF72212
:100B4000000EF86E0900F5500EBEF28E12005A6FBC
:100B50006F6D20446972656374696F6E3A20496EE7
:100B6000766572740000F2CF0EF0F29EF76A840F81
:100B7000F66E0B0EF722000EF86E0900F5500EBE51
:100B8000F28E12005A6F6F6D20446972656374694A
:100B90006F6E3A204E6F726D616C0000F2CF0EF0F6
:100BA000F29EF76ABA0FF66E0B0EF722000EF86E81
:100BB0000900F5500EBEF28E120045787420507276
:100BC0006573657420696E332D36204469726563E0
:100BD00074696F6E3A204F75747075740000F2CFAF
:100BE0000EF0F29EF76AFC0FF66E0B0EF722000E67
:100BF000F86E0900F5500EBEF28E12004578742092
:100C000050726573657420696E332D3620446972A5
:100C1000656374696F6E3A20496E70757400F2CF27
:100C20000EF0F29EF76A3C0FF66E0C0EF722000EE5
:100C3000F86E0900F5500EBEF28E1200486F737404
:100C40002053657269616C20496E7075743A204555
:100C50006E61626C65640000F2CF0EF0F29EF76A7E
:100C6000760FF66E0C0EF722000EF86E0900F550A6
:100C70000EBEF28E1200486F737420536572696164
:100C80006C20496E7075743A2044697361626C65BA
:100C90006400F2CF0EF0F29EF76AB00FF66E0C0E03
:100CA000F722000EF86E0900F5500EBEF28E12000B
:100CB00053657269616C204563686F3A20456E61C7
:100CC000626C65640000F2CF0EF0F29EF76AE40FEA
:100CD000F66E0C0EF722000EF86E0900F5500EBEEF
:100CE000F28E120053657269616C204563686F3A39
:100CF0002044697361626C656400F2CF0EF0F29E6D
:100D0000F76A180FF66E0D0EF722000EF86E090046
:100D1000F5500EBEF28E120043616D2053656C20BB
:100D2000466F6C6C6F777320507265766965773AA1
:100D300020456E61626C65640000F2CF0EF0F29E99
:100D4000F76A580FF66E0D0EF722000EF86E0900C6
:100D5000F5500EBEF28E120043616D2053656C207B
:100D6000466F6C6C6F777320507265766965773A61
:100D70002044697361626C656400F2CF0EF0F29EEC
:100D8000F76A980FF66E0D0EF722000EF86E090046
:100D9000F5500EBEF28E12000000F2CF0EF0F29E61
:100DA000F76AB80FF66E0D0EF722000EF86E090006
:100DB000F5500EBEF28E120053797374656D204D9E
:100DC0006F64653A204175746F00F2CF0EF0F29EA9
:100DD000F76AE80FF66E0D0EF722000EF86E0900A6
:100DE000F5500EBEF28E120053797374656D204D6E
:100DF0006F64653A204D616E75616C00F2CF0EF044
:100E0000F29EF76A1A0FF66E0E0EF722000EF86EBB
:100E10000900F5500EBEF28E1200566964656F200F
:100E2000466F726D61743A2050414C00F2CF0EF063
:100E3000F29EF76A4A0FF66E0E0EF722000EF86E5B
:100E40000900F5500EBEF28E1200566964656F20DF
:100E5000466F726D61743A204E5453430000F2CFD6
:100E60000EF0F29EF76A7C0FF66E0E0EF722000E61
:100E7000F86E0900F5500EBEF28E120044696167EB
:100E80006E6F73746963204D6F64653A204F6E0016
:100E9000F2CF0EF0F29EF76AAE0FF66E0E0EF7224C
:100EA000000EF86E0900F5500EBEF28E1200446975
:100EB00061676E6F73746963204D6F64653A204F8C
:100EC00066660000F2CF0EF0F29EF76AE20FF66E51
:100ED0000E0EF722000EF86E0900F5500EBEF28ECF
:100EE000120053657269616C20496E666F3A204F3B
:100EF0006E00F2CF0EF0F29EF76A100FF66E0F0E34
:100F0000F722000EF86E0900F5500EBEF28E1200A8
:100F100053657269616C20496E666F3A204F666650
:100F20000000F2CF0EF0F29EF76A400FF66E0F0E41
:100F3000F722000EF86E0900F5500EBEF28E120078
:100F40004F75747075742027436F6C6F7220426107
:100F5000727327204F6E204E6F20496E707574207B
:100F6000536F757263650000F2CF0EF0F29EF76A60
:100F7000860FF66E0F0EF722000EF86E0900F55080
:100F80000EBEF28E12004F75747075742027426C7D
:100F9000616E6B27204F6E204E6F20496E70757406
:100FA00020536F7572636500F2CF0EF0F29EF76A00
:100FB000C60FF66E0F0EF722000EF86E0900F55000
:100FC0000EBEF28E1200506F776572207570205041
:100FD00072657365743A205072657365742031329E
:100FE0000000F2CF0EF0F29EF76A000FF66E100EC0
:100FF000F722000EF86E0900F5500EBEF28E1200B8
:10100000506F776572207570205072657365743A01
:1010100020486F6D652043616D00F2CF0EF0F29EA7
:10102000F76A380FF66E100EF722000EF86E090000
:10103000F5500EBEF28E1200504320457870616E5E
:10104000646572204D6F64653A20532D566964655E
:101050006F00F2CF0EF0F29EF76A700FF66E100E70
:10106000F722000EF86E0900F5500EBEF28E120047
:10107000504320457870616E646572204D6F6465E1
:101080003A204E6F6E650000F2CF0EF0F29EF76AC6
:10109000A60FF66E100EF722000EF86E0900F5503E
:1010A0000EBEF28E1200504320457870616E64656A
:1010B00072204D6F64653A20436F6D706F73697471
:1010C0006500F2CF0EF0F29EF76AE00FF66E100E9A
:1010D000F722000EF86E0900F5500EBEF28E1200D7
:1010E000507265736574204C6F636174696F6E3AFA
:1010F00020312D3620496E43616D2C362D31322042
:101100004C6F63616C00F2CF0EF0F29EF76A240F11
:10111000F66E110EF722000EF86E0900F5500EBEA5
:10112000F28E1200507265736574204C6F636174A7
:10113000696F6E3A20312D3132204C6F63616C0043
:10114000F2CF0EF0F29EF76A5E0FF66E110EF722E6
:10115000000EF86E0900F5500EBEF28E1200446FBC
:1011600046696E644163746976655072657365742F
:101170007320506F7274202564206261640A0D0030
:10118000F2CF0EF0F29EF76A9E0FF66E110EF72266
:10119000000EF86E0900F5500EBEF28E12002020EF
:1011A0002053797374656D204D656E752020200085
:1011B000F2CF0EF0F29EF76ACE0FF66E110EF72206
:1011C000000EF86E0900F5500EBEF28E12002020BF
:1011D00053657269616C20496E707574202020001F
:1011E000F2CF0EF0F29EF76AFE0FF66E110EF722A6
:1011F000000EF86E0900F5500EBEF28E120020208F
:1012000053657269616C204563686F20202020005F
:10121000F2CF0EF0F29EF76A2E0FF66E120EF72244
:10122000000EF86E0900F5500EBEF28E120020205E
:10123000436C656172204D656D6F727920202000CE
:10124000F2CF0EF0F29EF76A5E0FF66E120EF722E4
:10125000000EF86E0900F5500EBEF28E120020202E
:10126000436C656172205072657365747320200051
:10127000F2CF0EF0F29EF76A8E0FF66E120EF72284
:10128000000EF86E0900F5500EBEF28E12002020FE
:101290002053657269616C20496E666F20202000C2
:1012A000F2CF0EF0F29EF76ABE0FF66E120EF72224
:1012B000000EF86E0900F5500EBEF28E12002020CE
:1012C00049646C6520446973706C6179202020004A
:1012D000F2CF0EF0F29EF76AEE0FF66E120EF722C4
:1012E000000EF86E0900F5500EBEF28E120020209E
:1012F000566964656F20466F726D6174202020000E
:10130000F2CF0EF0F29EF76A1E0FF66E130EF72262
:10131000000EF86E0900F5500EBEF28E120020206D
:10132000506F776572205570205072657365740038
:10133000F2CF0EF0F29EF76A4E0FF66E130EF72202
:10134000000EF86E0900F5500EBEF28E120020203D
:10135000507265736574204C6F636174696F6E00C1
:10136000F2CF0EF0F29EF76A7E0FF66E130EF722A2
:10137000000EF86E0900F5500EBEF28E120020200D
:101380002020504320457870616E646572202000F3
:10139000F2CF0EF0F29EF76AAE0FF66E130EF72242
:1013A000000EF86E0900F5500EBEF28E12002020DD
:1013B00052657475726E20746F204D61696E2000E5
:1013C000F2CF0EF0F29EF76ADE0FF66E130EF722E2
:1013D000000EF86E0900F5500EBEF28E12002020AD
:1013E0005472616E736974696F6E204D656E75001D
:1013F000F2CF0EF0F29EF76A0E0FF66E140EF72281
:10140000000EF86E0900F5500EBEF28E120020207C
:10141000204566666563742053656C6563742000BF
:10142000F2CF0EF0F29EF76A3E0FF66E140EF72220
:10143000000EF86E0900F5500EBEF28E120020204C
:101440002054696D6520496E74657276616C200068
:10145000F2CF0EF0F29EF76A6E0FF66E140EF722C0
:10146000000EF86E0900F5500EBEF28E120020201C
:10147000204D61696E204F66662054696D652000BD
:10148000F2CF0EF0F29EF76A9E0FF66E140EF72260
:10149000000EF86E0900F5500EBEF28E12002020EC
:1014A0002050616E20446972204D656E75202000C9
:1014B000F2CF0EF0F29EF76ACE0FF66E140EF72200
:1014C000000EF86E0900F5500EBEF28E12002020BC
:1014D000202020416C6C20506F72747320202000FB
:1014E000F2CF0EF0F29EF76AFE0FF66E140EF722A0
:1014F000000EF86E0900F5500EBEF28E120020208C
:1015000020202020506F72742030312020202000B5
:10151000F2CF0EF0F29EF76A2E0FF66E150EF7223E
:10152000000EF86E0900F5500EBEF28E120020205B
:1015300020202020506F7274203032202020200084
:10154000F2CF0EF0F29EF76A5E0FF66E150EF722DE
:10155000000EF86E0900F5500EBEF28E120020202B
:1015600020202020506F7274203033202020200053
:10157000F2CF0EF0F29EF76A8E0FF66E150EF7227E
:10158000000EF86E0900F5500EBEF28E12002020FB
:1015900020202020506F7274203034202020200022
:1015A000F2CF0EF0F29EF76ABE0FF66E150EF7221E
:1015B000000EF86E0900F5500EBEF28E12002020CB
:1015C00020202020506F72742030352020202000F1
:1015D000F2CF0EF0F29EF76AEE0FF66E150EF722BE
:1015E000000EF86E0900F5500EBEF28E120020209B
:1015F00020202020506F72742030362020202000C0
:10160000F2CF0EF0F29EF76A1E0FF66E160EF7225C
:10161000000EF86E0900F5500EBEF28E120020206A
:1016200054696C7420446972204D656E75202000E9
:10163000F2CF0EF0F29EF76A4E0FF66E160EF722FC
:10164000000EF86E0900F5500EBEF28E120020203A
:10165000202052657363616E20566964656F2000B7
:10166000F2CF0EF0F29EF76A7E0FF66E160EF7229C
:10167000000EF86E0900F5500EBEF28E120020200A
:101680002052657363616E2043616D657261730002
:10169000F2CF0EF0F29EF76AAE0FF66E160EF7223C
:1016A000000EF86E0900F5500EBEF28E12002020DA
:1016B0002044656661756C742043616D65726100DC
:1016C000F2CF0EF0F29EF76ADE0FF66E160EF722DC
:1016D000000EF86E0900F5500EBEF28E12002020AA
:1016E0002044656661756C74205072657365740082
:1016F000F2CF0EF0F29EF76A0E0FF66E170EF7227B
:10170000000EF86E0900F5500EBEF28E1200202079
:101710002050616E53656E736974697669747900DF
:10172000F2CF0EF0F29EF76A3E0FF66E170EF7221A
:10173000000EF86E0900F5500EBEF28E1200202049
:1017400054696C7453656E73697469766974790051
:10175000F2CF0EF0F29EF76A6E0FF66E170EF722BA
:10176000000EF86E0900F5500EBEF28E1200202019
:10177000204465662049646C652052746E20200008
:10178000F2CF0EF0F29EF76A9E0FF66E170EF7225A
:10179000000EF86E0900F5500EBEF28E12002020E9
:1017A00020202050616E2053706565642020200049
:1017B000F2CF0EF0F29EF76ACE0FF66E170EF722FA
:1017C000000EF86E0900F5500EBEF28E12002020B9
:1017D00020202020537461727400F2CF0EF0F29E2C
:1017E000F76AF80FF66E170EF722000EF86E090072
:1017F000F5500EBEF28E120020202020202020590D
:1018000065730000F2CF0EF0F29EF76A220FF66EBB
:10181000180EF722000EF86E0900F5500EBEF28E7B
:10182000120020202020202020204E6F0000F2CF28
:101830000EF0F29EF76A4C0FF66E180EF722000EAD
:10184000F86E0900F5500EBEF28E12002020202006
:1018500020204E6F726D616C0000F2CF0EF0F29E90
:10186000F76A780FF66E180EF722000EF86E090070
:10187000F5500EBEF28E1200202020202020496E4E
:10188000766572740000F2CF0EF0F29EF76AA40F34
:10189000F66E180EF722000EF86E0900F5500EBE17
:1018A000F28E120020202020202020496E707574B6
:1018B0000000F2CF0EF0F29EF76AD00FF66E180E0F
:1018C000F722000EF86E0900F5500EBEF28E1200DF
:1018D0002020202020204F75747075740000F2CFF6
:1018E0000EF0F29EF76AFC0FF66E180EF722000E4D
:1018F000F86E0900F5500EBEF28E12002020362040
:1019000043616D3120362043616D3200F2CF0EF01D
:10191000F29EF76A2A0FF66E190EF722000EF86E85
:101920000900F5500EBEF28E1200202020416C6C92
:101930002031322043616D310000F2CF0EF0F29E73
:10194000F76A580FF66E190EF722000EF86E0900AE
:10195000F5500EBEF28E1200202020202020204FB5
:1019600066660000F2CF0EF0F29EF76A820FF66E06
:10197000190EF722000EF86E0900F5500EBEF28E19
:101980001200202020202020204F6E200000F2CFC7
:101990000EF0F29EF76AAC0FF66E190EF722000EEB
:1019A000F86E0900F5500EBEF28E120020202020A5
:1019B00020426C61636B202020200000F2CF0EF0EB
:1019C000F29EF76ADA0FF66E190EF722000EF86E25
:1019D0000900F5500EBEF28E120020202020204378
:1019E0006F6C6F72204261727300F2CF0EF0F29E44
:1019F000F76A080FF66E1A0EF722000EF86E09004D
:101A0000F5500EBEF28E12002020202020204E54D1
:101A100053430000F2CF0EF0F29EF76A320FF66EDB
:101A20001A0EF722000EF86E0900F5500EBEF28E67
:101A3000120020202020202050414C200000F2CF16
:101A40000EF0F29EF76A5C0FF66E1A0EF722000E89
:101A5000F86E0900F5500EBEF28E120020202020F4
:101A600020486F6D652043616D6572612000F2CF83
:101A70000EF0F29EF76A8C0FF66E1A0EF722000E29
:101A8000F86E0900F5500EBEF28E120020202020C4
:101A90002050726573657420313220202000F2CF0F
:101AA0000EF0F29EF76ABC0FF66E1A0EF722000EC9
:101AB000F86E0900F5500EBEF28E12002020202094
:101AC00020416C6C204C6F63616C20202000F2CFB1
:101AD0000EF0F29EF76AEC0FF66E1A0EF722000E69
:101AE000F86E0900F5500EBEF28E1200202036204E
:101AF000496E43616D2036204C6F63616C00F2CFFC
:101B00000EF0F29EF76A1C0FF66E1B0EF722000E07
:101B1000F86E0900F5500EBEF28E12002020202033
:101B20002020204E4F4E4520202020202000F2CFA4
:101B30000EF0F29EF76A4C0FF66E1B0EF722000EA7
:101B4000F86E0900F5500EBEF28E12002020202003
:101B500020532D566964656F202020202000F2CF8D
:101B60000EF0F29EF76A7C0FF66E1B0EF722000E47
:101B7000F86E0900F5500EBEF28E120020202020D3
:101B8000436F6D706F736974652020202000F2CF61
:101B90000EF0F29EF76AAC0FF66E1B0EF722000EE7
:101BA000F86E0900F5500EBEF28E120020436C65EF
:101BB0006172696E67205072657365747300F2CF4D
:101BC0000EF0F29EF76ADC0FF66E1B0EF722000E87
:101BD000F86E0900F5500EBEF28E12002020202073
:101BE00020204E6F6E652020202020202000F2CF84
:101BF0000EF0F29EF76A0C0FF66E1C0EF722000E26
:101C0000F86E0900F5500EBEF28E12002020202042
:101C100043726F7373466164652020202000F2CF09
:101C20000EF0F29EF76A3C0FF66E1C0EF722000EC5
:101C3000F86E0900F5500EBEF28E12002020486F9B
:101C400072697A2052202D3E204C20202000F2CFB5
:101C50000EF0F29EF76A6C0FF66E1C0EF722000E65
:101C6000F86E0900F5500EBEF28E12002020486F6B
:101C700072697A204C202D3E205220202000F2CF85
:101C80000EF0F29EF76A9C0FF66E1C0EF722000E05
:101C9000F86E0900F5500EBEF28E12002020566537
:101CA00072746963616C2054202D3E204200F2CF93
:101CB0000EF0F29EF76ACC0FF66E1C0EF722000EA5
:101CC000F86E0900F5500EBEF28E12002020566507
:101CD00072746963616C2042202D3E205400F2CF63
:101CE0000EF0F29EF76AFC0FF66E1C0EF722000E45
:101CF000F86E0900F5500EBEF28E12002020436FE0
:101D0000726E657220554C202D3E20425200F2CF5B
:101D10000EF0F29EF76A2C0FF66E1D0EF722000EE3
:101D2000F86E0900F5500EBEF28E12002020436FAF
:101D3000726E6572204252202D3E20554C00F2CF2B
:101D40000EF0F29EF76A5C0FF66E1D0EF722000E83
:101D5000F86E0900F5500EBEF28E12002050432D91
:101D6000457870616E64657220532D566900F2CF1C
:101D70000EF0F29EF76A8C0FF66E1D0EF722000E23
:101D8000F86E0900F5500EBEF28E12002050432D61
:101D9000457870616E64657220436F6D7000F2CF9C
:101DA0000EF0F29EF76ABC0FF66E1D0EF722000EC3
:101DB000F86E0900F5500EBEF28E12000D0A205783
:101DC0006169745F50435F457870616E64657252FB
:101DD0006573706F6E736520256C6420286D7329A0
:101DE0000D0A0000F2CF0EF0F29EF76A020FF66EB7
:101DF0001E0EF722000EF86E0900F5500EBEF28E90
:101E000012000D0A20576169745F50435F45787076
:101E1000616E646572526573706F6E736520000049
:101E2000F2CF0EF0F29EF76A3E0FF66E1E0EF7220C
:101E3000000EF86E0900F5500EBEF28E1200496ECB
:101E40007075742053656C6563742025630A0D00FA
:101E5000F2CF0EF0F29EF76A6E0FF66E1E0EF722AC
:101E6000000EF86E0900F5500EBEF28E120053659A
:101E700061726368696E6720666F72204174746175
:101E8000636865642043616D657261730D0A0000CB
:101E9000F2CF0EF0F29EF76AAE0FF66E1E0EF7222C
:101EA000000EF86E0900F5500EBEF28E1200506F53
:101EB00072742025643A20200000F2CF0EF0F29ECA
:101EC000F76AD80FF66E1E0EF722000EF86E0900A4
:101ED000F5500EBEF28E120050432D457870616EA3
:101EE0006465722044657465637465640D0A00005E
:101EF000F2CF0EF0F29EF76A0E0FF66E1F0EF7226B
:101F0000000EF86E0900F5500EBEF28E1200205041
:101F100063457870616E64657220506F727436002C
:101F2000F2CF0EF0F29EF76A3E0FF66E1F0EF7220A
:101F3000000EF86E0900F5500EBEF28E1200204E13
:101F40006F2043616D20202020506F72742030007C
:101F5000F2CF0EF0F29EF76A6E0FF66E1F0EF722AA
:101F6000000EF86E0900F5500EBEF28E12002056DB
:101F7000432D43353069202020506F72742030008B
:101F8000F2CF0EF0F29EF76A9E0FF66E1F0EF7224A
:101F9000000EF86E0900F5500EBEF28E120043617D
:101FA0006E6F6E2044657465637465640D0A00008D
:101FB000F2CF0EF0F29EF76ACE0FF66E1F0EF722EA
:101FC000000EF86E0900F5500EBEF28E12000D0ADA
:101FD0002057616974466565644261636B2054698A
:101FE0006D656F7574203230303020286D73290D87
:101FF0000A00F2CF0EF0F29EF76A100FF66E200E76
:10200000F722000EF86E0900F5500EBEF28E120097
:102010000D0A2057616974466565644261636B20EF
:102020000000F2CF0EF0F29EF76A400FF66E200E1F
:10203000F722000EF86E0900F5500EBEF28E120067
:102040000A0D2043616D657261547970652000004E
:10205000F2CF0EF0F29EF76A6E0FF66E200EF722A8
:10206000000EF86E0900F5500EBEF28E1200546993
:102070006D656F75740A0D200000F2CF0EF0F29EB0
:10208000F76A980FF66E200EF722000EF86E090020
:10209000F5500EBEF28E12000D0A536F6E79204578
:1020A00056492D4433302F3331200D0A0000F2CF32
:1020B0000EF0F29EF76ACC0FF66E200EF722000E9D
:1020C000F86E0900F5500EBEF28E120020455649FA
:1020D0002D4433302F3331506F7274203000F2CFE3
:1020E0000EF0F29EF76AFC0FF66E200EF722000E3D
:1020F000F86E0900F5500EBEF28E12000D0A536FF5
:102100006E79204556492D4433300D0A0000F2CF38
:102110000EF0F29EF76A2C0FF66E210EF722000EDB
:10212000F86E0900F5500EBEF28E12002045564999
:102130002D443330202020506F7274203000F2CFB5
:102140000EF0F29EF76A5C0FF66E210EF722000E7B
:10215000F86E0900F5500EBEF28E12000D0A56619F
:102160006464696F204164642D412D43616D0D0AE3
:102170000000F2CF0EF0F29EF76A900FF66E210E7D
:10218000F722000EF86E0900F5500EBEF28E120016
:10219000204164642D412D43616D20506F72742085
:1021A0003000F2CF0EF0F29EF76AC00FF66E210EED
:1021B000F722000EF86E0900F5500EBEF28E1200E6
:1021C0000D0A536F6E79204556492D443130300D3C
:1021D0000A00F2CF0EF0F29EF76AF00FF66E210EB3
:1021E000F722000EF86E0900F5500EBEF28E1200B6
:1021F000204556492D443130302020506F727420D4
:102200003000F2CF0EF0F29EF76A200FF66E220E2B
:10221000F722000EF86E0900F5500EBEF28E120085
:102220000D0A536F6E79204556492D4437300D0AFB
:102230000000F2CF0EF0F29EF76A500FF66E220EFB
:10224000F722000EF86E0900F5500EBEF28E120055
:10225000204556492D443730202020506F7274207D
:102260003000F2CF0EF0F29EF76A800FF66E220E6B
:10227000F722000EF86E0900F5500EBEF28E120025
:102280000D0A536F6E7920425243482D3730300D7E
:102290000A00F2CF0EF0F29EF76AB00FF66E220E31
:1022A000F722000EF86E0900F5500EBEF28E1200F5
:1022B00020425243482D3730302020506F72742016
:1022C0003000F2CF0EF0F29EF76AE00FF66E220EAB
:1022D000F722000EF86E0900F5500EBEF28E1200C5
:1022E0000D0A456C6D6F2043616D6572610D0A00CA
:1022F000F2CF0EF0F29EF76A0E0FF66E230EF72263
:10230000000EF86E0900F5500EBEF28E1200204548
:102310006C6D6F202020202020506F7274203000C0
:10232000F2CF0EF0F29EF76A3E0FF66E230EF72202
:10233000000EF86E0900F5500EBEF28E12000D0A66
:10234000536F6E79204252432D3330300D0A000016
:10235000F2CF0EF0F29EF76A6E0FF66E230EF722A2
:10236000000EF86E0900F5500EBEF28E12002042EB
:1023700052432D333030202020506F7274203000B3
:10238000F2CF0EF0F29EF76A9E0FF66E230EF72242
:10239000000EF86E0900F5500EBEF28E12000D0A06
:1023A000536F6E79204252432D5A3730300D0A0058
:1023B000F2CF0EF0F29EF76ACE0FF66E230EF722E2
:1023C000000EF86E0900F5500EBEF28E120020428B
:1023D00052432D5A3730302020506F727420300015
:1023E000F2CF0EF0F29EF76AFE0FF66E230EF72282
:1023F000000EF86E0900F5500EBEF28E12000D0AA6
:1024000056616464696F2048442D31380D0A00001C
:10241000F2CF0EF0F29EF76A2E0FF66E240EF72220
:10242000000EF86E0900F5500EBEF28E120020204C
:1024300048442D3138202020506F72742030000025
:10244000F2CF0EF0F29EF76A5E0FF66E240EF722C0
:10245000000EF86E0900F5500EBEF28E12000D0A45
:10246000536F6E79204556492D4844310D0A0000BE
:10247000F2CF0EF0F29EF76A8E0FF66E240EF72260
:10248000000EF86E0900F5500EBEF28E12002045C7
:1024900056492D484431202020506F72742030005E
:1024A000F2CF0EF0F29EF76ABE0FF66E240EF72200
:1024B000000EF86E0900F5500EBEF28E12000D0AE5
:1024C00056616464696F204365696C696E6756493B
:1024D00045570D0A0000F2CF0EF0F29EF76AF40F96
:1024E000F66E240EF722000EF86E0900F5500EBEAF
:1024F000F28E12002043562F43564D50202020507C
:102500006F7274203000F2CF0EF0F29EF76A240F43
:10251000F66E250EF722000EF86E0900F5500EBE7D
:10252000F28E1200496E76616C69642043616D65BC
:1025300072610D0A0000F2CF0EF0F29EF76A540F9E
:10254000F66E250EF722000EF86E0900F5500EBE4D
:10255000F28E120020496E76616C69642043616DD1
:1025600065726100F2CF0EF0F29EF76A820FF66E8E
:10257000250EF722000EF86E0900F5500EBEF28E01
:1025800012000D0A536F6E79204556492D443330A1
:102590002872290D0A00F2CF0EF0F29EF76AB40FEE
:1025A000F66E250EF722000EF86E0900F5500EBEED
:1025B000F28E1200204556492D443330287229509E
:1025C0006F7274203000F2CF0EF0F29EF76AE40FC3
:1025D000F66E250EF722000EF86E0900F5500EBEBD
:1025E000F28E12000A0D2041542F4D445F4D6F644E
:1025F00065496E712000F2CF0EF0F29EF76A140F5B
:10260000F66E260EF722000EF86E0900F5500EBE8B
:10261000F28E12002054696D656F75740A0D2000EA
:10262000F2CF0EF0F29EF76A3E0FF66E260EF722FC
:10263000000EF86E0900F5500EBEF28E12000D0A63
:102640002057616974536F6E7941636B2054696DD3
:10265000656F757420256C6420286D73290D0A0040
:10266000F2CF0EF0F29EF76A7E0FF66E260EF7227C
:10267000000EF86E0900F5500EBEF28E12000D0A23
:102680002057616974536F6E7941636B28256C64C0
:1026900029200000F2CF0EF0F29EF76AB20FF66E1C
:1026A000260EF722000EF86E0900F5500EBEF28ECF
:1026B00012000D0A2057616974536F6E79205469B6
:1026C0006D656F757420256C6420286D73290D0A63
:1026D0000000F2CF0EF0F29EF76AF00FF66E260EB3
:1026E000F722000EF86E0900F5500EBEF28E1200B1
:1026F0000D0A2057616974536F6E79200000F2CF84
:102700000EF0F29EF76A1C0FF66E270EF722000EEF
:10271000F86E0900F5500EBEF28E12002054696D5D
:10272000656F757420256C6420286D73290D0A006F
:10273000F2CF0EF0F29EF76A4E0FF66E270EF722DA
:10274000000EF86E0900F5500EBEF28E12000A0D52
:102750002042616420436F6D6D616E640A0D00005C
:10276000F2CF0EF0F29EF76A7E0FF66E270EF7227A
:10277000000EF86E0900F5500EBEF28E12000D0A22
:10278000205761697443616E6F6E2054696D656F87
:10279000757420256C6420286D73290D0A00F2CF12
:1027A0000EF0F29EF76ABC0FF66E270EF722000EAF
:1027B000F86E0900F5500EBEF28E12000D0A205779
:1027C00061697443616E6F6E2000F2CF0EF0F29E6D
:1027D000F76AE80FF66E270EF722000EF86E090072
:1027E000F5500EBEF28E12000D0A20576169744337
:1027F000616E6F6E41636B2054696D656F757420F7
:10280000256C6420286D73290D0A0000F2CF0EF0AC
:10281000F29EF76A2A0FF66E280EF722000EF86E67
:102820000900F5500EBEF28E12000D0A20576169A4
:102830007443616E6F6E41636B200000F2CF0EF047
:10284000F29EF76A5A0FF66E280EF722000EF86E07
:102850000900F5500EBEF28E120057616974436193
:102860006E6F6E41636B202532782C2532782028DC
:10287000253278290D0A0000F2CF0EF0F29EF76A99
:10288000960FF66E280EF722000EF86E0900F5502E
:102890000EBEF28E1200446F557064617465436120
:1028A0006D65726153746174653A20537461746527
:1028B000466C61673D202532582C204C6173743D75
:1028C0002532582C204163746976653D2532580ABB
:1028D0000D3E0000F2CF0EF0F29EF76AF20FF66E98
:1028E000280EF722000EF86E0900F5500EBEF28E8B
:1028F0001200446F55706461746543616D65726167
:1029000053746174653A20446966666572656E63E6
:10291000653D2532780A0D00F2CF0EF0F29EF76A7F
:10292000360FF66E290EF722000EF86E0900F550EC
:102930000EBEF28E1200446F55706461746543617F
:102940006D65726153746174653A20546F204175EE
:10295000746F0A0D3E00F2CF0EF0F29EF76A740F0C
:10296000F66E290EF722000EF86E0900F5500EBE25
:10297000F28E1200446F55706461746543616D6539
:10298000726153746174653A2052657365742042B4
:1029900072696768746E657320746F206465666120
:1029A000756C740A0D3E0000F2CF0EF0F29EF76ACD
:1029B000C60FF66E290EF722000EF86E0900F550CC
:1029C0000EBEF28E1200446F5570646174654361EF
:1029D0006D65726153746174653A20546F204D6166
:1029E0006E75616C0A0D3E00F2CF0EF0F29EF76A32
:1029F000060FF66E2A0EF722000EF86E0900F5504B
:102A00000EBEF28E12000A0D50726F647563742050
:102A10004E616D653A20257325730A0D0000F2CFD3
:102A20000EF0F29EF76A3C0FF66E2A0EF722000EA9
:102A3000F86E0900F5500EBEF28E12002020202004
:102A4000436F6D70696C65643A2025732061742052
:102A500025730A0D0000F2CF0EF0F29EF76A740F94
:102A6000F66E2A0EF722000EF86E0900F5500EBE23
:102A7000F28E120032312D4A616E2D313000F2CFCC
:102A80000EF0F29EF76A9C0FF66E2A0EF722000EE9
:102A9000F86E0900F5500EBEF28E120030383A344E
:102AA000353A31370000F2CF0EF0F29EF76AC40FCC
:102AB000F66E2A0EF722000EF86E0900F5500EBED3
:102AC000F28E12000D0A53797374656D205365748C
:102AD00074696E67733A0A0D0A0D44656661756C18
:102AE000742043616D6572613A2025640A0D446566
:102AF0006661756C74205072657365743A20256444
:102B00000A0D0000F2CF0EF0F29EF76A220FF66E69
:102B10002B0EF722000EF86E0900F5500EBEF28E55
:102B200012000D0A54696C7453706565642020505E
:102B3000616E5370656564202049646C6520526540
:102B40007475726E202050616E656C204C696768E8
:102B500074730A0D0000F2CF0EF0F29EF76A740F44
:102B6000F66E2B0EF722000EF86E0900F5500EBE21
:102B7000F28E1200202020256420202020202020FA
:102B800020202564202020202020202020256420B3
:102B9000202020202020202020202025640A0D0A2B
:102BA0000D00F2CF0EF0F29EF76AC00FF66E2B0EFC
:102BB000F722000EF86E0900F5500EBEF28E1200DC
:102BC0000D0A4A6F79737469636B2053656E73697C
:102BD000746976697479202050616E202054696C84
:102BE00074202049646C65205A6F6E650A0D0000E0
:102BF000F2CF0EF0F29EF76A0E0FF66E2C0EF72251
:102C0000000EF86E0900F5500EBEF28E1200202064
:102C100020202020202020202020202020202020B4
:102C20002020202025642020202025642020202012
:102C3000202025640A0D0A0D0000F2CF0EF0F29E4E
:102C4000F76A580FF66E2C0EF722000EF86E090088
:102C5000F5500EBEF28E12002050616E2044697253
:102C6000656374696F6E20627920506F72743A20C8
:102C700031203220332034203520360A0D00F2CFA7
:102C80000EF0F29EF76A9C0FF66E2C0EF722000EE5
:102C9000F86E0900F5500EBEF28E120020202020A2
:102CA0002020202020202020202020202020202024
:102CB00020202020256320256320256320256320F4
:102CC00025632025630A0D00F2CF0EF0F29EF76A0D
:102CD000E60FF66E2C0EF722000EF86E0900F55086
:102CE0000EBEF28E12000D0A54696C742044697293
:102CF000656374696F6E20627920506F72743A2038
:102D000031203220332034203520360A0D00F2CF16
:102D10000EF0F29EF76A2C0FF66E2D0EF722000EC3
:102D2000F86E0900F5500EBEF28E12000A0D5072B8
:102D300065736574733A0A0D0A0D0000F2CF0EF048
:102D4000F29EF76A5A0FF66E2D0EF722000EF86EFD
:102D50000900F5500EBEF28E120043616D205072D4
:102D600065204D6F64656C202020202020202020CD
:102D7000202020202020202050616E202020546917
:102D80006C7420205A6F6F6D20466F63757320201E
:102D90004272696768746E6573730000F2CF0EF05B
:102DA000F29EF76ABA0FF66E2D0EF722000EF86E3D
:102DB0000900F5500EBEF28E1200205B4272696768
:102DC00068742C466F6375732C4157422C424C43F8
:102DD0005D0A0D0A0D00F2CF0EF0F29EF76AF40FB5
:102DE000F66E2D0EF722000EF86E0900F5500EBE9D
:102DF000F28E120020256420202025326420253107
:102E0000387320253258254C582020254C58202036
:102E1000254C582020254C582020202020254C5877
:102E20000000F2CF0EF0F29EF76A400FF66E2E0E03
:102E3000F722000EF86E0900F5500EBEF28E120059
:102E40002020202020202000F2CF0EF0F29EF76AF2
:102E5000660FF66E2E0EF722000EF86E0900F55082
:102E60000EBEF28E12004F6E202020202020000087
:102E7000F2CF0EF0F29EF76A8E0FF66E2E0EF7224C
:102E8000000EF86E0900F5500EBEF28E12004F666D
:102E90006620202020200000F2CF0EF0F29EF76A7C
:102EA000B60FF66E2E0EF722000EF86E0900F550E2
:102EB0000EBEF28E12004F6E202020200000F2CFB6
:102EC0000EF0F29EF76ADC0FF66E2E0EF722000E61
:102ED000F86E0900F5500EBEF28E12004F666620A5
:102EE00020200000F2CF0EF0F29EF76A020FF66E7D
:102EF0002F0EF722000EF86E0900F5500EBEF28E6E
:102F000012004F6E20202000F2CF0EF0F29EF76AE2
:102F1000260FF66E2F0EF722000EF86E0900F55000
:102F20000EBEF28E12004F6666202000F2CF0EF029
:102F3000F29EF76A4A0FF66E2F0EF722000EF86E19
:102F40000900F5500EBEF28E12004F6E0000F2CF57
:102F50000EF0F29EF76A6C0FF66E2F0EF722000E3F
:102F6000F86E0900F5500EBEF28E12004F66660034
:102F7000F2CF0EF0F29EF76A8E0FF66E2F0EF7224A
:102F8000000EF86E0900F5500EBEF28E12000A0D0A
:102F9000436F6D6D616E6420436F6D706C65746519
:102FA0000A0D3E00F2CF0EF0F29EF76AC20FF66EE7
:102FB0002F0EF722000EF86E0900F5500EBEF28EAD
:102FC00012000A0D43616D204D6F64656C0A0D009F
:102FD000F2CF0EF0F29EF76AEE0FF66E2F0EF7228A
:102FE000000EF86E0900F5500EBEF28E120020257C
:102FF0006420204E6F2043616D6572610A0D0000F0
:10300000F2CF0EF0F29EF76A1E0FF66E300EF72228
:10301000000EF86E0900F5500EBEF28E12000A0D79
:10302000203E0000F2CF0EF0F29EF76A420FF66EDD
:10303000300EF722000EF86E0900F5500EBEF28E2B
:1030400012003E2573204E6F7420466F756E640A21
:103050000D3E0000F2CF0EF0F29EF76A720FF66E90
:10306000300EF722000EF86E0900F5500EBEF28EFB
:1030700012000A0D3E204A53443730202D204A6F5B
:1030800079737469636B20536C6F772044373020F9
:103090004F66660A0D3E2000F2CF0EF0F29EF76AF0
:1030A000B60FF66E300EF722000EF86E0900F550DE
:1030B0000EBEF28E12000A0D3E204A5344373020D5
:1030C0002D204A6F79737469636B20536C6F77207E
:1030D000443730204F6E2C5761697454696D6528F0
:1030E0002575290A0D3E2000F2CF0EF0F29EF76AF8
:1030F000060FF66E310EF722000EF86E0900F5503D
:103100000EBEF28E12000A0D3E2043616D657261A3
:10311000202564204E6F7420617661696C61626C59
:10312000650A0D3E2000F2CF0EF0F29EF76A440FC2
:10313000F66E310EF722000EF86E0900F5500EBE45
:10314000F28E120020313A43726F737346616465E8
:103150000000F2CF0EF0F29EF76A700FF66E310E9D
:10316000F722000EF86E0900F5500EBEF28E120026
:1031700020323A486F72697A20523E4C0000F2CFFA
:103180000EF0F29EF76A9C0FF66E310EF722000EDB
:10319000F86E0900F5500EBEF28E120020333A4848
:1031A0006F72697A204C3E520000F2CF0EF0F29E10
:1031B000F76AC80FF66E310EF722000EF86E09009E
:1031C000F5500EBEF28E120020343A56657274200D
:1031D000543E4200F2CF0EF0F29EF76AF20FF66E06
:1031E000310EF722000EF86E0900F5500EBEF28E79
:1031F000120020353A5665727420423E5400F2CFD8
:103200000EF0F29EF76A1C0FF66E320EF722000ED9
:10321000F86E0900F5500EBEF28E120020363A43C9
:103220006F726E657220554C3E425200F2CF0EF026
:10323000F29EF76A4A0FF66E320EF722000EF86E13
:103240000900F5500EBEF28E120020373A436F721D
:103250006E65722042523E554C00F2CF0EF0F29E47
:10326000F76A780FF66E320EF722000EF86E09003C
:10327000F5500EBEF28E120020303A4E6F6E650091
:10328000F2CF0EF0F29EF76A9E0FF66E320EF72224
:10329000000EF86E0900F5500EBEF28E12000A0DF7
:1032A0003E205472616E53656C3D25730A0D3E20BD
:1032B0000000F2CF0EF0F29EF76AD00FF66E320EDB
:1032C000F722000EF86E0900F5500EBEF28E1200C5
:1032D0000A0D3E205472616E54696D653D2532645D
:1032E000207365630A0D3E200000F2CF0EF0F29EBF
:1032F000F76A080FF66E330EF722000EF86E09001B
:10330000F5500EBEF28E12000A0D3E20566964651D
:103310006F2056657273696F6E204669726D7761B2
:1033200072652825303258292C20536F66747761D6
:1033300072652825303258290A0D3E200000F2CF50
:103340000EF0F29EF76A5C0FF66E330EF722000E57
:10335000F86E0900F5500EBEF28E12000A0D3E20E6
:103360004A6F79737469636B204E65757472616C12
:10337000205A6F6E65202564200A0D3E2000F2CF92
:103380000EF0F29EF76A9C0FF66E330EF722000ED7
:10339000F86E0900F5500EBEF28E12000A0D3E20A6
:1033A000446973706C617920436F6C6F7242617213
:1033B00073206F6E2049646C6520446973706C6182
:1033C000790A0D3E2000F2CF0EF0F29EF76AE40F6C
:1033D000F66E330EF722000EF86E0900F5500EBEA1
:1033E000F28E12000A0D3E20446973706C617920E0
:1033F000426C61636B206F6E2049646C6520446988
:1034000073706C61790A0D3E2000F2CF0EF0F29ECF
:10341000F76A280FF66E340EF722000EF86E0900D8
:10342000F5500EBEF28E1200566964656F204D6F26
:103430006465206973200000F2CF0EF0F29EF76AF7
:10344000560FF66E340EF722000EF86E0900F55096
:103450000EBEF28E12000A0D3E204D61696E4F665F
:103460006654696D653D253264207365630A0D3EBF
:103470002000F2CF0EF0F29EF76A900FF66E340E37
:10348000F722000EF86E0900F5500EBEF28E120003
:103490000A0D3E2041637469766520566964656F44
:1034A00020466F726D6174206973204E5453430A35
:1034B0000D3E2000F2CF0EF0F29EF76AD20FF66EAC
:1034C000340EF722000EF86E0900F5500EBEF28E93
:1034D00012000A0D3E2041637469766520566964C6
:1034E000656F20466F726D61742069732050414C86
:1034F0000A0D3E200000F2CF0EF0F29EF76A140F84
:10350000F66E350EF722000EF86E0900F5500EBE6D
:10351000F28E12000A0D3E204163746976652056D2
:103520006964656F20466F726D61742069732075E0
:103530006E6B6E6F776E2028253278290A0D3E203B
:103540000000F2CF0EF0F29EF76A600FF66E350EB5
:10355000F722000EF86E0900F5500EBEF28E120032
:103560004F6E2043616D65726120496E69742C2035
:1035700073656E6420486F6D6520636F6D6D616E5D
:10358000640A0D3E2000F2CF0EF0F29EF76AA40FFF
:10359000F66E350EF722000EF86E0900F5500EBEDD
:1035A000F28E12004F6E2043616D65726120496E8C
:1035B00069742C2073656E64205072657365742085
:1035C000313220636F6D6D616E6420736571756556
:1035D0006E63650A0D3E2000F2CF0EF0F29EF76A90
:1035E000F60FF66E350EF722000EF86E0900F55054
:1035F0000EBEF28E12000A0D3E204A6F7973746976
:10360000636B2050616E2053656E736974697669CF
:103610007479202564200A0D3E200000F2CF0EF0C0
:10362000F29EF76A3A0FF66E360EF722000EF86E2B
:103630000900F5500EBEF28E12000A0D3E5365745D
:1036400044656661756C74202564200A0D3E200077
:10365000F2CF0EF0F29EF76A6E0FF66E360EF7227C
:10366000000EF86E0900F5500EBEF28E12000A0D23
:103670003E44656661756C7443616D202564200A63
:103680000D3E2000F2CF0EF0F29EF76AA20FF66E0A
:10369000360EF722000EF86E0900F5500EBEF28EBF
:1036A00012000A0D3E204175746F2053656C6563EE
:1036B0007420566964656F20466F726D617420696D
:1036C00073204F6E0A0D3E200000F2CF0EF0F29EE6
:1036D000F76AE80FF66E360EF722000EF86E090054
:1036E000F5500EBEF28E12000A0D3E204175746F29
:1036F0002053656C65637420566964656F20466F5E
:10370000726D6174206973204F66660A0D3E200059
:10371000F2CF0EF0F29EF76A2E0FF66E370EF722FA
:10372000000EF86E0900F5500EBEF28E12000A0D62
:103730003E204A6F79737469636B2054696C7420FE
:1037400053656E7369746976697479202564200AFB
:103750000D3E2000F2CF0EF0F29EF76A720FF66E69
:10376000370EF722000EF86E0900F5500EBEF28EED
:10377000120050726F636573732055313320254CEE
:103780005820254C580A0D00F2CF0EF0F29EF76A31
:10379000A60FF66E370EF722000EF86E0900F550F0
:1037A0000EBEF28E120050726F6365737320553136
:1037B0003420254C5820254C580A0D00F2CF0EF02D
:1037C000F29EF76ADA0FF66E370EF722000EF86EE9
:1037D0000900F5500EBEF28E1200202020507265B6
:1037E00076696577496E205043200000F2CF0EF0D5
:1037F000F29EF76A0A0FF66E380EF722000EF86E88
:103800000900F5500EBEF28E120020202050726585
:1038100076696577496E20302000F2CF0EF0F29E77
:10382000F76A380FF66E380EF722000EF86E0900B0
:10383000F5500EBEF28E12005072657669657749BA
:103840006E2025640A0D3E00F2CF0EF0F29EF76A5C
:10385000660FF66E380EF722000EF86E0900F5506E
:103860000EBEF28E120020202020205043204F75E3
:103870007470757420202000F2CF0EF0F29EF76A6B
:10388000960FF66E380EF722000EF86E0900F5500E
:103890000EBEF28E120020202020204D61696E495C
:1038A0006E20302020202000F2CF0EF0F29EF76A2A
:1038B000C60FF66E380EF722000EF86E0900F550AE
:1038C0000EBEF28E12004D61696E496E2025640AAB
:1038D0000D3E0000F2CF0EF0F29EF76AF20FF66E88
:1038E000380EF722000EF86E0900F5500EBEF28E6B
:1038F0001200202020202043616D2053656C203071
:1039000020202000F2CF0EF0F29EF76A220FF66E12
:10391000390EF722000EF86E0900F5500EBEF28E39
:10392000120043616D6572612025640A0D3E00003E
:10393000F2CF0EF0F29EF76A4E0FF66E390EF722B6
:10394000000EF86E0900F5500EBEF28E12002043F4
:10395000616D2053656C2030204E6F2043616D00F7
:10396000F2CF0EF0F29EF76A7E0FF66E390EF72256
:10397000000EF86E0900F5500EBEF28E1200507265
:103980006F636573732055313520254C5820254CC5
:10399000580A0D00F2CF0EF0F29EF76AB20FF66EE3
:1039A000390EF722000EF86E0900F5500EBEF28EA9
:1039B000120020496E2043616D2053746F726520A0
:1039C00030300000F2CF0EF0F29EF76AE20FF66E92
:1039D000390EF722000EF86E0900F5500EBEF28E79
:1039E0001200496E43616D2053746F726520256427
:1039F0000A0D3E00F2CF0EF0F29EF76A120FF66E3D
:103A00003A0EF722000EF86E0900F5500EBEF28E47
:103A10001200202052656164696E672043616D6504
:103A200072610000F2CF0EF0F29EF76A420FF66E5E
:103A30003A0EF722000EF86E0900F5500EBEF28E17
:103A40001200202053746F72696E67205072657384
:103A500065740000F2CF0EF0F29EF76A720FF66EF8
:103A60003A0EF722000EF86E0900F5500EBEF28EE7
:103A700012002053746F72652030302050726573CD
:103A800065740000F2CF0EF0F29EF76AA20FF66E98
:103A90003A0EF722000EF86E0900F5500EBEF28EB7
:103AA000120053746F72652025640A0D3E00F2CF38
:103AB0000EF0F29EF76ACC0FF66E3A0EF722000E69
:103AC000F86E0900F5500EBEF28E12002053746F8E
:103AD0007265203030204661696C65640000F2CF69
:103AE0000EF0F29EF76AFC0FF66E3A0EF722000E09
:103AF000F86E0900F5500EBEF28E120020496E20BD
:103B000043616D2050726573657420303020000071
:103B1000F2CF0EF0F29EF76A2E0FF66E3B0EF722F2
:103B2000000EF86E0900F5500EBEF28E12005072B3
:103B3000657365742025640A0D3E0000F2CF0EF017
:103B4000F29EF76A5A0FF66E3B0EF722000EF86EE1
:103B50000900F5500EBEF28E120020204C6F6164F9
:103B6000696E67205072657365740000F2CF0EF0C5
:103B7000F29EF76A8A0FF66E3B0EF722000EF86E81
:103B80000900F5500EBEF28E120020202050726502
:103B9000736574203030202020200000F2CF0EF01A
:103BA000F29EF76ABA0FF66E3B0EF722000EF86E21
:103BB0000900F5500EBEF28E1200202020507265D2
:103BC000736574203030204261640000F2CF0EF043
:103BD000F29EF76AEA0FF66E3B0EF722000EF86EC1
:103BE0000900F5500EBEF28E12002020204E6F20EC
:103BF000507265736574203030200000F2CF0EF0F3
:103C0000F29EF76A1A0FF66E3C0EF722000EF86E5F
:103C10000900F5500EBEF28E120020202050726571
:103C200076696577204F6E2020200000F2CF0EF0DD
:103C3000F29EF76A4A0FF66E3C0EF722000EF86EFF
:103C40000900F5500EBEF28E1200446973706C616B
:103C50007920507265766965770A0D3E0000F2CFD3
:103C60000EF0F29EF76A7C0FF66E3C0EF722000E05
:103C7000F86E0900F5500EBEF28E12002020205082
:103C8000726576696577204F666620200000F2CF66
:103C90000EF0F29EF76AAC0FF66E3C0EF722000EA5
:103CA000F86E0900F5500EBEF28E12004469737072
:103CB0006C6179204F66660A0D3E0000F2CF0EF06F
:103CC000F29EF76ADA0FF66E3C0EF722000EF86EDF
:103CD0000900F5500EBEF28E12002020204D6169C1
:103CE0006E204F6E20202000F2CF0EF0F29EF76A79
:103CF000060FF66E3D0EF722000EF86E0900F55025
:103D00000EBEF28E1200446973706C6179204D61B1
:103D1000696E0A0D3E00F2CF0EF0F29EF76A340F84
:103D2000F66E3D0EF722000EF86E0900F5500EBE3D
:103D3000F28E12002020204D61696E204F666620B1
:103D40002000F2CF0EF0F29EF76A600FF66E3D0E85
:103D5000F722000EF86E0900F5500EBEF28E12002A
:103D600050726F636573732055313620254C58208F
:103D7000254C580A0D00F2CF0EF0F29EF76A940F10
:103D8000F66E3D0EF722000EF86E0900F5500EBEDD
:103D9000F28E1200204261636B4C69676874436D58
:103DA00070204F666600F2CF0EF0F29EF76AC40FE5
:103DB000F66E3D0EF722000EF86E0900F5500EBEAD
:103DC000F28E1200424C43204F66660A0D3E000000
:103DD000F2CF0EF0F29EF76AEE0FF66E3D0EF7226E
:103DE000000EF86E0900F5500EBEF28E1200204251
:103DF00061636B4C69676874436D70204F6E20007F
:103E0000F2CF0EF0F29EF76A1E0FF66E3E0EF7220C
:103E1000000EF86E0900F5500EBEF28E1200424CF4
:103E200043204F6E0A0D3E00F2CF0EF0F29EF76A6D
:103E3000460FF66E3E0EF722000EF86E0900F550A2
:103E40000EBEF28E12002020204D61696E20456E5C
:103E500061626C6564200000F2CF0EF0F29EF76A9A
:103E6000760FF66E3E0EF722000EF86E0900F55042
:103E70000EBEF28E12002020204D61696E20446932
:103E80007361626C65642000F2CF0EF0F29EF76AF7
:103E9000A60FF66E3E0EF722000EF86E0900F550E2
:103EA0000EBEF28E12004D61696E496E20300A0D11
:103EB0003E00F2CF0EF0F29EF76AD00FF66E3E0E85
:103EC000F722000EF86E0900F5500EBEF28E1200B9
:103ED0002020537973204D616E75616C204D6F64A5
:103EE0006500F2CF0EF0F29EF76A000FF66E3F0EFD
:103EF000F722000EF86E0900F5500EBEF28E120089
:103F00005379734D6F6465204D616E75616C0A0D58
:103F10003E00F2CF0EF0F29EF76A300FF66E3F0EC3
:103F2000F722000EF86E0900F5500EBEF28E120058
:103F3000202020537973204175746F204D6F646584
:103F40002000F2CF0EF0F29EF76A600FF66E3F0E81
:103F5000F722000EF86E0900F5500EBEF28E120028
:103F60005379734D6F6465204175746F0A0D3E007F
:103F7000F2CF0EF0F29EF76A8E0FF66E3F0EF7222A
:103F8000000EF86E0900F5500EBEF28E1200506F52
:103F9000776572204F66660A0D3E0000F2CF0EF084
:103FA000F29EF76ABA0FF66E3F0EF722000EF86E19
:103FB0000900F5500EBEF28E1200506F7765722028
:103FC0004F6E0A0D3E00F2CF0EF0F29EF76AE40F3C
:103FD000F66E3F0EF722000EF86E0900F5500EBE89
:103FE000F28E120020204272696768746E657373E6
:103FF000205570202000F2CF0EF0F29EF76A140FC9
:10400000F66E400EF722000EF86E0900F5500EBE57
:10401000F28E12004272696768742055700A0D3E74
:104020000000F2CF0EF0F29EF76A400FF66E400EDF
:10403000F722000EF86E0900F5500EBEF28E120047
:1040400020204272696768746E65737320446E2025
:104050002000F2CF0EF0F29EF76A700FF66E400E5F
:10406000F722000EF86E0900F5500EBEF28E120017
:1040700042726967687420446F776E0A0D3E0000D3
:10408000F2CF0EF0F29EF76A9E0FF66E400EF72208
:10409000000EF86E0900F5500EBEF28E12002020C0
:1040A0004272696768746E657373204175746F003E
:1040B000F2CF0EF0F29EF76ACE0FF66E400EF722A8
:1040C000000EF86E0900F5500EBEF28E120042721C
:1040D00069676874204175746F0A0D3E0000F2CF65
:1040E0000EF0F29EF76AFC0FF66E400EF722000EFD
:1040F000F86E0900F5500EBEF28E120020204272BA
:10410000696768746E657373204D616E2000F2CF2D
:104110000EF0F29EF76A2C0FF66E410EF722000E9B
:10412000F86E0900F5500EBEF28E120042726967F9
:104130006874204D616E75616C0A0D3E0000F2CF0F
:104140000EF0F29EF76A5C0FF66E410EF722000E3B
:10415000F86E0900F5500EBEF28E120020202020CD
:10416000466F637573204E65617220202000F2CF88
:104170000EF0F29EF76A8C0FF66E410EF722000EDB
:10418000F86E0900F5500EBEF28E1200466F637590
:1041900073204E6561720A0D3E00F2CF0EF0F29E62
:1041A000F76AB80FF66E410EF722000EF86E09009E
:1041B000F5500EBEF28E120020202020466F63754F
:1041C00073204661722020200000F2CF0EF0F29E94
:1041D000F76AE80FF66E410EF722000EF86E09003E
:1041E000F5500EBEF28E1200466F63757320466165
:1041F000720A0D3E0000F2CF0EF0F29EF76A140F25
:10420000F66E420EF722000EF86E0900F5500EBE53
:10421000F28E120020202020466F637573204175B6
:10422000746F20200000F2CF0EF0F29EF76A440F68
:10423000F66E420EF722000EF86E0900F5500EBE23
:10424000F28E120020202020466F637573204D618E
:104250006E75616C0000F2CF0EF0F29EF76A740F7B
:10426000F66E420EF722000EF86E0900F5500EBEF3
:10427000F28E1200466F637573204175746F0A0DDC
:104280003E00F2CF0EF0F29EF76AA00FF66E420EDD
:10429000F722000EF86E0900F5500EBEF28E1200E5
:1042A000204175746F576869746542616C204F6670
:1042B0006600F2CF0EF0F29EF76AD00FF66E420E55
:1042C000F722000EF86E0900F5500EBEF28E1200B5
:1042D000415742204F66660A0D3E0000F2CF0EF0B5
:1042E000F29EF76AFA0FF66E420EF722000EF86E93
:1042F0000900F5500EBEF28E1200204175746F5702
:104300006869746542616C204F6E2000F2CF0EF038
:10431000F29EF76A2A0FF66E430EF722000EF86E31
:104320000900F5500EBEF28E1200415742204F6E2A
:104330000A0D3E00F2CF0EF0F29EF76A520FF66EB3
:10434000430EF722000EF86E0900F5500EBEF28EF5
:10435000120053746172742049646C652052657454
:1043600075726E2054696D65720D0A00F2CF0EF001
:10437000F29EF76A8A0FF66E430EF722000EF86E71
:104380000900F5500EBEF28E120020507265736562
:10439000742050474D204D6F64652000F2CF0EF021
:1043A000F29EF76ABA0FF66E430EF722000EF86E11
:1043B0000900F5500EBEF28E1200204C6F61646948
:1043C0006E6720507265736574313200F2CF0EF063
:1043D000F29EF76AEA0FF66E430EF722000EF86EB1
:1043E0000900F5500EBEF28E1200204E6F20507262
:1043F00065736574313220466F756E640000F2CFCC
:104400000EF0F29EF76A1C0FF66E440EF722000EB5
:10441000F86E0900F5500EBEF28E120053797374D7
:10442000656D206973204175746F0A0D0000F2CF2D
:104430000EF0F29EF76A4C0FF66E440EF722000E55
:10444000F86E0900F5500EBEF28E120053797374A7
:10445000656D2069732050414C0A0D00F2CF0EF0BB
:10446000F29EF76A7A0FF66E440EF722000EF86E8F
:104470000900F5500EBEF28E120053797374656D0B
:10448000206973204E5453430A0D0000F2CF0EF002
:10449000F29EF76AAA0FF66E440EF722000EF86E2F
:1044A0000900F5500EBEF28E1200436F6D3120529E
:1044B000656365697665204572726F722873293D60
:1044C0002532780A0D00F2CF0EF0F29EF76AE40F63
:1044D000F66E440EF722000EF86E0900F5500EBE7F
:1044E000F28E1200436F6D32205265636569766506
:1044F000204572726F722873293D2532780A0D00AB
:10450000F2CF0EF0F29EF76A1E0FF66E450EF722FE
:10451000000EF86E0900F5500EBEF28E12000C501F
:10452000726F64756374696F6E566965774658007B
:10453000F2CF0EF0F29EF76A4E0FF66E450EF7229E
:10454000000EF86E0900F5500EBEF28E12000A0041
:10455000F2CF0EF0F29EF76A6E0FF66E450EF7225E
:10456000000EF86E0900F5500EBEF28E12002020EB
:104570005374617274696E67205570202000F2CF09
:104580000EF0F29EF76A9C0FF66E450EF722000EB3
:10459000F86E0900F5500EBEF28E120043616D6593
:1045A0007261205061737320436F6D706C65746528
:1045B0000A0D0000F2CF0EF0F29EF76AD20FF66EEF
:1045C000450EF722000EF86E0900F5500EBEF28E71
:1045D000120043616D657261205061737320496EF2
:1045E000636F6D706C6574650A0D0000F2CF0EF09C
:1045F000F29EF76A0A0FF66E460EF722000EF86E6C
:104600000900F5500EBEF28E120043616D657261B5
:10461000204E6F7420417661696C61626C650A0D91
:104620000000F2CF0EF0F29EF76A400FF66E460ED3
:10463000F722000EF86E0900F5500EBEF28E120041
:1046400050726F64756374696F6E5669657746580A
:1046500025730A0D0000F2CF0EF0F29EF76A740F78
:10466000F66E460EF722000EF86E0900F5500EBEEB
:10467000F28E120020202020436F6D70696C6564FB
:104680003A2025732061742025730A0D3E00F2CF75
:104690000EF0F29EF76AAC0FF66E460EF722000E91
:1046A000F86E0900F5500EBEF28E12002046696EBB
:1046B00064696E672043616D657261730000F2CFBB
:1046C0000EF0F29EF76ADC0FF66E460EF722000E31
:1046D000F86E0900F5500EBEF28E120020436C6594
:1046E0006172696E6720416C6C2020200000F2CF5F
:1046F0000EF0F29EF76A0C0FF66E470EF722000ED0
:10470000F86E0900F5500EBEF28E1200446F44752B
:104710006D700000F2CF0EF0F29EF76A320FF66E67
:10472000470EF722000EF86E0900F5500EBEF28E0D
:104730001200456E61626C652053657269616C0A96
:104740000D00F2CF0EF0F29EF76A600FF66E470E84
:10475000F722000EF86E0900F5500EBEF28E120020
:1047600020204E6F74206F6E205072657365742028
:104770000000F2CF0EF0F29EF76A900FF66E470E31
:10478000F722000EF86E0900F5500EBEF28E1200F0
:10479000204C6F6164696E672044656661756C7456
:1047A0007300F2CF0EF0F29EF76AC00FF66E470E5E
:1047B000F722000EF86E0900F5500EBEF28E1200C0
:1047C0002020506F776572696E6720557020202019
:1047D0000000F2CF0EF0F29EF76AF00FF66E470E71
:1047E000F722000EF86E0900F5500EBEF28E120090
:1047F0000A2020506F776572696E6720446F776E6C
:104800002000C69E9E966ECEC9FF020EC6BE05D083
:104810009EA6FED7000EC5BC010E016E000CC69C04
:10482000C586C5B6FED700B0C59A00A0C58AC588A2
:10483000C5B8FED7C9CF01F0000C0E01696BC58069
:10484000C5B0FED70A0E006E002EFED700D067510D
:10485000FE0B6A6F6E6F0001D4DF0A0E006E002E31
:10486000FED700D068CE6EFECCDF0A0E006E002EA2
:10487000FED700D0C582C5B2FED70A0E006E002E4C
:10488000FED700D00E01675101096A6F6E6F0001FB
:10489000B8DF0A0E006E002EFED700D0006ABFDF20
:1048A00001C069FE0A0E006E002EFED700D0C5843E
:1048B000C5B4FED70D0E006E002EFED70E0169CED8
:1048C00001F00001000C0E01636B646B656B6251BB
:1048D000FE0B666F61CE67FE686F0001AEDF01C040
:1048E00065FE0E0162510109666F61CE67FE686F59
:1048F0000001A3DF01C064FE0E01636B6551631309
:1049000063CE01F064CE02F00001000C0E015F6B7B
:10491000606B4C80400E616F080E626F0001D3DF48
:1049200002C060FE01C05FFEF292DEEF03F00E01F6
:104930005F6B606B4C82440E616F080E626F00010A
:10494000C2DF02C060FE01C05FFEF092DEEF03F046
:104950000E015F6B606B4C84420E616F080E626FDC
:104960000001B1DF02C060FE01C05FFEF090DEEF2B
:1049700003F00E015F6B606B4C86460E616F080E94
:10498000626F0001A0DF02C060FE01C05FFEF09414
:10499000DEEF03F00E016251016A615D03E261CE58
:1049A00000F00CD0006A080E636F61370036625168
:1049B000005CD8B0006E0136632FF7D70001000C01
:1049C00001012151040DF3500E01606B5F6F036A0A
:1049D000010131510E015F25016E6051032201502A
:1049E000250FE96E010E0320EA6EC282C2B2FED725
:1049F000C4CFEFFF01012151040DF3500E01606B94
:104A00005F6F036A010131510E015F25016E605134
:104A100003220150250FE96E010E0320EA6EEF50CC
:104A20007B0827E201012151040DF3500E01606B58
:104A30005F6F036A010131510E015F25016E605104
:104A400003220150250FE96E010E0320EA6EEF509C
:104A500084080FE3D89001012135036A320FE96E13
:104A6000010E0320EA6EEC6AED52800EEF6E77D0F5
:104A70000E01D89001012135036A320F016E010E3B
:104A8000032201C05FFE03C060FE01012151040D3D
:104A9000F3500E01626B616F250E6125E96E010E08
:104AA0006221EA6EEF50626B616F01012151040DCA
:104AB000F3500E01646B636F010E6325016E000EEF
:104AC0006421036E0150250FE96E010E0320EA6E8A
:104AD000EF50036A61270350622301012151040D45
:104AE000F3500E01646B636F020E6325016E000EBE
:104AF0006421036E0150250FE96E010E0320EA6E5A
:104B0000EF50036A61270350622301012151040D14
:104B1000F3500E01646B636F030E6325016E000E8C
:104B20006421036E0150250FE96E010E0320EA6E29
:104B3000EF50036A6127035062236231036E6131D3
:104B4000026E033202323F0E031660CEEAFF5FCEE2
:104B5000E9FF03C0ECFFED5202C0EFFF0101010EBF
:104B60003125030B316F010E21250E01606F616F3E
:104B7000030E626F00010EDF00C021F1010121353B
:104B8000006E0036FC0E0016C250C30B0010C26E41
:104B90005D2E1FD05C2A5E2A1B0E5D6E5BA80FD0B7
:104BA0000001600760530AE15B983BC190F13CC192
:104BB00091F13BC18FF14A804A82498C010158BE74
:104BC00002D05BA006D05E50030803E2589E5B90C3
:104BD000458A9E900001DEEF03F0F294DEEF03F0D1
:104BE000C580C5B0FED70A0E006E002EFED700D0DD
:104BF0000E016A51FE0B6D6F6E6F000102DE0A0E30
:104C0000006E002EFED700D06BCE6EFEFADD0A0ECF
:104C1000006E002EFED700D06CCE6EFEF2DD0A0EC6
:104C2000006E002EFED700D0C584C5B4FED70D0E91
:104C3000006E002EFED7000C0E0164510109676F53
:104C400066CE68FE696B696B63CE6AFE6B6F66CE7B
:104C50006CFE0001C5DF0E016451FE0B676F65CE6F
:104C600068FE696B63CE6AFE6B6F65CE6CFE0001F9
:104C7000B7DF000C0E01646B656B010E635DF40F12
:104C800051E20C0F000198EF26F00E01656B080E43
:104C9000646F48D00E01656B040E646F43D0010150
:104CA00038A105D00E01656B010E646F04D00E01B2
:104CB000656B020E646F36D0010138A105D00E017C
:104CC000656B020E646F04D00E01656B010E646F9C
:104CD00029D0800E0E01656F646B24D0400E0E014A
:104CE000656F646B1FD0200E0E01656F646B1AD068
:104CF000100E0E01656F646B15D0080E0E01656F06
:104D0000646B10D0040E0E01656F646B0BD0020E45
:104D10000E01656F646B06D0010E0E01656F646B4A
:104D200001D00E0164CE01F065CE02F00001000C4E
:104D300008AE03D0F2CF0EF0F29EE824F76AF73601
:104D4000630FF66E4D0EF722000EF86EFB6E0A0032
:104D5000F550FA6E0800F55008AE02D00EBEF28E85
:104D6000F96E184D0E4D044DFA4CF04CE64CDC4CEF
:104D7000D24CB84C9E4C944C8A4C0E01646B656BC3
:104D8000635102080EE3010E635D006E400E646F16
:104D9000656B005205E0D89064376537002EFBD76D
:104DA00021D0635104080EE3030E635D006E400ED4
:104DB000656F646B005205E0D89064376537002E4C
:104DC000FBD710D0635106080DE3050E635D006E3E
:104DD000400E646F656B005205E0D890643765370C
:104DE000002EFBD764CE01F065CE02F00001000C6E
:104DF0000E015F6B606B616B626B58AA03D0589CAD
:104E0000A08281D1A092588C58A060D04F504D14F0
:104E1000636F50504E14646F635304E1645302E1B6
:104E200058A20BD04D50FF0A006E4E50FF0A036E81
:104E300000504F160350501604D04D504F124E5094
:104E400050125150010A000105E0030A0EE0010A68
:104E50001AE024D04C0E0E01636F646B50C066FEE6
:104E60004FC065FE0001E8DE1BD050C063FE0E019E
:104E7000646B646B480E6A6F010E6B6F50C06CFE02
:104E80000001AEDE0DD04A0E0E01636F646B50C0A0
:104E900066FE4FC065FE0001CFDE02D0588200D012
:104EA00058A205D0516A506A4F6A5890589258A03B
:104EB00006D0A082589C0E0126D108D0000158B41B
:104EC00006D0589C589458960E011DD1000158A642
:104ED00007D0589458960E015F6B596A14D100019F
:104EE00058A40ED15952D8B40BD10E015F6B59C0E2
:104EF00062FE62510C080EE3036A6251D70FE96E3D
:104F0000010E0320EA6EEF5203E162CE5FFE02D093
:104F1000622BEFD75F5318E1592C01D015D0010E49
:104F2000596E59C062FE62510C080EE3036A625169
:104F3000D70FE96E010E0320EA6EEF5203E162CE55
:104F40005FFE02D0622BEFD75F53D8B475D0FF0E4F
:104F5000521A531A300E5216536A5F515A5C02E1CC
:104F6000587801D0589858B808D05FCE63FE000139
:104F700081DE01505212025053128AC163FE0001B9
:104F8000FCDE02C061FE01C060FE01018A51020820
:104F90001AE30E0160515614636F61515714646F28
:104FA00063530BE1645309E1605152126151531292
:104FB000605156126151571204D03F0E5216576A73
:104FC000566A27D00101FF0E541A551A54500E018B
:104FD0006015636F55506115646F63530AE1645344
:104FE00008E13F0E54165516605154126151551286
:104FF00003D03F0E54165516FF0E541A551A4A0E7A
:10500000636F646B55C066FE54C065FE000114DE1C
:105010000E01FF0E521A531A4C0E636F646B53C08D
:1050200066FE52C065FE000107DE5FCE5AF0010E3B
:105030000E015F25596E5ED0592C5CD0FF0E521ABE
:10504000531AF00E5216536A8AC163FE000195DEB0
:1050500002C061FE01C060FE01018A51020824E322
:1050600052500E016015636F53506115646F6353A6
:105070000AE1645308E1300E5216536A605152122D
:105080006151531203D0300E5216536AFF0E521A5A
:10509000531A4C0E636F646B53C066FE52C065FEBC
:1050A0000001CADD26D00101FF0E541A551A5450D2
:1050B0000E016015636F55506115646F63530AE10B
:1050C000645308E13F0E5416551660515412615155
:1050D000551203D03F0E54165516FF0E541A551A8A
:1050E0004A0E636F646B55C066FE54C065FE0001D6
:1050F000A3DD0E0162510C0802E2010E596E00019F
:10510000589CA0820E01A1920001DEEF03F0036A19
:105110006151680FE96E000E0320EA6E9EAAFED769
:10512000AECFEFFF036A6151680FE96E000E0320F6
:10513000EA6E6751EF5C01E1662B010E61253F0BC2
:10514000616F5B9E01013ABD04D061C063F05B8C6E
:1051500001D05B9C9E9A0001DEEF03F0036A62516E
:10516000A90FE96E000E0320EA6EA4AAFED76ECF47
:10517000EFFF010E62250E01606F616F780E626FA6
:10518000000108DC00C062F0A891A49ADEEF03F0F1
:10519000080EEA6E650EE96EEF500EE0050E016E28
:1051A000006A002EFED7012EFBD72E0E006E002EB9
:1051B000FED700D0EF2EF2D7000C080EEA6EA80E34
:1051C000E96EEF500EE0050E016E006A002EFED76C
:1051D000012EFBD72E0E006E002EFED700D0EF2E34
:1051E000F2D7000C0801AD39F00B006E0F0E8C14D5
:1051F00000108C6E00008C80020E006E002EFED718
:1052000000008C900001000C8350006E00380F0BE2
:10521000016E000C0F0E9514F009956E8C84000041
:105220008C800000F1DF01C0ADF88C9000008C8014
:1052300000D000D0E9DF01C0ACF88C900F0E9514BF
:10524000956E0801AD39006EF00E00160050AC11DD
:10525000016E00012EEF29F08C92DCD701C0ACF872
:10526000080101AE02D00001F8D78C92AAB18C825D
:1052700000008C9400008C90AB39AC6F0F0EAC1713
:10528000ACC8ADF80001AEDF0801AB510F0BAC6F3D
:10529000AD6F0001A7DF000C0F0E9514956E959071
:1052A000959295948C928C948C900F0E0801A86F17
:1052B000000183DF010E0401646F645103080DE3F4
:1052C000030E0801AD6F00018DDF050E0801A86F08
:1052D000000173DF0401642BF0D7020E0801AD6FEB
:1052E000000180DF0401646B6451030814E3036A66
:1052F0006451F2CF65F4F29E000103EC04F0040166
:1053000065BFF28E656F0801AA6BAB6F0001A4DF69
:105310000401642BE9D700010DEFEEF0A5C8A7F852
:10532000A4C8A6F8A7C803F00801A6C8E9FFA7C843
:10533000EAFFEF5206E0A62BD8B4A72B0001F2D764
:105340000801A451A65D006EA551A759036E00C0C7
:1053500001F00001000C0801A72D01D003D0400E80
:10536000A86F01D0A86B010EA65DA827A8518009DF
:10537000A96FAA6BAB6F00016FDF000C0801A5518C
:105380000C0A000105E0060A0FE0020A15E01BD036
:105390000801AA6B010EAB6F00015EDF020E08016F
:1053A000A86F00010ADF17D0010E0801A66F020ED8
:1053B000A76F0001D0DF0FD00801AA6B100EAB6FF2
:1053C00000014ADF08D0010E0801AA6FA5C8ABF89A
:1053D000000142DF00D0000C0801A36BA2C8A5F8B1
:1053E000A1C8A4F800019ADF0152D8B48ED0A2C897
:1053F000A5F8A1C8A4F892DF01500801A35DD8B0B8
:1054000085D0036AA351A125E96EA2510320EA6E5B
:10541000EF50010A00010DE0030A26E0010A3FE017
:10542000080A58E0070A5EE0060A5CE0020A5AE051
:1054300059D00801A35317E1010EA66FA76F000111
:105440008ADF200E0801A56F000198DF010E080118
:10545000A66F020EA76F00017EDF200E0801A56F68
:1054600000018CDF08014ED00801A35317E1010EA3
:10547000A66FA76F00016FDF3E0E0801A56F000148
:105480007DDF010E0801A66F020EA76F000163DF2A
:10549000200E0801A56F000171DF080133D008015B
:1054A000A35317E1010EA66FA76F000154DF200E72
:1054B0000801A56F000162DF010E0801A66F020E50
:1054C000A76F000148DF3E0E0801A56F000156DFFF
:1054D000080118D0010E0801A66FA76F00013BDF7D
:1054E000080110D0036A0801A351A125E96EA25159
:1054F0000320EA6EEFCFA4F8A4C8A5F800013EDFB0
:10550000080100D0A32B000172D708010001000C94
:10551000010E016E4FEFEEF0196AF2BE198EF29E87
:105520004C0E0E01636F040E646F666B656B0001B9
:105530001CEC26F019BEF28E196AF2BE198EF29E8C
:105540004C0E0E01636F060E646F666B656B000197
:105550001CEC26F019BEF28E196AF2BE198EF29E6C
:105560004C0E0E016A6F0B0E6B6F6C6B0001F0EC52
:1055700025F019BEF28E196AF2BE198EF29E480EFF
:105580000E01636F040E646F666B656B00011CECAB
:1055900026F019BEF28E196AF2BE198EF29E480EDE
:1055A0000E01636F060E646F666B656B00011CEC89
:1055B00026F019BEF28E196AF2BE198EF29E480EBE
:1055C0000E016A6F0A0E6B6F6C6B0001F0EC25F038
:1055D00019BEF28E196AF2BE198EF29E4A0E0E01A3
:1055E000636F040E646F666B656B00011CEC26F044
:1055F00019BEF28E196AF2BE198EF29E4A0E0E0183
:10560000636F060E646F666B656B00011CEC26F021
:1056100019BEF28E196AF2BE198EF29E4A0E0E0162
:105620006A6F0A0E6B6F6C6B0001F0EC25F019BE0F
:10563000F28E196AF2BE198EF29E4E0E0E01636F43
:10564000040E646F666B656B00011CEC26F019BEDE
:10565000F28E196AF2BE198EF29E4E0E0E01636F23
:10566000060E646F666B656B00011CEC26F019BEBC
:10567000F28E196AF2BE198EF29E4E0E0E016A6FFC
:105680000A0E6B6F6C6B0001F0EC25F019BEF28E08
:10569000196AF2BE198EF29E400E0E01636F040E5F
:1056A000646F666B656B00011CEC26F019BEF28E10
:1056B000196AF2BE198EF29E400E0E01636F060E3D
:1056C000646FFF0E666F656F00011CEC26F019BE5B
:1056D000F28E196AF2BE198EF29E400E0E016A6FAA
:1056E0000A0E6B6F6C6B0001F0EC25F019BEF28EA8
:1056F000196AF2BE198EF29E440E0E01636F040EFB
:10570000646F666B656B00011CEC26F019BEF28EAF
:10571000196AF2BE198EF29E440E0E01636F060ED8
:10572000646FFF0E666F656F00011CEC26F019BEFA
:10573000F28E196AF2BE198EF29E440E0E016A6F45
:105740000A0E6B6F6C6B0001F0EC25F019BEF28E47
:10575000196AF2BE198EF29E420E0E01636F040E9C
:10576000646F666B656B00011CEC26F019BEF28E4F
:10577000196AF2BE198EF29E420E0E01636F060E7A
:10578000646FFF0E666F656F00011CEC26F019BE9A
:10579000F28E196AF2BE198EF29E420E0E016A6FE7
:1057A0000A0E6B6F6C6B0001F0EC25F019BEF28EE7
:1057B000196AF2BE198EF29E460E0E01636F040E38
:1057C000646F666B656B00011CEC26F019BEF28EEF
:1057D000196AF2BE198EF29E460E0E01636F060E16
:1057E000646FFF0E666F656F00011CEC26F019BE3A
:1057F000F28E196AF2BE198EF29E460E0E016A6F83
:105800000A0E6B6F6C6B0001F0EC25F019BEF28E86
:10581000000C9EA8FED7AD6E000C0401646BF2CFA5
:1058200065F4F29EAA6A070EA96EA69CA69EA680A3
:10583000A85065BFF28E646F64AB16D0010139A524
:105840000FD00401656B65510001FFEC21F00401EC
:10585000652B0001DEDF100E0401655DF4E101013E
:10586000000E016E2FD0040164A317D0010139A5E9
:105870000FD00401656B6551000117EC22F00401A3
:10588000652B0001C6DF0F0E0401655DF4E1010127
:10589000020E016E17D016D00401010139A50FD0F8
:1058A0000401656B655100012EEC22F00401652BAB
:1058B0000001AFDF100E0401655DF4E10101010E8E
:1058C000016E00D00001000C04019851010A000192
:1058D0000DE0030AD8B40ED1010AD8B483D1070A67
:1058E000D8B448D2040AD8B40DD30CD3010EEA6E52
:1058F000E40EE96EF2CF99F4F29E000EC0EC08F0CF
:105900000A000900F550EE6E0009FBE1040199BFA1
:10591000F28E010EEA6EF60EE96EF2CF99F4F29E67
:10592000000E0001D8EC08F00A000900F550EE6EF8
:105930000009FBE1040199BFF28E020EEA6E080E27
:10594000E96EF2CF99F4F29E000E0001F0EC08F03F
:105950000A000900F550EE6E0009FBE1040199BF51
:10596000F28E020EEA6E1A0EE96EF2CF99F4F29EF2
:10597000000E000108EC09F00A000900F550EE6E77
:105980000009FBE1040199BFF28E020EEA6E2C0EB3
:10599000E96EF2CF99F4F29E000E000120EC09F0BE
:1059A0000A000900F550EE6E0009FBE1040199BF01
:1059B000F28E020EEA6E3E0EE96EF2CF99F4F29E7E
:1059C000000E000138EC09F00A000900F550EE6EF7
:1059D0000009FBE1040199BFF28E020EEA6E500E3F
:1059E000E96EF2CF99F4F29E000E000150EC09F03E
:1059F0000A000900F550EE6E0009FBE1040199BFB1
:105A0000F28E020EEA6E620EE96EF2CF99F4F29E09
:105A1000000E000168EC09F00A000900F550EE6E76
:105A20000009FBE1040199BFF28E020EEA6E740ECA
:105A3000E96EF2CF99F4F29E000E000180EC09F0BD
:105A40000A000900F550EE6E0009FBE1040199BF60
:105A5000F28E020EEA6E860EE96EF2CF99F4F29E95
:105A6000000E000198EC09F00A000900F550EE6EF6
:105A70000009FBE1040199BFF28E020EEA6E980E56
:105A8000E96EF2CF99F4F29E000E0001B0EC09F03D
:105A90000A000900F550EE6E0009FBE1040199BF10
:105AA000F28E020EEA6EAA0EE96EF2CF99F4F29E21
:105AB000000E0001C8EC09F00A000900F550EE6E76
:105AC0000009FBE1040199BFF28E010E03015E6F34
:105AD000036A5E51690FE96E030E0320EA6E0B0E36
:105AE000EF6E036A5E516E0FE96E030E0320EA6EDD
:105AF000EF6AF9D2010EEA6EE40EE96EF2CF99F484
:105B0000F29E000EE0EC09F00A000900F550EE6E7E
:105B10000009FBE1040199BFF28E010EEA6EF60E58
:105B2000E96EF2CF99F4F29E000E0001F8EC09F054
:105B30000A000900F550EE6E0009FBE1040199BF6F
:105B4000F28E020EEA6E080EE96EF2CF99F4F29E22
:105B5000000E000110EC0AF00A000900F550EE6E8C
:105B60000009FBE1040199BFF28E020EEA6E1A0EE3
:105B7000E96EF2CF99F4F29E000E000128EC0AF0D3
:105B80000A000900F550EE6E0009FBE1040199BF1F
:105B9000F28E020EEA6E2C0EE96EF2CF99F4F29EAE
:105BA000000E0001C8EC09F00A000900F550EE6E85
:105BB0000009FBE1040199BFF28E020E03015E6F42
:105BC000036A5E51690FE96E030E0320EA6E040E4C
:105BD000EF6E036A5E516E0FE96E030E0320EA6EEC
:105BE000EF6A81D2010EEA6EE40EE96EF2CF99F40B
:105BF000F29E000E40EC0AF00A000900F550EE6E2D
:105C00000009FBE1040199BFF28E010EEA6EF60E67
:105C1000E96EF2CF99F4F29E000E000158EC0AF002
:105C20000A000900F550EE6E0009FBE1040199BF7E
:105C3000F28E020EEA6E080EE96EF2CF99F4F29E31
:105C4000000E000170EC0AF00A000900F550EE6E3B
:105C50000009FBE1040199BFF28E020EEA6E1A0EF2
:105C6000E96EF2CF99F4F29E000E000188EC0AF082
:105C70000A000900F550EE6E0009FBE1040199BF2E
:105C8000F28E020EEA6E2C0EE96EF2CF99F4F29EBD
:105C9000000E0001A0EC0AF00A000900F550EE6EBB
:105CA0000009FBE1040199BFF28E020EEA6E3E0E7E
:105CB000E96EF2CF99F4F29E000E0001B8EC0AF002
:105CC0000A000900F550EE6E0009FBE1040199BFDE
:105CD000F28E020EEA6E500EE96EF2CF99F4F29E49
:105CE000000E0001D0EC0AF00A000900F550EE6E3B
:105CF0000009FBE1040199BFF28E020EEA6E620E0A
:105D0000E96EF2CF99F4F29E000E0001E8EC0AF081
:105D10000A000900F550EE6E0009FBE1040199BF8D
:105D2000F28E020EEA6E740EE96EF2CF99F4F29ED4
:105D3000000E0001C8EC09F00A000900F550EE6EF3
:105D40000009FBE1040199BFF28E030E03015E6FAF
:105D5000036A5E51690FE96E030E0320EA6E080EB6
:105D6000EF6E036A5E516E0FE96E030E0320EA6E5A
:105D7000EF6AB9D1010EEA6EE40EE96EF2CF99F442
:105D8000F29E000E00EC0BF00A000900F550EE6EDA
:105D90000009FBE1040199BFF28E010EEA6EF60ED6
:105DA000E96EF2CF99F4F29E000E000158EC0AF071
:105DB0000A000900F550EE6E0009FBE1040199BFED
:105DC000F28E020EEA6E080EE96EF2CF99F4F29EA0
:105DD000000E000170EC0AF00A000900F550EE6EAA
:105DE0000009FBE1040199BFF28E020EEA6E1A0E61
:105DF000E96EF2CF99F4F29E000E000188EC0AF0F1
:105E00000A000900F550EE6E0009FBE1040199BF9C
:105E1000F28E020EEA6E2C0EE96EF2CF99F4F29E2B
:105E2000000E0001A0EC0AF00A000900F550EE6E29
:105E30000009FBE1040199BFF28E020EEA6E3E0EEC
:105E4000E96EF2CF99F4F29E000E0001B8EC0AF070
:105E50000A000900F550EE6E0009FBE1040199BF4C
:105E6000F28E020EEA6E500EE96EF2CF99F4F29EB7
:105E7000000E0001D0EC0AF00A000900F550EE6EA9
:105E80000009FBE1040199BFF28E020EEA6E620E78
:105E9000E96EF2CF99F4F29E000E0001E8EC0AF0F0
:105EA0000A000900F550EE6E0009FBE1040199BFFC
:105EB000F28E020EEA6E740EE96EF2CF99F4F29E43
:105EC000000E0001C8EC09F00A000900F550EE6E62
:105ED0000009FBE1040199BFF28E040E03015E6F1D
:105EE000036A5E51690FE96E030E0320EA6E080E25
:105EF000EF6E036A5E516E0FE96E030E0320EA6EC9
:105F0000EF6AF1D0010EEA6EE40EE96EE26A320E3B
:105F1000E16EE752E6CFEEFFFCE1010EEA6EF60E0F
:105F2000E96EE26A200EE16EE752E6CFEEFFFCE199
:105F3000020EEA6E080EE96EF2CF99F4F29E000EA0
:105F4000E0EC09F00A000900F550EE6E0009FBE1F3
:105F5000040199BFF28E020EEA6E1A0EE96EF2CFBC
:105F600099F4F29E000E000118EC0BF00A000900F3
:105F7000F550EE6E0009FBE1040199BFF28E020EAE
:105F8000EA6E2C0EE96EF2CF99F4F29E000E00013B
:105F900030EC0BF00A000900F550EE6E0009FBE151
:105FA000040199BFF28E020EEA6E3E0EE96EF2CF48
:105FB00099F4F29E000E000148EC0BF00A00090073
:105FC000F550EE6E0009FBE1040199BFF28E020E5E
:105FD000EA6E500EE96EF2CF99F4F29E000E0001C7
:105FE00060EC0BF00A000900F550EE6E0009FBE1D1
:105FF000040199BFF28E020EEA6E620EE96EF2CFD4
:1060000099F4F29E000E000178EC0BF00A000900F2
:10601000F550EE6E0009FBE1040199BFF28E020E0D
:10602000EA6E740EE96EF2CF99F4F29E000E000152
:1060300090EC0BF00A000900F550EE6E0009FBE150
:10604000040199BFF28E020EEA6E860EE96EF2CF5F
:1060500099F4F29E000E0001A8EC0BF00A00090072
:10606000F550EE6E0009FBE1040199BFF28E020EBD
:10607000EA6E980EE96EF2CF99F4F29E000E0001DE
:10608000C0EC0BF00A000900F550EE6E0009FBE1D0
:10609000040199BFF28E020EEA6EAA0EE96EF2CFEB
:1060A00099F4F29E000E000140EC0AF00A0009008B
:1060B000F550EE6E0009FBE1040199BFF28E030179
:1060C0005E6B036A5E51690FE96E030E0320EA6E90
:1060D000130EEF6E036A5E516E0FE96E030E03201E
:1060E000EA6EEF6A00D00001000C0801A26703D03D
:1060F000A36702D007D0A32BA1C8EEFFA22FFCD725
:10610000A32FFAD70001000CA2C8A7F8A1C8A6F8CF
:106110000801A55324E0A4C803F0A3C8E9FFA4C85C
:10612000EAFFEF521CE0A7C803F0A651A62BD8B493
:10613000A72BA86F03C0A9F8A4C803F0A351A32BF1
:10614000D8B4A42BE96E03C0EAFFEFCFAAF8A9C820
:10615000EAFFA8C8E9FFAAC8EFFFA507DAD7A55349
:106160000CE0A7C803F0A651A62BD8B4A72BE96E64
:1061700003C0EAFFEF6AA507F2D7A1C801F0A2C8E1
:1061800002F00001000CA8B360D0080EEA6E7B0E8E
:10619000E96E0801A16BA36B130EA26F0001A5DFCE
:1061A000A8A936D004014AA304D04AA502D0000110
:1061B0002FD0010138A516D0080EEA6E7B0EE96ECD
:1061C000F2CFA1F8F29E000E00019FEC0EF00A0043
:1061D0000900F550EE6E0009FBE10801A1BFF28E47
:1061E00015D00101080EEA6E7B0EE96EF2CFA1F820
:1061F000F29E000E0001B7EC0EF00A000900F55007
:10620000EE6E0009FBE10801A1BFF28E0FD0000184
:10621000080E0801A26F7B0EA16F010EA46FE40EA1
:10622000A36F120EA56F00016FDF08010C0E7B6FCC
:10623000080EA26F7B0EA16F0001ECEC29F0050E99
:106240000801A86F0001DDEC28F0080EEA6E8E0E42
:10625000E96E0801A16BA36B130EA26F000145DF6D
:10626000080E0801A26F8E0EA16F7AC8A4F879C833
:10627000A3F8120EA56F000147DF0A0E08018E6F0A
:10628000080EA26F8E0EA16F0001ECEC29F0000C3D
:10629000040179C4E9FF7AC4EAFFEFCF7DF47CC43E
:1062A00003F07BC4E9FF7CC4EAFFEF507D5D15E19C
:1062B0007AC403F079C4E9FF03C0EAFFEF5203E1B7
:1062C000000E016E1FD07AC403F07951792BD8B437
:1062D0007A2B7B2BD8B47C2BDCD77AC403F079C41F
:1062E000E9FF7AC4EAFFEFCF7DF47CC403F07BC4FE
:1062F000E9FF7CC4EAFFEF507D5D02E2FF0E01D0B2
:10630000010E016E0001C8EF31F00401646B656B92
:10631000666B200E676F686F696F6A6F6B6F6C6F6B
:106320006D6F6E6F6F6F706F716F726F736F746F71
:10633000756F766F776F786B030E666FE70E656F1C
:10634000646B645111081BE3036A6451670FE96EC3
:10635000040E0320EA6EF2CF7BF4F29E66C4AAFF1D
:1063600065C4A9FFA69CA69EA680A8507BBFF28EFE
:10637000EF6E010E6527000E6623642BE2D7040E34
:106380007A6F670E796F7C6B320E7B6F000180D75E
:10639000015204E1010E016E04D003D0000E016E23
:1063A00000D066EFF0F004017D6B7E6B7F6BF2CF67
:1063B00080F4F29E030EAA6EFF0EA96EA69CA69E06
:1063C000A680A85080BFF28E7F6F7E6B7D6B7E5162
:1063D00003081CE37EC4AAFF7DC4A9FFFF0EA86EBC
:1063E000A69CA69EA684F2CF00F0F29E0F01550E49
:1063F000A76EAA0EA76EA682A6B2FED7A6940050DC
:10640000F21204017D2BD8B47E2BE1D77F51010815
:1064100019E3030EAA6EFF0EA96E7FC4A8FFA69C07
:10642000A69EA684F2CF00F0F29E0F01550EA76E35
:10643000AA0EA76EA682A6B2FED7A6940050F212AC
:1064400017D00401030EAA6EFF0EA96EA86AA69CBF
:10645000A69EA684F2CF00F0F29E0F01550EA76E05
:10646000AA0EA76EA682A6B2FED7A6940050F2127C
:1064700000018DEF32F00401966B976B986B996B6E
:106480009A6B976B200E966F986B985105082DE3C9
:10649000996B99510B0827E39A6B9A510B0821E3EA
:1064A00097C403F09651962BD8B4972B9B6F03C0DB
:1064B0009CF403C0AAFFA96EA86AA69CA69EA68407
:1064C000F2CF00F0F29E0F01550EA76EAA0EA76E36
:1064D000A682A6B2FED7A6940050F21204019A2B0F
:1064E000DCD7992BD6D7982BD0D7986B98510C081E
:1064F0000AE3036A9851D70FE96E010E0320EA6E92
:10650000EF6A982BF3D70001000C0401786B796BCC
:106510007A6B7B6B7C6B000146D7AA6AA96A010E75
:10652000A86EA69CA69EA684F2CF00F0F29E0F0154
:10653000550EA76EAA0EA76EA682A6B2FED7A69487
:106540000050F212AA6A010EA96EA86EA69CA69E21
:10655000A684F2CF00F0F29E550EA76EAA0EA76E8B
:10656000A682A6B2FED7A6940050F212AA6A020E24
:10657000A96E0F0EA86EA69CA69EA684F2CF00F070
:10658000F29E550EA76EAA0EA76EA682A6B2FED7E1
:10659000A6940050F212AA6A030EA96E120EA86EFB
:1065A000A69CA69EA684F2CF00F0F29E550EA76E82
:1065B000AA0EA76EA682A6B2FED7A6940050F2122B
:1065C000AA6A040EA96EA86EA69CA69EA684F2CF07
:1065D00000F0F29E550EA76EAA0EA76EA682A6B276
:1065E000FED7A6940050F212AA6A050EA96E0A0EF2
:1065F000A86EA69CA69EA684F2CF00F0F29E550E31
:10660000A76EAA0EA76EA682A6B2FED7A6940050C9
:10661000F212AA6A060EA96E600EA86EA69CA69E2D
:10662000A684F2CF00F0F29E550EA76EAA0EA76EBA
:10663000A682A6B2FED7A6940050F212AA6A070E4E
:10664000A96EA86AA69CA69EA684F2CF00F0F29E30
:10665000550EA76EAA0EA76EA682A6B2FED7A69466
:106660000050F212F2CF7DF4F29E030EAA6EFF0EDE
:10667000A96EA69CA69EA680A85004017DBFF28E9E
:106680007E6FAA6A080EA96E7EC4A8FFA69CA69E6D
:10669000A684F250006EF29E0F01550EA76EAA0E50
:1066A000A76EA682A6B2FED7A6940050F212AA6ADE
:1066B000090EA96E190EA86EA69CA69EA684F2CFFE
:1066C00000F0F29E550EA76EAA0EA76EA682A6B285
:1066D000FED7A6940050F212AA6A0A0EA96EA86A02
:1066E000A69CA69EA684F2CF00F0F29E550EA76E41
:1066F000AA0EA76EA682A6B2FED7A6940050F212EA
:10670000AA6A0B0EA96E140EA86EA69CA69EA6845D
:10671000F2CF00F0F29E550EA76EAA0EA76EA682CB
:10672000A6B2FED7A6940050F212AA6A0C0EA96E69
:10673000140EA86EA69CA69EA684F2CF00F0F29E30
:10674000550EA76EAA0EA76EA682A6B2FED7A69475
:106750000050F212AA6A0D0EA96E180EA86EA69C21
:10676000A69EA684F2CF00F0F29E550EA76EAA0E4A
:10677000A76EA682A6B2FED7A6940050F212AA6A0D
:106780000E0EA96E180EA86EA69CA69EA684F2CF29
:1067900000F0F29E550EA76EAA0EA76EA682A6B2B4
:1067A000FED7A6940050F212AA6A100EA96EA86A2B
:1067B000A69CA69EA684F2CF00F0F29E550EA76E70
:1067C000AA0EA76EA682A6B2FED7A6940050F21219
:1067D000AA6A110EA96EA86AA69CA69EA684F2CFEC
:1067E00000F0F29E550EA76EAA0EA76EA682A6B264
:1067F000FED7A6940050F212AA6A0F0EA96E0E0ED2
:10680000A86EA69CA69EA684F2CF00F0F29E550E1E
:10681000A76EAA0EA76EA682A6B2FED7A6940050B7
:10682000F212AA6A120EA96EA86AA69CA69EA68457
:10683000F2CF00F0F29E550EA76EAA0EA76EA682AA
:10684000A6B2FED7A6940050F212000114DE030E89
:106850000401796FE70E786F7C6B7C51110827E398
:10686000036A7C51320FE96E000E0320EA6EEFCF0F
:106870007DF479C4AAFF78C4A9FF7DC4A8FFA69CB3
:10688000A69EA684F2CF00F0F29E0F01550EA76ED1
:10689000AA0EA76EA682A6B2FED7A6940050F21248
:1068A000010E04017827000E79237C2BD6D77B6B51
:1068B0007A6B7C6B7C51110843E3036A7C51200F97
:1068C000E96E000E0320EA6EEFCF7DF47D512F08B4
:1068D00003E27D51390802E2000E01D0010E0108E9
:1068E0002DE17B532BE17A51050828E3036A7C51A3
:1068F000200FE96E000E0320EA6EEFCF7DF479C41D
:10690000AAFF78C4A9FF7DC4A8FFA69CA69EA68462
:10691000F2CF00F0F29E0F01550EA76EAA0EA76EE1
:10692000A682A6B2FED7A6940050F21204017A2BDA
:10693000D8B47B2B010E7827000E79237C2BBAD795
:106940000001000C0E015A515C03F3CF01F0F4CFAB
:1069500000F05D03F35000265B515C03F350002010
:10696000026E0001000C0401A96BAA6BAB6BA7536C
:1069700003E0A751060804E2000E016E6AD108D0B8
:10698000A85303E0A8510C0803E2000E016E61D188
:10699000AA6B900EA96F010EA75D036AAC6F03C0CE
:1069A000ADF4AAC45BFEA9C45AFE03C05DFEE8CFE5
:1069B0005CFE0001C7DF02C0AAF401C0A9F4200EEA
:1069C0000401A927000EAA23010EA85D0C0DF350A7
:1069D000036AA9270350AA23AA51036EA951A92B20
:1069E000D8B4AA2BAC6F03C0ADF4F2CFAEF4F29ED4
:1069F000ADC4AAFFACC4A9FFA69CA69EA680A850C1
:106A0000AEBFF28EAB6FAB51F00BD8B41FD1AB5110
:106A1000F00BAC6F01014D51F00B0401AC5DD8A43B
:106A200015D1ABC44DF1AA51036EA951A92BD8B40D
:106A3000AA2BAC6F03C0ADF4F2CFAEF4F29EADC49E
:106A4000AAFFACC4A9FFA69CA69EA680A850AEBF74
:106A5000F28E01014E6F0401AA51036EA951A92BB8
:106A6000D8B4AA2BAC6F03C0ADF4F2CFAEF4F29E53
:106A7000ADC4AAFFACC4A9FFA69CA69EA680A85040
:106A8000AEBFF28E0101506F4F6B0401AA51036E2D
:106A9000A951A92BD8B4AA2BAC6F03C0ADF4F2CF87
:106AA000AEF4F29EADC4AAFFACC4A9FFA69CA69EFC
:106AB000A680A850AEBFF28E01014F130401AA5167
:106AC000036EA951A92BD8B4AA2BAC6F03C0ADF4A7
:106AD000F2CFAEF4F29EADC4AAFFACC4A9FFA69C4F
:106AE000A69EA680A850AEBFF28E0101526F516BD8
:106AF0000401AA51036EA951A92BD8B4AA2BAC6FDB
:106B000003C0ADF4F2CFAEF4F29EADC4AAFFACC4A4
:106B1000A9FFA69CA69EA680A850AEBFF28E01013A
:106B200051130401AA51036EA951A92BD8B4AA2B61
:106B3000AC6F03C0ADF4F2CFAEF4F29EADC4AAFFC9
:106B4000ACC4A9FFA69CA69EA680A850AEBFF28E9C
:106B50000101546F536B0401AA51036EA951A92B73
:106B6000D8B4AA2BAC6F03C0ADF4F2CFAEF4F29E52
:106B7000ADC4AAFFACC4A9FFA69CA69EA680A8503F
:106B8000AEBFF28E010153130401AA51036EA95145
:106B9000A92BD8B4AA2BAC6F03C0ADF4F2CFAEF4DE
:106BA000F29EADC4AAFFACC4A9FFA69CA69EA68077
:106BB000A850AEBFF28E0101566F556B0401AA5169
:106BC000036EA951A92BD8B4AA2BAC6F03C0ADF4A6
:106BD000F2CFAEF4F29EADC4AAFFACC4A9FFA69C4E
:106BE000A69EA680A850AEBFF28E010155130401E7
:106BF000AA51036EA951A92BD8B4AA2BAC6F03C01C
:106C0000ADF4F2CFAEF4F29EADC4AAFFACC4A9FFBE
:106C1000A69CA69EA680A850AEBFF28E0101586F1A
:106C2000576BF2CFACF4F29EAAC4AAFFA9C4A9FF85
:106C3000A69CA69EA680A8500401ACBFF28E0101BE
:106C40005713010E016E040104D003D0000E016E33
:106C500000D00001000C04017C6BF2CF7DF4F29EA9
:106C6000AA6AA96AA69CA69EA680A8507DBFF28E9D
:106C700001013B6FF2CF7DF4F29EAA6A010EA96E6C
:106C8000A69CA69EA680A85004017DBFF28E01019D
:106C90003C6FF2CF7DF4F29EAA6A020EA96EA69C0A
:106CA000A69EA680A85004017DBFF28E01013D6F13
:106CB000F2CF7DF4F29EAA6A030EA96EA69CA69E50
:106CC000A680A85004017DBFF28E01013E6FF2CF75
:106CD0007DF4F29EAA6A040EA96EA69CA69EA680CA
:106CE000A85004017DBFF28E0101416FF2CF7DF407
:106CF000F29EAA6A050EA96EA69CA69EA680A85022
:106D000004017DBFF28E0101436FF2CF7DF4F29E4C
:106D1000AA6A060EA96EA69CA69EA680A85004018B
:106D20007DBFF28E01013A6FF2CF7DF4F29EAA6A26
:106D3000070EA96EA69CA69EA680A85004017DBF42
:106D4000F28E0101396FF2CF7DF4F29EAA6A080E2D
:106D5000A96EA69CA69EA680A85004017DBFF28EB7
:106D60000101386FF2CF7DF4F29EAA6A100EA96E6F
:106D7000A69CA69EA680A85004017DBFF28E0101AC
:106D80003F6FF2CF7DF4F29EAA6A110EA96EA69C07
:106D9000A69EA680A85004017DBFF28E0101406F1F
:106DA000F2CF7DF4F29EAA6A090EA96EA69CA69E59
:106DB000A680A85004017DBFF28E0101446FF2CF7E
:106DC0007DF4F29EAA6A0A0EA96EA69CA69EA680D3
:106DD000A85004017DBFF28E7C6F0101456B040158
:106DE0007C51200A00010BE0300A0CE0180A0DE08B
:106DF0000C0A0EE0060A0FE0030A10E012D00101AF
:106E0000452B00010101452B00010101452B00012B
:106E10000101452B00010101452B00010101452B1A
:106E20000001F2CF7DF4F29EAA6A0B0EA96EA69C19
:106E3000A69EA680A85004017DBFF28E0101466F78
:106E4000F2CF7DF4F29EAA6A0C0EA96EA69CA69EB5
:106E5000A680A85004017DBFF28E0101476FF2CFDA
:106E60007DF4F29EAA6A0D0EA96EA69CA69EA6802F
:106E7000A85004017DBFF28E0101486FF2CF7DF46E
:106E8000F29EAA6A0E0EA96EA69CA69EA680A85087
:106E900004017DBFF28E0101496FF2CF7DF4F29EB5
:106EA000AA6A120EA96EA69CA69EA680A8500401EE
:106EB0007DBFF28E01014B6FF2CF7DF4F29EAA6A84
:106EC0000F0EA96EA69CA69EA680A85004017DBFA9
:106ED000F28E01014A6F4A51280802E2280E4A6FD9
:106EE0004851180802E2180E486F4951180802E28A
:106EF000180E496F3BC1A7F43CC1A8F4000133DD73
:106F0000010E016E6CEF65F0036A6551A90FE96E21
:106F1000000E0320EA6EEFCFA5F80801010E000174
:106F200065250801A76F196AF2BE198EF29EE8CF97
:106F300061FE780E0E01626F0001CAEC24F019BEEA
:106F4000F28E00C065F06551625D01E1A881080123
:106F5000A5C801F00001000C0801AABF10D00F0E57
:106F6000006EA93900160A0E005C03E2300E0026FE
:106F700002D0AA51002600509EA8FED7AD6E0F0E7B
:106F8000A9170A0EA95D02E2300E02D0AA9FAA51EB
:106F9000A927A9519EA8FED7AD6E0001000C640E72
:106FA0000801A86F0001DDEC28F0010139A507D028
:106FB0000D0E000109EC2CF00A0E09EC2CF000017A
:106FC0006551625D19E0A0DF01C07DF4010139A5C2
:106FD0000CD07DC4A9F8570E0801AA6F0001BCDFD0
:106FE000200E09EC2CF007D00101320E0801A86F29
:106FF0000001DDEC28F0E4D7000C200E080180A988
:10700000300E816F7FC800F07FAF07D0001E002ACE
:1070100000C07FF82D0E816F808F0150196AF2BE7B
:10702000198EF29E7FC861FE640E0E01626F000130
:10703000CAEC24F019BEF28E00C07FF8300E012495
:107040000801826F196AF2BE198EF29E7FC861FE36
:107050000A0E0E01626F0001CAEC24F019BEF28E16
:10706000300E00240801846F300E0124836F81C824
:1070700000F080A702D080AF809580B90BD080AFA0
:1070800022D080B520D000C082F880B31CD000C0D0
:1070900083F819D0300E825D16E100C082F8200E10
:1070A000816F80A704D08095808380AF8093300E5D
:1070B000835D09E100C083F8200E826F80A7F7D7B7
:1070C000809380AF809180A504D081519EA8FED787
:1070D000AD6E80A304D082519EA8FED7AD6E80A174
:1070E00004D083519EA8FED7AD6E84519EA8FED7D2
:1070F000AD6E0001000CA4A8FED76D6E000C080157
:10710000A66BA76BA4C8E9FFA5C8EAFFEFCFA7F855
:10711000A7533EE0010139A507D00D0E000109EC8F
:107120002CF00A0E09EC2CF0010E0801A66FA651F6
:10713000A75D2EE3010139A515D0036A0801A65108
:10714000A425E96EA5510320EA6EEFCFA8F8A8C8E0
:10715000A9F8570EAA6F0001FFDE200E09EC2CF0F3
:1071600007D00101010E0801A86F0001DDEC28F035
:10717000036A0801A651A425E96EA5510320EA6E11
:10718000EFCFA8F8A8510001B6DF0801A62BCFD792
:107190000001000CEACF9FF8E9CF9EF8080198AFF4
:1071A00008D09E8F9EA99E2B971F981F972BD8B40F
:1071B000982B9839F0099A6F9A27E20F9B6F320F3C
:1071C0009D6F98510F0B9B279B279D27E90F9C6F65
:1071D0009C279C2797390F0B9C279D279C379D3711
:1071E0009D1F9D3797510F0B9D279A37070E996F5B
:1071F0000A0E9C079D27FDE39B079C27FDE39A074A
:107200009B27FDE399079A27FDE3080EEA6E990E86
:10721000E96E070E9E159E9DE9069E1507E19EB933
:10722000E92A9EB903D0200E006E1CD0E9269D0EDF
:10723000E95CD8B49E8DEF50006E08E19EBD06D08B
:107240009EB914D09EB702D0200E0BD09EAF06D0B0
:107250002D0E006EED509E9D9E9F04D09E879E99A0
:10726000300E002600509EA8FED7AD6EEE509EADAB
:10727000DED70001000C0801926B936B946B956B49
:1072800096910001A8A151D095C85BFE94C85AFE02
:107290000E015D6B320E5C6F0001A2EC34F002C097
:1072A00098F801C097F808018551025C33E303E1C7
:1072B0008451975D2FE3010139A528D00801976B10
:1072C0009751000110EC13F00801972B000109EC15
:1072D0002CF0170E0801975DF3E1100EE96E85C8DA
:1072E00098F884C897F8000155DF1A0E0801976FC7
:1072F0009751000110EC13F00801972B000109ECE5
:107300002CF0210E0801975DF3E10101000E016EE2
:10731000F1D00801320EA86F0001DDEC28F0080161
:10732000942BD8B4952BADD70001080EEA6E860ECB
:10733000E96E0801A16BA36B0C0EA26F000175EC46
:1073400030F0010139A51DD00801976B975100015C
:1073500030EC13F00801972B000109EC2CF00F0E14
:107360000801975DF3E1100EE96E85C898F884C8AE
:1073700097F800010FDF290E09EC2CF0200E09EC24
:107380002CF00001A8B1B5D0BFDD01C092F8080112
:1073900096A165D0923D35D0010139A50BD092C898
:1073A000A9F8370E0801AA6F0001D6DD200E09ECFE
:1073B0002CF0010108018751410803E08751420880
:1073C00006E1010E016E010195D019D00801875127
:1073D000510803E0875152080EE1080EEA6E860E4E
:1073E000E96EA16BA36B0C0EA26F000175EC30F07F
:1073F0000801969105D0000E016E01017BD00801B5
:107400002DD0036A9351860FE96E080E0320EA6EB1
:1074100092C8EFFF010139A515D0036A0801935105
:10742000860FE96E080E0320EA6EEFCF97F897C833
:10743000A9F8370EAA6F00018FDD200E09EC2CF0A1
:1074400007D00101320E0801A86F0001DDEC28F021
:107450000801932B93510B0801E2969144D092516D
:10746000900824E1936B036A9351860FE96E080E2E
:107470000320EA6E92C8EFFF010139A513D0036A19
:1074800008019351860FE96E080E0320EA6EEFCFD4
:1074900097F897C8A9F8370EAA6F00015DDD200E96
:1074A00009EC2CF00801932B96811DD0010139A520
:1074B00013D05B0E000109EC2CF092C8A9F8370E2E
:1074C0000801AA6F000148DD5D0E09EC2CF0200ECA
:1074D00009EC2CF007D00101320E0801A86F000161
:1074E000DDEC28F00801320EA86F0001DDEC28F079
:1074F00049D701010001000C0801A46B0001A8B1EB
:1075000004D002DD01C0A4F8FAD7000C060E080171
:107510006F6F810E706F010E716F040E726F070E28
:10752000736F746BFF0E756F090E766F810E776F38
:10753000010E786F060E796F010E7A6F7B6B7C6B94
:10754000030E7D6F7E6FFF0E7F6F836B6C517F0B21
:10755000806F6D517F0B816F6E517F0B826F0101C8
:107560004D39006E0F0E001600500B080BE108019C
:107570008253D8A402D0010105D0010141517F0BF3
:107580000801826F0801805305E1010E806F030E30
:107590007D6F09D06C51800B800803E1010E7D6F77
:1075A00002D0020E7D6F80C87BF8815305E1010E89
:1075B000816F030E7E6F09D06D51800B800803E14F
:1075C000010E7E6F02D0020E7E6F81C87CF8010131
:1075D0004D39006E0F0E001600500A0855E00801E4
:1075E0007D51030803E17E51030839E0010159830D
:1075F000080E0801A56F760EA46F000180DD010161
:107600004D39006E0F0E00160050010807E04D398D
:10761000006E0F0E00160050050809E1030E080168
:10762000856FE80E846F000126DE16D001014D390A
:10763000006E0F0E0016005003080FE14B530DE0D3
:107640000801856BFA0E846F000115DE4BC183F8CB
:1076500083C8A8F8DDEC28F0010114D0080101016D
:1076600059A310D05993080E0801A56F760EA46F88
:10767000000145DD030E0801856FE80E846F0001EF
:10768000FADD0101000138DF0801825302E1746B69
:107690000DD06E51800B800805E18251070B200947
:1076A000746F04D08251070B3009746F745343E038
:1076B00001014D39006E0F0E001600500B0803E15A
:1076C00059A101D04ED0080E0801A56F6F0EA46F0E
:1076D000000115DD010159814D39006E0F0E0016B4
:1076E0000050010807E04D39006E0F0E00160050E3
:1076F000050809E1030E0801856FE80E846F00019B
:10770000BADD16D001014D39006E0F0E0016005083
:1077100003080FE14B530DE00801856BFA0E846FEF
:107720000001A9DD4BC183F883C8A8F8DDEC28F07F
:10773000010114D00801010159A110D05991080E7E
:107740000801A56F6F0EA46F0001D9DC030E0801BC
:10775000856FE80E846F00018EDD01010001CCDE33
:1077600001010001000C0801A551090805E3300ED4
:10777000A525016E05D004D0370EA525016E00D0D9
:107780000001000C080E08016F6FFF0E706F300EC5
:10779000716F726F736B600E746F300E756F766FF2
:1077A000EF0E776F070E786FFF0E796F300E7A6FDE
:1077B0007B6F7C6BA20E7D6F300E7E6FEF0E7F6F46
:1077C000090E806FFF0E816F300E826F836F846BA6
:1077D000500E856F866B876B886BEF0E896F090E75
:1077E0008A6FFF0E8B6F300E8C6F8D6F8E6B510E0C
:1077F0008F6F906B916B926BEF0E936F080E946F7F
:10780000FF0E956F300E966F976F986BB40E996F51
:10781000310E9A6F9B6BEF0E9C6F6C517F0B9D6FBF
:107820006D517F0B9E6F6E517F0B9F6F9F5315E1C4
:1078300004010B513008D8A402D008010ED0000179
:107840005BDE080E0801A56F780EA46F000157DCFF
:107850007EC80BF40101599108019D531CE19E5310
:107860001AE104010951300806E10A513008D8A490
:1078700002D0080110D000013FDE080E0801A56FFC
:107880006F0EA46F00013BDC75C809F476C80AF4DA
:107890000101599308019D5305E19E5303E19F5354
:1078A00001E134D19D5303E1300E756F09D06C5165
:1078B000800B800803E1320E756F02D0310E756FB8
:1078C0009E5303E1300E766F09D06D51800B800816
:1078D00003E1310E766F02D0320E766F036A9EC8D6
:1078E000A4F803C0A5F80E015B6B1E0E5A6F03C00F
:1078F0005DFE9EC85CFE0001A2EC34F0080E08019B
:107900000124A06F000E0220A16F036A9DC8A4F895
:1079100003C0A5F80E015B6B210E5A6F03C05DFE1C
:107920009DC85CFE0001A2EC34F0080E08010124A1
:10793000A26F000E0220A36FA35306E1A251090813
:1079400003E3A36B0A0EA26FA351020809E2FF0A28
:1079500003E1A251200804E2030EA36F200EA26FE0
:10796000A15306E1A051090803E3A16B0A0EA06F21
:10797000A151010809E2FF0A03E1A0516E0804E2E7
:10798000020EA16F6E0EA06FA3510F0BA46FA56F17
:107990000001E9DE01C086F80801A2C800F0003A43
:1079A0000F0E001600500F0BA46FA56F0001DBDE59
:1079B00001C087F80801A2510F0BA46FA56F000149
:1079C000D2DE01C088F80801A1510F0BA46FA56F8A
:1079D0000001C9DE01C090F80801A0C800F0003A1B
:1079E0000F0E001600500F0BA46FA56F0001BBDE39
:1079F00001C091F80801A0510F0BA46FA56F000101
:107A0000B2DE01C092F808019D5318E075513008AC
:107A100015E00101598308019D5101015A5D0DE0F6
:107A20009DC85AF1000168DD080E0801A56F800E9F
:107A3000A46F00017FEC38F0010108019E5318E0AB
:107A40007651300815E00101598308019E5101016A
:107A50005B5D0DE09EC85BF100014EDD080E080184
:107A6000A56F8A0EA46F00017FEC38F001010801B8
:107A7000765104010A5D05E1080175510401095DB3
:107A80000EE075C809F476C80AF4000135DD080E69
:107A90000801A56F6F0EA46F00017FEC38F008019C
:107AA0009F5334E06E51800B800803E1320E7E6FED
:107AB00002D0310E7E6F0101598108019F510101F1
:107AC0005C5D11E09FC85CF108019F51070B300914
:107AD0009B6F000111DD080E0801A56F940EA46FC5
:107AE00000017FEC38F008017E5104010B5D0DE0D0
:107AF0007EC80BF4000100DD080E0801A56F780EAA
:107B0000A46F00017FEC38F0040108010001000CB3
:107B10006B50060B2AE0010139A51ED004019A6BB7
:107B20009A51000163EC22F004019A2B000109EC48
:107B30002CF0160E04019A5DF3E16BCFA9F8570EF5
:107B40000801AA6F0001ACEC37F00A0E09EC2CF02A
:107B50000D0E09EC2CF001016B6A010E0801656F36
:107B60000001C8EC28F0900E6B6EEFEF3DF00101C4
:107B70004D39006E0F0E00160050FF0FF20F14E289
:107B80000E0F000123EF3EF008016C6B6D6B6E6B06
:107B90000001BCDC010108D008016C6B6D6B6E6BE1
:107BA0000001F0DD010100D0040199B102D08D96F1
:107BB00001D08D86969699B302D08D9801D08D888C
:107BC000969899B502D08D9A01D08D8A969A050E15
:107BD0000801A86F0001DDEC28F08EDC99D799C46C
:107BE0008AF1036A04019951250F016E000E0322E8
:107BF0000150380FE96E010E0320EA6EEFCF4DF110
:107C00000101D89004019935036A3A0F016E000E04
:107C100003220150380FE96E010E0320EA6EECCF0B
:107C200003F0ED52EFCF57F1010103C058F14E6B55
:107C3000506B4F6B526B516B546B536B566B556B58
:107C4000596B0001000CF2CF0EF0F29EE824F76AA7
:107C5000F736710FF66E7C0EF722000EF86EFB6E93
:107C60000A00F550FA6E0800F5500EBEF28EF96E5D
:107C7000887B887B887B887B887B887B887B887BEC
:107C8000887B887B887B987BA87B887B050E04019A
:107C90009E6F5B0E9F6F490EA06F4E0EA16F300E50
:107CA000A26F5D0EA36F9C51075D46E09CC407F474
:107CB0009DB102D08D9601D08D8696969DB302D04F
:107CC0008D9801D08D8896989DB502D08D9A01D05F
:107CD0008D8A969A050E0801A86F0001DDEC28F048
:107CE0009CC4A2F4040E0801A56F9E0EA46F0001AF
:107CF0007FEC38F0050E0801A86F0001DDEC28F0DC
:107D00007CEC3AF001018AB102D08D9601D08D86CB
:107D100096968AB302D08D9801D08D8896988AB5B0
:107D200002D08D9A01D08D8A969A050E0801A86F0F
:107D30000001DDEC28F004010001000C7CEC3AF0BD
:107D400004019B2D14D0010138A708D0300E040186
:107D50009C6F060E9D6F000199DF07D0310E040164
:107D60009C6F060E9D6F000191DF07D00401330E5A
:107D70009C6F060E9D6F000189DF000C0401B16B42
:107D8000B26BB36BB46BFF0EB56FB6910001A8A1D7
:107D900052D0B4C45BFEB3C45AFE0E015D6B320E0A
:107DA0005C6F0001A2EC34F002C0B8F401C0B7F47B
:107DB00004019C51025C33E303E19B51B75D2FE367
:107DC000010139A529D00401B76BB7510001CFECEF
:107DD0000EF00401B72B000109EC2CF01C0E04017D
:107DE000B75DF3E1100EE96E9CC498F89BC497F858
:107DF0000001CAEC38F01F0E0401B76FB751000143
:107E0000CFEC0EF00401B72B000109EC2CF0260E8C
:107E10000401B75DF3E10101FF0E016ED3D0320E14
:107E20000801A86F0001DDEC28F00401B32BD8B4E1
:107E3000B42BACD70001040EEA6E9D0EE96E08016A
:107E4000A16BA36B140EA26F000175EC30F0010161
:107E500039A50FD00401B76BB7510001F2EC0EF059
:107E60000401B72B000109EC2CF01C0E0401B75DD6
:107E7000F3E10401B26BFF0EB56F0001A8B191D020
:107E800084EC37F001C0B1F40401B6B132D0B26B6A
:107E9000B1515B0819E1036AB2519D0FE96E040EFE
:107EA0000320EA6EB1C4EFFFB22BB681010139A500
:107EB00009D00401B151000109EC2CF0200E09ECAD
:107EC0002CF0010114D00401010139A510D0280EB5
:107ED000000109EC2CF00401B151000109EC2CF077
:107EE000290E09EC2CF0200E09EC2CF0010157D0E2
:107EF0000401036AB2519D0FE96E040E0320EA6E7D
:107F0000B1C4EFFF010139A508D00401B15100014E
:107F100009EC2CF0200E09EC2CF00401B1515D08A5
:107F200037E19E51490826E19F514E0823E1A151B6
:107F30005D0820E1A0C4B5F4010139A519D0040100
:107F4000B76BB751000110EC0FF00401B72B000123
:107F500009EC2CF00D0E0401B75DF3E1B551000101
:107F600009EC2CF00A0E09EC2CF00D0E09EC2CF0AB
:107F7000000117D0010139A507D00A0E000109EC54
:107F80002CF00D0E09EC2CF00401B26BB69107D069
:107F9000B22BB251130803E2000103D00401040123
:107FA0006CD7010139A507D00A0E000109EC2CF0AD
:107FB0000D0E09EC2CF000017CEC3AF00401B5C484
:107FC00001F00101000117EF40F0080E0401926F6B
:107FD0005B0E936F530E946F540E956F410E966F18
:107FE000540E976F550E986F530E996F5D0E9A6FE2
:107FF000010E9B6F0001A2DE640E0801A86F000154
:10800000DDEC28F0040E0801A56F920EA46F0001AC
:108010007FEC38F0320E0801A86F0001DDEC28F08B
:10802000030E04019C6FE80E9B6F0001A7D6015060
:10803000FAEF60F00601066B076B086B0991050EFD
:10804000EA6EF90EE96E0801A16BA36B0D0EA26F2B
:10805000000175EC30F0A8A155D008C65BFE07C63C
:108060005AFE0E015D6B190E5C6F0001A2EC34F03C
:1080700002C00BF601C00AF60501F8510601025CC8
:1080800035E305E10501F75106010A5D2FE3010122
:1080900039A529D006010A6B0A510001B0EC13F092
:1080A00006010A2B000109EC2CF0150E06010A5DF1
:1080B000F3E1100EE96EF8C598F8F7C597F80001DE
:1080C000CAEC38F0180E06010A6F0A510001B0EC34
:1080D00013F006010A2B000109EC2CF01F0E06011B
:1080E0000A5DF3E10101000E016EABD0190E08012B
:1080F000A86F0001DDEC28F00601072BD8B4082B8F
:108100000001A9D7010139A50FD006010A6B0A5158
:108110000001CFEC13F006010A2B000109EC2CF052
:108120000D0E06010A5DF3E10001A8B187D0036AD4
:1081300006010651F90F016E050E032201C00AF671
:1081400003C00BF6000184EC37F00BC6EAFF0AC649
:10815000E9FF01C0EFFF010139A515D0036A06014F
:108160000651F90FE96E050E0320EA6EEFCF0AF60D
:108170000AC6A9F8370E0801AA6F0001ACEC37F067
:10818000200E09EC2CF0060109B119D0036A065142
:10819000F90FE96E050E0320EA6EEF50FE080EE1BE
:1081A000036A0651F90FE96E050E0320EA6EEFCF60
:1081B000F9F5050106010981010E066F35D0036A44
:1081C0000651F90FE96E050E0320EA6EEF50EF0835
:1081D0001DE1010139A507D00D0E000109EC2CF0BD
:1081E0000A0E09EC2CF00501FC51300809E1FD51A3
:1081F000300806E1010E016E010123D005D0050112
:10820000000E016E01011DD007D00601320E0801DB
:10821000A86F0001DDEC28F0060106510B0802E30F
:10822000062B02D0066B09910001A8A106D0320EE0
:108230000801A86F0001DDEC28F077D7000E016E71
:1082400001010001000C0401F46BF56B060EF66FE2
:10825000FF0EF76F300EF86FF96FFA6B860EFB6F3B
:10826000EF0EFC6F060EFD6FFF0EFE6F300EFF6F00
:108270000501006F016B860E026FEF0E036F060E95
:10828000046FFF0E056F300E066F076F086B860ECA
:10829000096FEF0E0A6F060E0B6FFF0E0C6F300E9C
:1082A0000D6F0E6F0F6B860E106FEF0E116F060EB7
:1082B000126FFF0E136F300E146F156F166B860E54
:1082C000176FEF0E186F060E196FFF0E1A6F300E34
:1082D0001B6F1C6F1D6B860E1E6FEF0E1F6F070E40
:1082E000206FFF0E216F300E226F236F246BA50EBF
:1082F000256F3C0E266FEF0E276F070E286FFF0EBF
:10830000296F300E2A6F2B6F2C6BB40E2D6F300E31
:108310002E6FEF0E2F6F060E306FFF0E316F300E87
:10832000326F336F346B630E356FEF0E366F070E9F
:10833000376FFF0E386F300E396F3A6F3B6BB10EEF
:108340003C6F300E3D6FEF0E3E6F070E3F6FFF0E1E
:10835000406F300E416F426F436B900E446F300E92
:10836000456FEF0E466F070E476FFF0E486F300EDA
:10837000496F4A6F4B6BA00E4C6F310E4D6FEF0E75
:108380004E6F070E4F6FFF0E506F300E516F526FD2
:10839000536BA00E546F300E556FEF0E566F070ED5
:1083A000576FFF0E586F300E596F5A6F5B6BA50EEB
:1083B0005C6F310E5D6FEF0E5E6F070E5F6FFF0E2D
:1083C000606F300E616F626F636BA50E646F300E6D
:1083D000656FEF0E666F070E676FFF0E686F300EEA
:1083E000696F6A6F6B6BA70E6C6F300E6D6FEF0E5F
:1083F0006E6F070E6F6FFF0E706F300E716F726FC2
:10840000736BA70E746F310E756FEF0E766F070EDC
:10841000776FFF0E786F300E796F7A6F7B6BA70ED8
:108420007C6F310E7D6FEF0E7E6F070E7F6FFF0E3C
:10843000806F300E816F826F836BA50E846F320E5A
:10844000856FEF0E866F070E876FFF0E886F300EF9
:10845000896F8A6F8B6BA50E8C6F320E8D6FEF0E4E
:108460008E6F090E8F6FFF0E906F300E916F926FAF
:10847000936BA50E946F3B0E956F966B976BEF0EFB
:10848000986F080E996FFF0E9A6F300E9B6F9C6F5E
:108490009D6BA50E9E6F340E9F6F300EA06FEF0E7A
:1084A000A16F070EA26FFF0EA36F300EA46FA56F12
:1084B000A66BA10EA76F300EA86FEF0EA96F070E67
:1084C000AA6FFF0EAB6F300EAC6FAD6FAE6BA10E2F
:1084D000AF6F310EB06FEF0EB16F070EB26FFF0EC0
:1084E000B36F300EB46FB56FB66BA10EB76F330EAE
:1084F000B86FEF0EB96F070EBA6FFF0EBB6F300E7D
:10850000BC6FBD6FBE6BA10EBF6F320EC06FEF0EA2
:10851000C16F070EC26FFF0EC36F300EC46FC56F01
:10852000C66BA10EC76F310EC86FEF0EC96F090E73
:10853000CA6FFF0ECB6F300ECC6FCD6FB00ECE6F0B
:10854000CF6BD06BD16BD26BEF0ED36F060ED46FA7
:10855000FF0ED56F300ED66FD76FD86B570ED96F11
:10856000EF0EDA6F070EDB6FFF0EDC6F300EDD6F84
:10857000DE6FDF6B580EE06F310EE16FEF0EE26FD2
:10858000090EE36FFF0EE46F300EE56FE66FE76BE9
:10859000500EE86F310EE96FEA6FEB6FEF0EEC6F84
:1085A000070EED6FFF0EEE6F300EEF6FF06FF16B99
:1085B000890EF26FF36BEF0EF46FF56BF66B04013F
:1085C000F251330A0001D8B497D0320AD8B49DD002
:1085D000030AD8B4A3D0010AD8B4A9D0070AD8B4E2
:1085E000AFD0010AD8B4B5D0030AD8B4BBD00E0AB4
:1085F000D8B4C1D0010AD8B4C7D0030AD8B4CDD0FA
:108600000D0AD8B4D3D00A0AD8B4D9D0030AD8B442
:10861000DFD0010AD8B4E5D01F0AD8B4EBD0010AE4
:10862000D8B4F1D0030AD8B4F7D0010AD8B4FDD039
:10863000260AD8B403D1010AD8B411D10C0AD8B48F
:108640001FD1220AD8B42DD1030AD8B436D10D0ACD
:10865000D8B43FD1010AD8B445D1030AD8B45CD10B
:10866000010AD8B45FD10F0AD8B462D1030AD8B4D2
:108670009CD1070AD8B4A2D1010AD8B4A8D1030A60
:10868000D8B4AED1010AD8B4B4D13F0AD8B4BAD163
:10869000030AD8B40CD2070AD8B416D2010AD8B447
:1086A00020D2030AD8B425D2010AD8B42BD20F0A9B
:1086B000D8B435D2010AD8B43BD2030AD8B446D2D2
:1086C000010AD8B44CD2070AD8B45DD2010AD8B492
:1086D00069D2030AD8B475D2010AD8B47CD21E0A72
:1086E000D8B481D2030AD8B487D2080AD8B48DD2BC
:1086F000010AD8B4F8D265D3050E0801A56F3F0E64
:10870000A46F00017FEC38F060D3040E0801A56F60
:10871000F60EA46F00017FEC38F057D3040E080169
:10872000A56FFD0EA46F00017FEC38F04ED3050E4F
:108730000801A56F040EA46F00017FEC38F045D34B
:10874000050E0801A56F0B0EA46F00017FEC38F039
:108750003CD3050E0801A56F120EA46F00017FEC3B
:1087600038F033D3050E0801A56F190EA46F000170
:108770007FEC38F02AD3050E0801A56F200EA46FF8
:1087800000017FEC38F021D3050E0801A56F280EFB
:10879000A46F00017FEC38F018D3050E0801A56F17
:1087A000300EA46F00017FEC38F00FD3050E0801E6
:1087B000A56F370EA46F00017FEC38F006D3050ECD
:1087C0000801A56F470EA46F00017FEC38F0FDD2C1
:1087D000050E0801A56F4F0EA46F00017FEC38F065
:1087E000F4D2050E0801A56F570EA46F00017FECAF
:1087F00038F0EBD2050E0801A56F5F0EA46F0001E3
:108800007FEC38F0E2D2050E0801A56F670EA46F69
:1088100000017FEC38F0D9D2050E0801A56F6F0E6C
:10882000A46F00017FEC38F0D0D2050E0801A56FCF
:10883000770EA46F00017FEC38F0C7D201018B5195
:108840000F0B30090501F36F8A0EF26F050E080158
:10885000A56FED0EA46F00017FEC38F0B6D20101D8
:108860008B510F0B30090501F36F890EF26F050E66
:108870000801A56FED0EA46F00017FEC38F0A5D2C2
:1088800001018B510F0B30090501F36F8B0EF26F55
:10889000050E0801A56FED0EA46F00017FEC38F006
:1088A00094D2300E0501A06F050E0801A56F990E38
:1088B000A46F00017FEC38F088D2310E0501A06F63
:1088C000050E0801A56F990EA46F00017FEC38F02A
:1088D0007CD2050E0801A56F870EA46F00017FEC06
:1088E00038F073D2050E0801A56F7F0EA46F00014A
:1088F0007FEC38F0640E0801A86F0001DDEC28F071
:10890000300E0501A06F050E0801A56F990EA46F2A
:1089100000017FEC38F059D2020E01015727000EFA
:108920005823000101015751D8B4580757070001D7
:108930000101585307E157510F0804E3586B100E1B
:10894000576F06D05851000803E2586BFF0E576F5F
:1089500058C1F6F557C1F5F50501F631F86FF53157
:10896000F76FF833F733F833F733F833F7330F0E85
:10897000F817F7C5A5F80001B3EC3BF001C096F578
:108980000501F5510F0BF76FF86BE8CFA5F8000163
:10899000B3EC3BF001C097F5050E0801A56F8F0EF3
:1089A000A46F00017FEC38F010D2050E0801A56F0E
:1089B000A20EA46F00017FEC38F007D2050E08016B
:1089C000A56FAA0EA46F00017FEC38F0FED1050E52
:1089D0000801A56FB20EA46F00017FEC38F0F5D14D
:1089E000050E0801A56FBA0EA46F00017FEC38F0E8
:1089F000ECD1050E0801A56FC20EA46F00017FEC3B
:108A000038F0E3D156C1F6F555C1F5F50501F76B20
:108A1000F651F00BF86FF76FF86BF833F733F83364
:108A2000F733F833F733F833F7330F0EF817F7C58A
:108A3000A5F80001B3EC3BF001C0CFF50501F76BE1
:108A4000F6510F0BF86FF76FF86BE8CFA5F8000140
:108A5000B3EC3BF001C0D0F50501F551F00BF76F19
:108A6000F86BF833F733F833F733F833F733F83379
:108A7000F7330F0EF817F7C5A5F80001B3EC3BF07C
:108A800001C0D1F50501F5510F0BF76FF86BE8CF79
:108A9000A5F80001B3EC3BF001C0D2F5050E0801CA
:108AA000A56FCA0EA46F00017FEC38F08ED10101D2
:108AB000415188090501F76F08016C6B6D6B6E6F92
:108AC0000001C2EC3BF081D10101415108090501CF
:108AD000F76F08016C6B6D6B6E6F0001C2EC3BF0C1
:108AE00074D108016C6B6D6B6E6B0001C2EC3BF0D6
:108AF0006CD108016C6B6D6B41C16EF80001C2EC6A
:108B00003BF063D101013D5180090501F76F080178
:108B10006C6B6D6F6E6B0001C2EC3BF056D10801BF
:108B20006C6B3DC16DF86E6B0001C2EC3BF04DD13A
:108B300001013E5180090501F76FE8CF6CF808018B
:108B40006D6B6E6B0001C2EC3BF03FD13EC16CF827
:108B500008016D6B6E6B0001C2EC3BF036D1010178
:108B60003E5180090501F76F01013D518009050162
:108B7000F86FF7C56CF8E8CF6DF808016E6B00016F
:108B8000C2EC3BF022D101013D5180090501F76F94
:108B90003EC16CF8E8CF6DF808016E6B0001C2ECC5
:108BA0003BF013D101013E5180090501F76FE8CF79
:108BB0006CF83DC16DF808016E6B0001C2EC3BF032
:108BC00004D13EC16CF83DC16DF808016E6B000127
:108BD000C2EC3BF0FAD008016C6B6D6B6E6B000160
:108BE000C2EC3BF0F2D0050E0801A56FD40EA46FC5
:108BF00000017FEC38F0E9D0050E0801A56FDB0E0F
:108C0000A46F00017FEC38F0E0D0036A3EC1F7F5B5
:108C100003C0F8F50E015B6B210E5A6F03C05DFEB9
:108C20003EC15CFE0001A2EC34F0080E05010124F7
:108C30000401F46F000E050102200401F56FF553E5
:108C400007E1F451070804E3F56B080EF46F0CD04C
:108C5000F551020809E2FF0A03E1F451200804E299
:108C6000030EF56F200EF46F500E0501E86FF76BE1
:108C70000401F5510F0B0501F86FF76FF86BE8CFA2
:108C8000A5F80001B3EC3BF001C0E9F50401F45193
:108C9000F00B0501F76FF86BF833F733F833F73360
:108CA000F833F733F833F7330F0EF817F7C5A5F895
:108CB0000001B3EC3BF001C0EAF50401F4510F0BE5
:108CC0000501F76FF86BE8CFA5F80001B3EC3BF0B6
:108CD00001C0EBF5050E0801A56FE30EA46F0001BE
:108CE0007FEC38F072D0036A3DC1F7F503C0F8F5A8
:108CF0000E015B6B1A0E5A6F03C05DFE3DC15CFE38
:108D00000001A2EC34F0080E050101240401F46F07
:108D1000000E050102200401F56FF55307E1F4513F
:108D2000070804E3F56B080EF46F0CD0F551010849
:108D300009E2FF0A03E1F4516E0804E2020EF56F46
:108D40006E0EF46F510E0501E86FF76B0401F551DB
:108D50000F0B0501F86FF76FF86BE8CFA5F800016E
:108D6000B3EC3BF001C0E9F50401F451F00B05014F
:108D7000F76FF86BF833F733F833F733F833F7332B
:108D8000F833F7330F0EF817F7C5A5F80001B3EC69
:108D90003BF001C0EAF50401F4510F0B0501F76F38
:108DA000F86BE8CFA5F80001B3EC3BF001C0EBF5A0
:108DB000050E0801A56FE30EA46F00017FEC38F0EB
:108DC00004D0000E016E0FD000D00401F32D09D0A5
:108DD000070E0501F86FD00EF76F00011AEC40F096
:108DE0000401010E016E0001000C0401926BA36BE3
:108DF000FE0EA46FA56BA66B0001A8A13AD0A6C475
:108E00005BFEA5C45AFE0E015D6B320E5C6F000165
:108E1000A2EC34F002C0A8F401C0A7F4040102508F
:108E200006081BE2FF0A03E1A751CF0816E2010181
:108E300039A510D00401A76BA7510001D8EC0FF0A1
:108E40000401A72B000109EC2CF0230E0401A75DFF
:108E5000F3E10101000E016E85D0320E0801A86F0A
:108E60000001DDEC28F00401A52BD8B4A62BC4D753
:108E70000001040EEA6E930EE96E0801A16BA36B6C
:108E8000100EA26F000175EC30F0010139A510D071
:108E90000401A76BA7510001F9EC0FF00401A72B07
:108EA000000109EC2CF0100E0401A75DF3E10101B3
:108EB0000001A8B13CD00401A3510F08D8B002D0E2
:108EC000000135D0000184EC37F001C092F40A0EA5
:108ED0000801A86F0001DDEC28F0010139A50DD0D3
:108EE00092C4A9F8370E0801AA6F0001ACEC37F064
:108EF000200E09EC2CF007D00101320E0801A86FFA
:108F00000001DDEC28F00401A451925D04E1A36BA3
:108F100092C493F40AD0A32B036AA351930FE96E72
:108F2000040E0320EA6E92C4EFFF0101C1D70401D1
:108F30009351FE0813E1036AA351930FE96E040EE7
:108F40000320EA6EEF50EF0809E1A351050806E19E
:108F5000010E016E010106D005D00401000E016E64
:108F6000010100D0000183EF61F00501E46BE56BC6
:108F7000E66BE76BE891E8930001A8A152D0E7C542
:108F80005BFEE6C55AFE0E015D6B320E5C6F0001A2
:108F9000A2EC34F002C0EAF501C0E9F50501D751B1
:108FA000025C33E303E1D651E95D2FE3010139A50A
:108FB00029D00501E96BE95100014AEC13F00501E4
:108FC000E92B000109EC2CF0140E0501E95DF3E139
:108FD000100EE96ED7C598F8D6C597F80001CAEC0F
:108FE00038F0170E0501E96FE95100014AEC13F062
:108FF0000501E92B000109EC2CF01E0E0501E95DCD
:10900000F3E10101000E016E2CD2320E0801A86FAF
:109010000001DDEC28F00501E62BD8B4E72BACD736
:109020000001050EEA6ED80EE96E0801A16BA36B74
:109030000C0EA26F000175EC30F0010139A50FD0C4
:109040000501E96BE951000169EC13F00501E92B19
:10905000000109EC2CF00C0E0501E95DF3E10001C3
:10906000A8B1FED184EC37F001C0E4F50501E8A316
:10907000A3D1E43D3AD1010139A50CD0E4C5A9F84A
:10908000370E0801AA6F0001ACEC37F0200E09EC96
:109090002CF001010501D851880803E0D85181085E
:1090A00010E1010139A508D00D0E000109EC2CF0EA
:1090B0000A0E09EC2CF00101010E016ED2D113D180
:1090C0000501D951510804E0D9515208D8A48CD0D7
:1090D000010139A507D00D0E000109EC2CF00A0E94
:1090E00009EC2CF00501E8A106D0010E016E01018A
:1090F000B8D178D00501010139A510D00501E96B7F
:10910000E951000169EC13F00501E92B000109ECBC
:109110002CF00C0E0501E95DF3E10101050EEA6E8C
:10912000D80EE96E0801A16BA36B0C0EA26F0001B3
:1091300075EC30F00501E8930001A8A152D0E7C515
:109140005BFEE6C55AFE0E015D6B320E5C6F0001E0
:10915000A2EC34F002C0EAF501C0E9F50501D751EF
:10916000025C33E303E1D651E95D2FE3010139A548
:1091700029D00501E96BE95100017FEC13F00501ED
:10918000E92B000109EC2CF0090E0501E95DF3E182
:10919000100EE96ED7C598F8D6C597F80001CAEC4D
:1091A00038F00C0E0501E96FE95100017FEC13F076
:1091B0000501E92B000109EC2CF0130E0501E95D16
:1091C000F3E10101000E016E4CD1320E0801A86FCF
:1091D0000001DDEC28F00501E62BD8B4E72BACD775
:1091E0000001010180D00501D951410804E0D951A5
:1091F0004208D8A476D0E881010139A510D0050134
:10920000E96BE951000169EC13F00501E92B00015C
:1092100009EC2CF00C0E0501E95DF3E10101050EEE
:10922000EA6ED80EE96E0801A16BA36B0C0EA26F5B
:10923000000175EC30F00501E8930001A8A152D0BF
:10924000E7C55BFEE6C55AFE0E015D6B320E5C6F34
:109250000001A2EC34F002C0EAF501C0E9F5050115
:10926000D751025C33E303E1D651E95D2FE30101FD
:1092700039A529D00501E96BE95100017FEC13F014
:109280000501E92B000109EC2CF0090E0501E95D4F
:10929000F3E1100EE96ED7C598F8D6C597F800012E
:1092A000CAEC38F00C0E0501E96FE95100017FECC2
:1092B00013F00501E92B000109EC2CF0130E050158
:1092C000E95DF3E10101000E016ECBD0320E080121
:1092D000A86F0001DDEC28F00501E62BD8B4E72BE0
:1092E000ACD70001010166D00501036AE551D80F32
:1092F000E96E050E0320EA6EE4C5EFFF010139A512
:1093000017D0036A0501E551D80FE96E050E032059
:10931000EA6EEFCFE9F5E9C5A9F8370E0801AA6FA3
:109320000001ACEC37F0200E09EC2CF007D0010165
:10933000320E0801A86F0001DDEC28F00501E52BD5
:10934000E5510B0802E2E89334D0D851900831E19E
:10935000E55102082EE1D951410A00010FE0030A4C
:109360000DE0120A0BE0010A09E0030A07E0320AE5
:1093700005E0010A03E0030A01E001D019D005016C
:10938000E893010139A50FD00501E96BE95100010E
:1093900098EC13F00501E92B000109EC2CF0100EFC
:1093A0000501E95DF3E10501E76BE66B000100D023
:1093B000050101014ED00501E451900806E0E45199
:1093C000810803E0E451880826E1E56B036AE55172
:1093D000D80FE96E050E0320EA6EE4C5EFFF010128
:1093E00039A515D0036A0501E551D80FE96E050EC0
:1093F0000320EA6EEFCFE9F5E9C5A9F8370E0801B9
:10940000AA6F0001ACEC37F0200E09EC2CF005013E
:10941000E52BE8831ED0010139A514D05B0E0001B5
:1094200009EC2CF0E4C5A9F8370E0801AA6F000179
:10943000ACEC37F05D0E09EC2CF0200E09EC2CF0B2
:1094400007D00101320E0801A86F0001DDEC28F001
:109450000501320E0801A86F0001DDEC28F000D6EE
:1094600001010001000C050E0401F46F810EF56F7F
:10947000090EF66F040EF76FF86BFF0EF96F050E0D
:10948000FA6F810EFB6F090EFC6FFD6B020EFE6F13
:10949000FF0EFF6F050E0501006F810E016F090EB3
:1094A000026F040E036F330E046FFF0E056F050E7F
:1094B000066F810E076F090E086F040E096F480EC4
:1094C0000A6FFF0E0B6F050E0C6F810E0D6F090EEC
:1094D0000E6F040E0F6F3E0E106FFF0E116F050E14
:1094E000126F810E136F090E146F040E156F380E74
:1094F000166FFF0E176F050E186F810E196F090E8C
:109500001A6F040E1B6F4E0E1C6FFF0E1D6F050EA3
:109510001E6F810E1F6F090E206F040E216F470E04
:10952000226FFF0E236F050E246F810E256F090E2B
:10953000266F060E276F120E286FFF0E296F050E7D
:109540002A6F810E2B6F090E2C6F040E2D6F480EA3
:109550002E6FFF0E2F6F090E306F810E316F010ECF
:10956000326F040E336F4E0E346F356B366B376BC4
:10957000386BFF0E396F060E3A6FFF0E3B6F880E89
:109580003C6F010E3D6F3E6B3F6FFF0E406F060E4E
:10959000416F810E426F010E436F060E446F456F9F
:1095A000020E466FFF0E476F060E486F810E496F21
:1095B000010E4A6F060E4B6F4C6F030E4D6FFF0E80
:1095C0004E6F060E4F6F810E506F010E516F040EDD
:1095D000526F536B020E546FFF0E556F060E566F8F
:1095E000810E576F010E586F040E596F5A6B030EA0
:1095F0005B6FFF0E5C6F060E5D6F810E5E6F010E7E
:109600005F6F040E606F330E616F020E626FFF0EAC
:10961000636F060E646F810E656F010E666F040E38
:10962000676F330E686F030E696FFF0E6A6F060E69
:109630006B6F810E6C6F010E6D6F040E6E6F350EC9
:109640006F6F706BFF0E716F060E726F810E736F0E
:10965000010E746F040E756F350E766F030E776F03
:10966000FF0E786F060E796F810E7A6F010E7B6F99
:10967000040E7C6F3E0E7D6F020E7E6FFF0E7F6FBD
:10968000060E806F810E816F010E826F040E836F54
:109690003E0E846F030E856FFF0E866F060E876F7A
:1096A000810E886F010E896F040E8A6F380E8B6FE2
:1096B000020E8C6FFF0E8D6F060E8E6F810E8F6FF8
:1096C000010E906F040E916F380E926F030E936F20
:1096D000FF0E946F060E956F810E966F010E976FB9
:1096E000040E986F080E996F210E9A6FFF0E9B6FF4
:1096F000060E9C6F810E9D6F010E9E6F040E9F6F74
:10970000080EA06F310EA16FFF0EA26F060EA36FA1
:10971000810EA46F010EA56F040EA66F080EA76F31
:10972000A86BFF0EA96F050EAA6F810EAB6F010E1D
:10973000AC6F060EAD6F040EAE6FFF0EAF6F050E71
:10974000B06F810EB16F010EB26F060EB36F050ED2
:10975000B46FFF0EB56F070EB66F810EB76F010EB7
:10976000B86F040EB96F3F0EBA6F010EBB6FBC6BC2
:10977000FF0EBD6F050EBE6F810EBF6F010EC06F75
:10978000040EC16F080EC26FFF0EC36F050EC46FCB
:10979000810EC56F010EC66F040EC76F480EC86FED
:1097A000FF0EC96F050ECA6F890ECB6F010ECC6F0D
:1097B000CD6F030ECE6FFF0ECF6F050ED06F810EF3
:1097C000D16F090ED26F070ED36F220ED46FFF0E2A
:1097D000D56F0401F251010A0001D8B4A3D0030AE5
:1097E000D8B4A9D0010AD8B4AFD0070AD8B4B4D03D
:1097F000010AD8B4BAD0030AD8B4C0D00E0AD8B47B
:10980000C6D0010AD8B4CCD0030AD8B4D2D00D0A3D
:10981000D8B4D8D00C0AD8B4DED0070AD8B4E4D073
:109820000C0AD8B4EAD00D0AD8B4F0D0030AD8B4E0
:10983000F6D0010AD8B4FCD01F0AD8B402D1010A6C
:10984000D8B408D1020AD8B40ED1070AD8B41FD1AF
:10985000010AD8B433D1030AD8B447D1010AD8B425
:109860004AD10F0AD8B44DD1030AD8B47AD1070A25
:10987000D8B480D1010AD8B486D1030AD8B49BD118
:10988000010AD8B4B0D13F0AD8B4B6D1190AD8B4B5
:10989000BCD10C0AD8B4C2D1010AD8B4D0D1030AC1
:1098A000D8B4DED1010AD8B4ECD10E0AD8B4FAD1BA
:1098B000020AD8B407D2010AD8B40AD2180AD8B416
:1098C0000DD2070AD8B417D2010AD8B421D2030A9C
:1098D000D8B426D2010AD8B42CD20F0AD8B436D2C2
:1098E000010AD8B43CD2030AD8B447D2010AD8B48A
:1098F0004DD2070AD8B45ED2010AD8B46AD2030A9C
:10990000D8B476D2010AD8B47DD21F0AD8B482D294
:10991000010AD8B488D2030AD8B48ED20E0AD8B4B9
:1099200094D29CD2040E0801A56FF40EA46F00011E
:109930007FEC38F099D2040E0801A56FFA0EA46FDF
:1099400000017FEC38F090D2050E0801A56FA46BE2
:1099500000017FEC38F088D2050E0801A56F060ED5
:10996000A46F00017FEC38F07FD2050E0801A56FCF
:109970000C0EA46F00017FEC38F076D2050E0801C2
:10998000A56F120EA46F00017FEC38F06DD2050EAA
:109990000801A56F180EA46F00017FEC38F064D2A7
:1099A000050E0801A56F1E0EA46F00017FEC38F0B4
:1099B0005BD2050E0801A56F240EA46F00017FEC99
:1099C00038F052D2050E0801A56F2A0EA46F0001CF
:1099D0007FEC38F049D2050E0801A56F410EA46F47
:1099E00000017FEC38F040D2050E0801A56F480E4B
:1099F000A46F00017FEC38F037D2050E0801A56F87
:109A00003A0EA46F00017FEC38F02ED2050E08014B
:109A1000A56F4F0EA46F00017FEC38F025D2050E24
:109A20000801A56F560EA46F00017FEC38F01CD220
:109A3000050E0801A56F5D0EA46F00017FEC38F0E4
:109A400013D2050E0801A56F640EA46F00017FEC10
:109A500038F00AD2050E0801A56F6B0EA46F000145
:109A60007FEC38F001D201014D39006E0F0E001667
:109A700000500B0803E1050E0501776F050E080184
:109A8000A56F720EA46F00017FEC38F0EDD10101DB
:109A90004D39006E0F0E0016005006080AE0050E44
:109AA0000801A56F790EA46F00017FEC38F005D096
:109AB0000101010E016EE7D10001D6D101014D393E
:109AC000006E0F0E0016005006080AE0050E080191
:109AD000A56F800EA46F00017FEC38F005D0010166
:109AE000010E016ED0D10001BFD1020E0101572736
:109AF000000E5823000101015751D8B458075707E9
:109B000000010101585307E15751010804E3586B64
:109B1000010E576F08D0585303E157510D0803E267
:109B2000586B0E0E576F5831036E5731026E033269
:109B3000023203320232033202320F0E031602C027
:109B400037F50501010157510F0BE8CF38F5050135
:109B5000050E0801A56F300EA46F00017FEC38F0F0
:109B600083D1050E0801A56F870EA46F00017FEC5D
:109B700038F07AD1050E0801A56F8E0EA46F000192
:109B80007FEC38F071D101014D39006E0F0E0016D7
:109B90000050060804E1020E05019A6F03D0200E62
:109BA00005019A6F050E0801A56F950EA46F0001BF
:109BB0007FEC38F059D101014D39006E0F0E0016BF
:109BC0000050060804E1030E0501A16F03D0300E1A
:109BD0000501A16F050E0801A56F9C0EA46F000181
:109BE0007FEC38F041D1050E0801A56FA30EA46FDC
:109BF00000017FEC38F038D1050E0801A56FBE0ECC
:109C0000A46F00017FEC38F02FD1050E0801A56F7D
:109C1000CA0EA46F00017FEC38F026D1010E0101BD
:109C20008B5D0F0B0501BC6F020EBB6F050E0801AB
:109C3000A56FB60EA46F00017FEC38F015D1010EB0
:109C400001018B5D0F0B0501BC6F010EBB6F050E93
:109C50000801A56FB60EA46F00017FEC38F004D1A7
:109C6000010E01018B5D0F0B0501BC6F040EBB6F74
:109C7000050E0801A56FB60EA46F00017FEC38F049
:109C8000F3D0010E01018B5D0F0B0501BC6F030EBC
:109C9000BB6F050E0801A56FB60EA46F00017FEC27
:109CA00038F0E2D0010E01018B5D0F0B0501BC6F96
:109CB000BB6B050E0801A56FB60EA46F00017FEC0B
:109CC00038F0D2D0010E016E0101DDD00001CCD000
:109CD000010E016E0101D7D00001C6D00101415132
:109CE00088090501D66F08016C6B6D6B6E6F000102
:109CF00086EC3AF0B9D00101415108090501D66F4F
:109D000008016C6B6D6B6E6F000186EC3AF0ACD0A5
:109D100008016C6B6D6B6E6B000186EC3AF0A4D0A1
:109D200008016C6B6D6B41C16EF8000186EC3AF076
:109D30009BD001013D5180090501D66F08016C6B74
:109D40006D6F6E6B000186EC3AF08ED008016C6B83
:109D50003DC16DF86E6B000186EC3AF085D00101D3
:109D60003E5180090501D66FE8CF6CF808016D6B94
:109D70006E6B000186EC3AF077D03EC16CF80801BA
:109D80006D6B6E6B000186EC3AF06ED001013E51B6
:109D900080090501D66F01013D5180090501D76F8A
:109DA000D6C56CF8E8CF6DF808016E6B000186EC43
:109DB0003AF05AD001013D5180090501D66F3EC1EC
:109DC0006CF8E8CF6DF808016E6B000186EC3AF094
:109DD0004BD001013E5180090501D66FE8CF6CF8E8
:109DE0003DC16DF808016E6B000186EC3AF03CD085
:109DF0003EC16CF83DC16DF808016E6B000186EC48
:109E00003AF032D008016C6B6D6B6E6B000186EC22
:109E10003AF02AD0050E0801A56FC40EA46F000108
:109E20007FEC38F021D0050E0801A56FAA0EA46FB3
:109E300000017FEC38F018D0050E0801A56FB00EB8
:109E4000A46F00017FEC38F00FD0050E0801A56F5C
:109E5000D00EA46F00017FEC38F006D0000E016E2A
:109E6000010111D0000100D00401F32D09D0070E2B
:109E70000501D76FD00ED66F0001B5EC47F0040195
:109E8000010E016E01010001000C0401C36BC46BE3
:109E9000C56BD66B900ED76F0D0EF26F010EF36F80
:109EA000000133EC4AF0040EEA6EC60EE96E0801BA
:109EB000A16BA36B100EA26F000175EC30F03C0E8D
:109EC0000401F26FF36B000133EC4AF0010139A594
:109ED0000FD00401D86BD8510001E3EC12F004015B
:109EE000D82B000109EC2CF0110E0401D85DF3E130
:109EF0000001A8A142D0C4C45BFEC3C45AFE0E0137
:109F00005D6B320E5C6F0001A2EC34F002C0D9F43C
:109F100001C0D8F40401D95303E1D851C70820E2A5
:109F2000010139A50FD00401D86BD8510001FBEC19
:109F300012F00401D82B000109EC2CF00B0E0401E7
:109F4000D85DF3E10401C25308E10E0EF26F010E79
:109F5000F36F000133EC4AF00401000E016E69D08A
:109F6000320E0801A86F0001DDEC28F00401C32BBC
:109F7000D8B4C42B0101BCD70001A8B134D004016E
:109F8000D6510308D8B002D000012DD0000184ECD6
:109F900037F001C0C5F40A0E0801A86F0001DDEC1E
:109FA00028F00401D751C55D04E1D66BC5C4C6F4E1
:109FB0000AD0D62B036AD651C60FE96E040E0320D1
:109FC000EA6EC5C4EFFF010139A50BD0C5C4A9F8DD
:109FD000570E0801AA6F0001ACEC37F0200E09EC17
:109FE0002CF00001CAD7010139A508D00A0E0001E2
:109FF00009EC2CF00D0E09EC2CF001010401D651F6
:10A0000003080BE1C93D09D0C751500806E1C8510A
:10A01000020803E3010E016E0CD0C25308E10E0EDC
:10A02000F26F010EF36F000133EC4AF00401000EF1
:10A03000016E0001000C01014D390401F16F0F0E9A
:10A04000F117010EF15DF20F15E20E0F00013CEF6A
:10A0500050F0EFC4F2F4F0C4F3F433EC4AF004012E
:10A0600009D0EFC4F2F4F0C4F3F423EC41F004019E
:10A0700001D004010001000CF2CF0EF0F29EE824A2
:10A08000F76AF736A30FF66EA00EF722000EF86EF1
:10A09000FB6E0A00F550FA6E0800F5500EBEF28E07
:10A0A000F96E52A052A052A052A052A052A052A0AB
:10A0B00052A052A052A052A062A072A052A00401CD
:10A0C000996B9A6B9B6BAC6B900EAD6F040EEA6E46
:10A0D000AE0EE96E0801A16BA36B140EA26F000116
:10A0E00075EC30F0040EEA6E9C0EE96E0801A16B6F
:10A0F000A36B100EA26F000175EC30F0020E04018C
:10A10000F26FF36B000133EC4AF0010139A50FD077
:10A110000401C26BC251000111EC10F00401C22B0A
:10A12000000109EC2CF00E0E0401C25DF3E1000108
:10A13000A8A137D09AC45BFE99C45AFE0E015D6B8C
:10A14000320E5C6F0001A2EC34F002C0C3F401C017
:10A15000C2F40401C35303E1C251C70815E201016F
:10A1600039A510D00401C26BC251000128EC10F0D7
:10A170000401C22B000109EC2CF00A0E0401C25D9F
:10A18000F3E10101C4EF54F0320E0801A86F0001A1
:10A19000DDEC28F00401992BD8B49A2B0101C7D724
:10A1A0000001A8B134D00401AC510F08D8B002D0DE
:10A1B00000012DD0000184EC37F001C09BF40A0EA1
:10A1C0000801A86F0001DDEC28F00401AD519B5D92
:10A1D00004E1AC6B9BC49CF40AD0AC2B036AAC5179
:10A1E0009C0FE96E040E0320EA6E9BC4EFFF010191
:10A1F00039A50BD09BC4A9F8570E0801AA6F00011E
:10A20000ACEC37F0200E09EC2CF00001CAD70101AC
:10A2100039A507D00A0E000109EC2CF00D0E09EC4F
:10A220002CF00401AC510408D8B034D39EC494F48B
:10A230009FC493F4A0C496F4A1C495F4A2C498F466
:10A24000A3C497F495C400F096C403F0040E965D81
:10A2500006E1020E005C0001D8B464D00401080ECF
:10A26000035C05E100520001D8B4C4D00401040E1F
:10A27000035C06E10D0E005C0001D8B4F8D00401C7
:10A28000040E035C06E10E0E005C0001D8B424D17C
:10A290000401050E035C06E1030E005C0001D8B466
:10A2A00051D10401050E035C06E1010E005C0001C2
:10A2B000D8B448D10401040E035C06E10F0E005C23
:10A2C0000001D8B4A9D10401050E035C06E1050E16
:10A2D000005C0001D8B4D5D10401050E035C06E191
:10A2E000040E005C0001D8B402D20401040E035C29
:10A2F00006E12C0E005C0001D8B463D20401200EEC
:10A30000035C06E1010E005C0001D8B45AD20401DE
:10A31000040E035C06E12D0E005C0001D8B451D29E
:10A32000040185D201014D6B010E0401C26F0001D1
:10A33000ACDD012C2BD0600E01014D1339A510D0DE
:10A340000401C26BC25100013DEC10F00401C22BAC
:10A35000000109EC2CF0140E0401C25DF3E10101CF
:10A36000040EEA6EAE0EE96EF2CFC2F4F29E000E5B
:10A37000000157EC10F00A000900F550EE6E0009DC
:10A38000FBE10401C2BFF28E29D0000101014D8919
:10A3900039A510D00401C26BC25100016FEC10F05E
:10A3A0000401C22B000109EC2CF0100E0401C25D67
:10A3B000F3E10101040EEA6EAE0EE96EF2CFC2F4D3
:10A3C000F29E000E000187EC10F00A000900F55023
:10A3D000EE6E0009FBE10401C2BFF28E925130091A
:10A3E000BE6F040E08017A6FAE0E796F0001C3ECE8
:10A3F00030F04ED201014D6B500E4D1339A510D0E7
:10A400000401C26BC25100019FEC10F00401C22B89
:10A41000000109EC2CF0140E0401C25DF3E101010E
:10A42000040EEA6EAE0EE96EF2CFC2F4F29E000E9A
:10A430000001B9EC10F00A000900F550EE6E0009B9
:10A44000FBE10401C2BFF28E92513009BE6F040ECF
:10A4500008017A6FAE0E796F0001C3EC30F0390E4F
:10A460000401EF6F010EF06F0001E5DD11D2010173
:10A470004D6B4D8B39A510D00401C26BC251000148
:10A48000D1EC10F00401C22B000109EC2CF0110EEC
:10A490000401C25DF3E10101040EEA6EAE0EE96E45
:10A4A000F2CFC2F4F29E000E0001E9EC10F00A00B7
:10A4B0000900F550EE6E0009FBE10401C2BFF28E07
:10A4C00092513009BE6F040E08017A6FAE0E796F9B
:10A4D0000001C3EC30F0DCD101014D6B300E4D13A7
:10A4E00039A510D00401C26BC251000101EC11F07A
:10A4F0000401C22B000109EC2CF0100E0401C25D16
:10A50000F3E10101040EEA6EAE0EE96EF2CFC2F481
:10A51000F29E000E000119EC11F00A000900F5503E
:10A52000EE6E0009FBE10401C2BFF28E92513009C8
:10A53000BE6F040E08017A6FAE0E796F0001C3EC96
:10A5400030F0A6D10401952D32D0965105082FE1A7
:10A55000932D2DD094532BE101014D6B900E4D1393
:10A5600039A510D00401C26BC251000131EC11F0C9
:10A570000401C22B000109EC2CF0110E0401C25D94
:10A58000F3E10101040EEA6EAE0EE96EF2CFC2F401
:10A59000F29E000E000149EC11F00A000900F5508E
:10A5A000EE6E0009FBE10401C2BFF28E29D0010169
:10A5B0004D6B4D8939A510D00401C26BC251000109
:10A5C00061EC11F00401C22B000109EC2CF00F0E1C
:10A5D0000401C25DF3E10101040EEA6EAE0EE96E04
:10A5E000F2CFC2F4F29E000E000178EC11F00A00E6
:10A5F0000900F550EE6E0009FBE10401C2BFF28EC6
:10A6000092513009BE6F040E08017A6FAE0E796F59
:10A610000001C3EC30F03CD101014D6B4D8F39A5E9
:10A6200010D00401C26BC251000190EC11F0040182
:10A63000C22B000109EC2CF0100E0401C25DF3E105
:10A640000101040EEA6EAE0EE96EF2CFC2F4F29E84
:10A65000000E0001A8EC11F00A000900F550EE6EA2
:10A660000009FBE10401C2BFF28E92513009BE6FB6
:10A67000040E08017A6FAE0E796F0001C3EC30F062
:10A6800007D101014D6B700E4D1339A510D0040197
:10A69000C26BC2510001C0EC11F00401C22B0001D9
:10A6A00009EC2CF0110E0401C25DF3E10101040E6E
:10A6B000EA6EAE0EE96EF2CFC2F4F29E000E000119
:10A6C000D8EC11F00A000900F550EE6E0009FBE12C
:10A6D0000401C2BFF28E92513009BE6F040E080110
:10A6E0007A6FAE0E796F0001C3EC30F0D1D0040167
:10A6F00097510E0831E198510E082EE101014D6B82
:10A70000B00E4D1339A510D00401C26BC251000127
:10A71000F0EC11F00401C22B000109EC2CF0100E3A
:10A720000401C25DF3E10101040EEA6EAE0EE96EB2
:10A73000F2CFC2F4F29E000E000108EC12F00A0003
:10A740000900F550EE6E0009FBE10401C2BFF28E74
:10A7500092513009BD6F2CD001014D6B4D8D39A543
:10A7600010D00401C26BC251000120EC12F00401B0
:10A77000C22B000109EC2CF0100E0401C25DF3E1C4
:10A780000101040EEA6EAE0EE96EF2CFC2F4F29E43
:10A79000000E000138EC12F00A000900F550EE6ED0
:10A7A0000009FBE10401C2BFF28E92513009BE6F75
:10A7B000040E08017A6FAE0E796F0001C3EC30F021
:10A7C00067D001014D6BA00E4D1339A510D00401C7
:10A7D000C26BC251000150EC12F00401C22B000107
:10A7E00009EC2CF0160E0401C25DF3E10101040E28
:10A7F000EA6EAE0EE96EF2CFC2F4F29E000E0001D8
:10A800006BEC12F00A000900F550EE6E0009FBE156
:10A810000401C2BFF28E92513009BE6F040E0801CE
:10A820007A6FAE0E796F0001C3EC30F031D00101C8
:10A8300039A510D00401C26BC251000183EC12F0A3
:10A840000401C22B000109EC2CF0100E0401C25DC2
:10A85000F3E101014D6B040EEA6EAE0EE96EF2CF2C
:10A86000C2F4F29E000E00019BEC12F00A000900F7
:10A87000F550EE6E0009FBE10401C2BFF28E040E3A
:10A8800008017A6FAE0E796F0001C3EC30F000D092
:10A890007AD00401AC51030846E19F3D44D09D515C
:10A8A000600803E09D5161083EE1C26B000145EC88
:10A8B0004FF0012C38D001014D6B600E4D1339A5BE
:10A8C00010D00401C26BC2510001B2EC12F00401BD
:10A8D000C22B000109EC2CF0130E0401C25DF3E160
:10A8E0000101040EEA6EAE0EE96EF2CFC2F4F29EE2
:10A8F000000E0001CBEC12F00A000900F550EE6EDC
:10A900000009FBE10401C2BFF28E92513009BE6F13
:10A91000040E08017A6FAE0E796F0001C3EC30F0BF
:10A92000010132D00001010139A510D00401C26B30
:10A93000C251000183EC12F00401C22B000109ECAA
:10A940002CF0100E0401C25DF3E101014D6B040E09
:10A95000EA6EAE0EE96EF2CFC2F4F29E000E000176
:10A960009BEC12F00A000900F550EE6E0009FBE1C5
:10A970000401C2BFF28E040E08017A6FAE0E796F29
:10A980000001C3EC30F001010001D6EF61F00801D5
:10A990007A6B7B6B7C6B7D6B7E6B795303E07951BB
:10A9A000060828E27F6B7F510001A0EC08F0080147
:10A9B0007F2B000109EC2CF0190E08017F5DF3E1FB
:10A9C00079C87FF81F0E806F0001FDEC37F01B0E79
:10A9D00008017F6F7F510001A0EC08F008017F2B78
:10A9E000000109EC2CF0210E08017F5DF3E1000E5F
:10A9F000016E7AD079C8D7F17D6B010E7C6F7D53E3
:10AA000073E17C510C0870E37B6B900E7A6F010E42
:10AA1000795D036A7F6F03C080F87BC85BFE7AC8EC
:10AA20005AFE03C05DFEE8CF5CFE0001A2EC34F0EC
:10AA300002C07BF801C07AF8200E08017A27000EC8
:10AA40007B23010E7C5D7F6F000E7D59806FE8CF08
:10AA50005BFE7FC85AFE0E015D6B0C0E5C6F000141
:10AA6000A2EC34F0015008017A2702507B23F2CF88
:10AA70007FF8F29E7BC8AAFF7AC8A9FFA69CA69E73
:10AA8000A680A8507FBFF28E7E6F7E51F00B09E04A
:10AA9000D70E7C25E96E010E7D21EA6EFF0EEF6E6A
:10AAA00007D0D70E7C25E96E010E7D21EA6EEF6A94
:10AAB000010139A514D0D70E08017C25E96E010EDD
:10AAC0007D21EA6EEFCF7FF87FC8A9F8570EAA6FF5
:10AAD0000001ACEC37F0200E09EC2CF0010108016C
:10AAE0007C2BD8B47D2B8BD70001000C0F0E0401FA
:10AAF000A76F810EA86F010EA96F060EAA6F020E36
:10AB0000AB6FAC6BAD6BAE6BAF6BB06BB16BB26B75
:10AB1000B36BB46BB56BFF0EB66FB76F090EB86F42
:10AB2000810EB96F010EBA6F040EBB6F470EBC6F7A
:10AB3000BD6BBE6BBF6BC06BFF0EC16F090EC26FEA
:10AB4000810EC36F010EC46F040EC56F480EC66F31
:10AB5000C76BC86BC96BCA6BFF0ECB6F090ECC6F8E
:10AB6000810ECD6F010ECE6F040ECF6F4E0ED06FE3
:10AB7000D16BD26BD36BD46BFF0ED56F070ED66F34
:10AB800001014D39006E0F0E001600500A08D8B4AE
:10AB9000CCD03EC1ACF43DC1ADF44D39006E0F0ECA
:10ABA0000016005008080EE04D39006E0F0E00161A
:10ABB0000050070807E04D39006E0F0E00160050D8
:10ABC000090811E10401A72B036AD651A70FE96E0A
:10ABD000040E0320EA6E01014E510F0BEF6E0401CB
:10ABE000D62BAD6B0101036A0401D651A70FE96EA4
:10ABF000040E0320EA6E010150390401D96F0F0ED3
:10AC0000D917D9510F0BEF6E010ED625036AA70F86
:10AC1000E96E040E0320EA6E50C1D9F4D9510F0B2E
:10AC2000EF6E020ED625036AA70FE96E040E03200D
:10AC3000EA6E010150310401DA6F01014F31040164
:10AC4000D96FDA33D933DA33D933DA33D9330F0E54
:10AC5000DA17D9510F0BEF6E030ED625036AA70F33
:10AC6000E96E040E0320EA6E01014F510F0BEF6EE7
:10AC7000040E0401D625036AA70FE96E040E032013
:10AC8000EA6E010152390401D96F0F0ED917D9515B
:10AC90000F0BEF6E050ED625036AA70FE96E040EA3
:10ACA0000320EA6E52C1D9F4D9510F0BEF6E060E94
:10ACB000D625036AA70FE96E040E0320EA6E010190
:10ACC00052310401DA6F010151310401D96FDA33D5
:10ACD000D933DA33D933DA33D9330F0EDA17D951FE
:10ACE0000F0BEF6E070ED625036AA70FE96E040E51
:10ACF0000320EA6E010151510F0BEF6E040E0801A3
:10AD0000A56FA70EA46F00017FEC38F04E0E050171
:10AD1000D76F200ED66F0001B5EC47F0012C01D0A3
:10AD200003D0000E016E4CD101014D39006E0F0EA3
:10AD300000160050050805E1010E016E000140D12A
:10AD4000010154390401D76F0F0ED717D7510F0BDC
:10AD5000BD6F54C1D7F4D7510F0BBE6F01015431F1
:10AD60000401D86F010153310401D76FD833D733B1
:10AD7000D833D733D833D7330F0ED817D7510F0B5B
:10AD8000BF6F010153510F0BE8CFC0F40401040E53
:10AD90000801A56FB80EA46F00017FEC38F0070E14
:10ADA0000501D76FD00ED66F0001B5EC47F0012C2E
:10ADB00001D003D0000E016E03D101014DA70AD0CE
:10ADC0001B0E0401EF6F010EF06F00011BEC50F041
:10ADD00059D001011C0E0401EF6F010EF06F00014C
:10ADE0001BEC50F001014D39006E0F0E00160050A3
:10ADF0000B080CE138B909D0370E0401EF6F010ED2
:10AE0000F06F00011BEC50F001013DD056390401F8
:10AE1000D76F0F0ED717D7510F0BC76F56C1D7F487
:10AE2000D7510F0BC86F010156310401D86F0101D2
:10AE300055310401D76FD833D733D833D733D8330C
:10AE4000D7330F0ED817D7510F0BC96F01015551CA
:10AE50000F0BE8CFCAF40401040E0801A56FC20E5F
:10AE6000A46F00017FEC38F0030E0501D76FE80EE8
:10AE7000D66F0001B5EC47F0012C01D003D0000ED5
:10AE8000016E9ED001014DA542D0140E0401EF6F5A
:10AE9000010EF06F00011BEC50F00101586B070E22
:10AEA000576FD8908A35036A3A0F016E000E03225D
:10AEB0000150380FE96E010E0320EA6E58C1ECFF15
:10AEC000ED5257C1EFFF0401D16BD26BD36B01017F
:10AED00057510F0BE8CFD4F40401040E0801A56FFD
:10AEE000CC0EA46F00017FEC38F0030E0501D76F84
:10AEF000E80ED66F0001B5EC47F0150E0401EF6FB8
:10AF0000010EF06F00011BEC50F046D00101140E51
:10AF10000401EF6F010EF06F00011BEC50F0010116
:10AF200058390401D76F0F0ED717D7510F0BD16FB8
:10AF300058C1D7F4D7510F0BD26F0101583104011A
:10AF4000D86F010157310401D76FD833D733D833C5
:10AF5000D733D833D7330F0ED817D7510F0BD36F42
:10AF6000010157510F0BE8CFD4F40401040E08017E
:10AF7000A56FCC0EA46F00017FEC38F0030E050125
:10AF8000D76FE80ED66F0001B5EC47F0012C01D069
:10AF900003D0000E016E14D001014DA109D00F0E97
:10AFA0000401EF6F010EF06F00011BEC50F008D0B0
:10AFB000100E0401EF6F010EF06F00011BEC50F05A
:10AFC0005CEF5EF00401FE6BFF6B0501006B01910D
:10AFD000040EEA6EF10EE96E0801A16BA36B0D0E73
:10AFE000A26F000175EC30F0A8A158D000C55BFE3F
:10AFF000FFC45AFE0E015D6B190E5C6F0001A2ECDE
:10B0000034F002C003F501C002F50401F05105015E
:10B01000025C35E305E10401EF510501025D2FE318
:10B02000010139A529D00501026B02510001E5ECAF
:10B0300013F00501022B000109EC2CF0180E05019C
:10B04000025DF3E1100EE96EF0C498F8EFC497F8D2
:10B050000001CAEC38F01B0E0501026F025100011D
:10B06000E5EC13F00501022B000109EC2CF0220E97
:10B070000501025DF3E10101FF0E016EFCD0190E26
:10B080000801A86F0001DDEC28F00401FF2BD8A413
:10B0900003D00501002B04010001A6D7010139A549
:10B0A0000FD00501026B0251000106EC14F00501FE
:10B0B000022B000109EC2CF0100E0501025DF3E1FA
:10B0C0000001A8B1D5D0036A0401FE51F10F016E51
:10B0D000040E032201C002F503C003F5000184EC55
:10B0E00037F003C5EAFF02C5E9FF01C0EFFF010128
:10B0F00039A515D0036A0401FE51F10FE96E040E63
:10B100000320EA6EEFCF02F502C5A9F8370E080159
:10B11000AA6F0001ACEC37F0200E09EC2CF0050111
:10B1200001B11BD0036A0401FE51F10FE96E040E58
:10B130000320EA6EEF50FE080EE1036AFE51F10FA4
:10B14000E96E040E0320EA6EEFCFF1F405010181F0
:10B15000010E0401FE6F82D00501036A0401FE5155
:10B16000F10FE96E040E0320EA6EEF50EF0866E17E
:10B17000010139A508D00D0E000109EC2CF00A0ED2
:10B1800009EC2CF0010139A546D00401F4510F0B54
:10B19000006E00380501026FF00E02170401F55130
:10B1A0000F0B05010213036B035100011EEC14F099
:10B1B0000501032B000109EC2CF00D0E0501035DC8
:10B1C000F3E1F4C4A9F8570E0801AA6F0001ACEC32
:10B1D00037F02C0E09EC2CF0F5C4A9F8570E080135
:10B1E000AA6F0001ACEC37F0200E09EC2CF0280E11
:10B1F00009EC2CF002C5A9F8570E0801AA6F00014E
:10B20000ACEC37F0290E09EC2CF00D0E09EC2CF00B
:10B210000A0E09EC2CF00401F4510F0B006E0038FB
:10B220000501026FF00E02170401F5510F0B050125
:10B230000211016E01011FD007D00401320E080176
:10B24000A86F0001DDEC28F00401FE510B0802E3B9
:10B25000FE2B04D0FE6B0501019104010001A8A1A1
:10B2600006D0320E0801A86F0001DDEC28F029D7C6
:10B27000EE0E016E01010001000C0E0E0401A76F1D
:10B28000FF0EA86F300EA96FAA6FAB6B620EAC6F8A
:10B29000AD6BAE6BAF6BB06BB16BB26BB36BB46BD2
:10B2A000EF0EB56F0A0EB66FFF0EB76F300EB86FA8
:10B2B000B96FBA6BB30EBB6FBC6BBD6BBE6BBF6BB4
:10B2C000EF0EC06F0A0EC16FFF0EC26F300EC36F5C
:10B2D000C46FC56BB00EC66FC76BC86BC96BCA6B4A
:10B2E000EF0ECB6F090ECC6FFF0ECD6F300ECE6F11
:10B2F000CF6FD06B500ED16FD26BD36BD46BEF0E80
:10B30000D56F090ED66FFF0ED76F300ED86FD96F7D
:10B31000DA6B510EDB6FDC6BDD6BDE6BEF0EDF6F1C
:10B32000080EE06FFF0EE16F300EE26FE36FE46B2B
:10B33000B40EE56F310EE66FE76BEF0EE86FE96B69
:10B34000EA6BEB6BEC6BED6BEE6B036A3EC1EFF4FB
:10B3500003C0F0F40E015B6B210E5A6F03C05DFE5B
:10B360003EC15CFE0001A2EC34F0080E0401012491
:10B37000EB6F000E0220EC6FEC5306E1EB51090875
:10B3800003E3EC6B0A0EEB6FEC51020809E2FF0AD3
:10B3900003E1EB51200804E2030EEC6F200EEB6F8B
:10B3A000EC510F0BEF6FE8CFA5F80001B3EC3BF0C9
:10B3B00001C0D2F40401EBC400F0003A0F0E0016F5
:10B3C00000500F0BEF6FE8CFA5F80001B3EC3BF096
:10B3D00001C0D3F40401EB510F0BEF6FE8CFA5F8D8
:10B3E0000001B3EC3BF001C0D4F4040E0801A56FDA
:10B3F000CC0EA46F00017FEC38F0030E0401F06F57
:10B40000E80EEF6F0001DEDD01C0EEF40401EE5343
:10B4100030E0EE51100803E0EE51500824E1020E36
:10B42000EF6FFA0E0801A86F0001DDEC28F00401AF
:10B43000EF2FF7D7040E0801A56FCC0EA46F000103
:10B440007FEC38F0030E0501F86FE80EF76F00018E
:10B450001AEC40F0012C01D004D0000E016E38EF40
:10B460005EF006D00401000E016E000138EF5EF0C0
:10B470000401036A3DC1EFF403C0F0F40E015B6BFD
:10B480001E0E5A6F03C05DFE3DC15CFE0001A2ECC2
:10B4900034F0080E04010124E96F000E0220EA6F67
:10B4A000EA5306E1E951070803E3EA6B080EE96F86
:10B4B000EA51010809E2FF0A03E1E9516E0804E2DA
:10B4C000020EEA6F6E0EE96FEA510F0BEF6FE8CFD5
:10B4D000A5F80001B3EC3BF001C0DCF40401E9C4C1
:10B4E00000F0003A0F0E001600500F0BEF6FE8CF80
:10B4F000A5F80001B3EC3BF001C0DDF40401E95113
:10B500000F0BEF6FE8CFA5F80001B3EC3BF001C0E3
:10B51000DEF4040E0801A56FD60EA46F00017FECC7
:10B5200038F0030E0401F06FE80EEF6F00014ADD02
:10B5300001C0EEF40401EE532DE0EE51100803E0DB
:10B54000EE51500823E1020EEF6FFA0E0801A86FCA
:10B550000001DDEC28F00401EF2FF7D7040E0801FD
:10B56000A56FD60EA46F00017FEC38F0030E050125
:10B57000F86FE80EF76F00011AEC40F0012C01D0D3
:10B5800003D0000E016E74D305D00401000E016ECD
:10B5900000016ED3010150390401EF6FF06B0F0E03
:10B5A000EF17EF510F0B006E036AEF6FE8CFA5F8AE
:10B5B0000001B3EC3BF001C0ADF450C1EFF4040165
:10B5C000F06BEF510F0B006E036AEF6FE8CFA5F839
:10B5D0000001B3EC3BF001C0AEF4010150310401B5
:10B5E000F06F01014F310401EF6FF033EF33F033AF
:10B5F000EF33F033EF330F0EF017EF510F0B006EF8
:10B60000036AEF6FE8CFA5F80001B3EC3BF001C08F
:10B61000AFF401014F510F0B006E036AE8CFEFF456
:10B62000E8CFA5F80001B3EC3BF001C0B0F4010194
:10B6300052390401EF6FF06B0F0EEF17EF510F0B44
:10B64000006E036AEF6FE8CFA5F80001B3EC3BF0A2
:10B6500001C0B1F452C1EFF40401F06BEF510F0BD4
:10B66000006E036AEF6FE8CFA5F80001B3EC3BF082
:10B6700001C0B2F4010152310401F06F01015131F6
:10B680000401EF6FF033EF33F033EF33F033EF3388
:10B690000F0EF017EF510F0B006E036AEF6FE8CF3C
:10B6A000A5F80001B3EC3BF001C0B3F40101515126
:10B6B0000F0B006E036AE8CFEFF4E8CFA5F80001A6
:10B6C000B3EC3BF001C0B4F4040E0801A56FA70E63
:10B6D000A46F00017FEC38F0170E0401F06F700EBC
:10B6E000EF6F00016FDC01C0EEF40401EE532EE0B9
:10B6F000EE51100803E0EE51500823E1080EEF6F01
:10B70000FA0E0801A86F0001DDEC28F00401EF2F0C
:10B71000F7D7040E0801A56FA70EA46F00017FECF8
:10B7200038F0070E0501F86FD00EF76F00011AEC24
:10B7300040F0012C01D003D0000E016E99D205D04B
:10B740000401000E016E000193D20401ED5301E1EA
:10B75000ED6BED51070802E2070EED6F370EE76F54
:10B76000040E0801A56FE00EA46F00017FEC38F015
:10B77000030E0401F06FE80EEF6F000123DC01C03F
:10B78000EEF40401EE532DE0EE51100803E0EE510B
:10B79000500823E1020EEF6FFA0E0801A86F0001B6
:10B7A000DDEC28F00401EF2FF7D7040E0801A56F98
:10B7B000E00EA46F00017FEC38F0030E0501F86F76
:10B7C000E80EF76F00011AEC40F0012C01D003D015
:10B7D000000E016E4DD205D00401000E016E000175
:10B7E00047D2010154390401EF6FF06B0F0EEF17D0
:10B7F000EF510F0B006E036AEF6FE8CFA5F8000161
:10B80000B3EC3BF001C0BCF454C1EFF40401F06BA5
:10B81000EF510F0B006E036AEF6FE8CFA5F8000140
:10B82000B3EC3BF001C0BDF4010154310401F06FF1
:10B83000010153310401EF6FF033EF33F033EF3395
:10B84000F033EF330F0EF017EF510F0B006E036A5A
:10B85000EF6FE8CFA5F80001B3EC3BF001C0BEF4F8
:10B86000010153510F0B006E036AE8CFEFF4E8CFEC
:10B87000A5F80001B3EC3BF001C0BFF4040E0801D1
:10B88000A56FB60EA46F00017FEC38F0030E040123
:10B89000F06FE80EEF6F0001E2EC57F001C0EEF43C
:10B8A0000401EE5328E0EE51100803E0EE51500879
:10B8B00022E1080EEF6FFA0E0801A86F0001DDEC1F
:10B8C00028F00401EF2FF7D7040E0801A56FB60E7C
:10B8D000A46F00017FEC38F0070E0501F86FD00E61
:10B8E000F76F00011AEC40F0012C01D003D0000EDC
:10B8F000016EBED1040101014DA742D01B0E04010F
:10B90000EF6FF06B00011BEC50F0030E0401F06FC1
:10B91000E80EEF6F0001E2EC57F001C0EEF4040115
:10B92000EE532CE0EE51100803E0EE51500821E1F7
:10B93000040EEF6FFA0E0801A86F0001DDEC28F08D
:10B940000401EF2FF7D71B0EEF6FF06B00011BEC1C
:10B9500050F0030E0501F86FE80EF76F00011AECC6
:10B9600040F0012C01D003D0000E016E81D105D032
:10B970000401000E016E00017BD10401FCD0010125
:10B980001C0E0401EF6FF06B00011BEC50F0030E76
:10B990000401F06FE80EEF6F0001E2EC57F001C018
:10B9A000EEF40401EE532BE0EE51100803E0EE51EB
:10B9B000500821E1040EEF6FFA0E0801A86F000194
:10B9C000DDEC28F00401EF2FF7D71C0EEF6FF06BC2
:10B9D00000011BEC50F0030E0501F86FE80EF76F45
:10B9E00000011AEC40F0012C01D003D0000E016ED2
:10B9F0003FD105D00401000E016E000139D10101D3
:10BA000056390401EF6FF06B0F0EEF17EF510F0B6C
:10BA1000006E036AEF6FE8CFA5F80001B3EC3BF0CE
:10BA200001C0C7F456C1EFF40401F06BEF510F0BE6
:10BA3000006E036AEF6FE8CFA5F80001B3EC3BF0AE
:10BA400001C0C8F4010156310401F06F0101553104
:10BA50000401EF6FF033EF33F033EF33F033EF33B4
:10BA60000F0EF017EF510F0B006E036AEF6FE8CF68
:10BA7000A5F80001B3EC3BF001C0C9F40101555138
:10BA80000F0B006E036AE8CFEFF4E8CFA5F80001D2
:10BA9000B3EC3BF001C0CAF4040E0801A56FC10E5F
:10BAA000A46F00017FEC38F0070E0401F06FD00E98
:10BAB000EF6F0001E2EC57F001C0EEF40401EE5329
:10BAC0005AE0EE51100803E0EE5150084FE1080E25
:10BAD000EF6FFA0E0801A86F0001DDEC28F00401F9
:10BAE000EF2FF7D7040E0801A56FC10EA46F000158
:10BAF0007FEC38F0070E0401F06FD00EEF6F0001FD
:10BB0000E2EC57F001C0EEF40401EE532EE0EE51EA
:10BB1000100803E0EE51500823E1080EEF6FFA0E13
:10BB20000801A86F0001DDEC28F00401EF2FF7D722
:10BB3000040E0801A56FC10EA46F00017FEC38F060
:10BB4000070E0501F86FD00EF76F00011AEC40F0F8
:10BB5000012C01D003D0000E016E8AD005D0040163
:10BB6000000E016E000184D0040105D0000E016EAC
:10BB700000017ED0040101014DA309D0110E040182
:10BB8000EF6F010EF06F00011BEC50F008D0130EA8
:10BB90000401EF6F010EF06F00011BEC50F0640E1A
:10BBA0000801A86F0001DDEC28F001014DB10AD0B9
:10BBB000100E0401EF6F010EF06F00011BEC50F04E
:10BBC00009D001010F0E0401EF6F010EF06F0001AB
:10BBD0001BEC50F0640E0801A86F0001DDEC28F0AA
:10BBE00001014DA52FD0586B480E576FD8908A355C
:10BBF000036A3A0F016E000E03220150380FE96EFE
:10BC0000010E0320EA6E58C1ECFFED5257C1EFFF61
:10BC1000140E0401F26F010EF36F000123EC41F0EA
:10BC2000180E0401F26F010EF36F000123EC41F0D6
:10BC3000150E0401F26F010EF36F000123EC41F0C9
:10BC400011D00101140E0401F26F010EF36F000117
:10BC500023EC41F0180E0401F26F010EF36F0001A6
:10BC600023EC41F0640E0801A86F0001DDEC28F020
:10BC700061EF5EF001014D39006E0F0E00160050AD
:10BC8000020A000117E0010A15E0060A13E00D0A96
:10BC900011E0010A0FE00E0A0DE0030A0BE00F0AA3
:10BCA00009E00A0A07E0070A05E00C0A03E0060AB1
:10BCB00006E00AD076EF55F001500AD009D03DEFEA
:10BCC00059F0015005D004D0000E016E01D000D013
:10BCD000000C92C479F8C7EC54F00101E33D2AD07E
:10BCE00092C4A7F40C0E0401A86F0001B3EC34F069
:10BCF000012C1FD0040EEA6E930EE96EF2CFA7F46A
:10BD0000F29E000ECEEC21F00A000900F550EE6E16
:10BD10000009FBE10401A7BFF28E040E08017A6F4F
:10BD2000930E796F0001C3EC30F0A4DF010E016EB9
:10BD30002BD00101040EEA6E930EE96EF2CFA7F448
:10BD4000F29E000E0001E6EC21F00A000900F55019
:10BD5000EE6E0009FBE10401A7BFF28E040E08019C
:10BD60007A6F930E796F0001C3EC30F0080E040176
:10BD7000A76FFA0E0801656F0001C8EC28F00401F6
:10BD8000A72FF7D7000E016E0001000C0401AF5180
:10BD9000390805E2370EAF5D016E05D004D0300ED4
:10BDA000AF5D016E00D00001000C0401A76BA86B11
:10BDB000A96B020EAA6F900EAB6F95C4E9FF96C4F3
:10BDC000EAFFEC6AED52EF6A040EEA6E970EE96E36
:10BDD0000801A16BA36B100EA26F000175EC30F08F
:10BDE00001014D39006E0F0E001600500C0805E1E0
:10BDF000050E0401AA6FFE0EAB6F020E0401AC6FBC
:10BE0000C80E0801A86F0001DDEC28F00401AC2F7A
:10BE1000F7D70001A8B13BD00401A7510F08D8B053
:10BE200002D0000134D0000184EC37F001C0A8F446
:10BE30000A0E0801A86F0001DDEC28F0010139A508
:10BE40000DD0A8C4A9F8570E0801AA6F0001ACECE8
:10BE500037F0200E09EC2CF007D001010A0E080182
:10BE6000A86F0001DDEC28F00401AB51A85D04E1EE
:10BE7000A76BA8C497F40AD0A72B036AA751970F02
:10BE8000E96E040E0320EA6EA8C4EFFFC2D7030ECA
:10BE90000401AA25A75D03E2000E016E6FD0010127
:10BEA0004D39006E0F0E001600500C0829E1AAC48F
:10BEB000A9F4030E0401AA25A95D01E022E2036AA8
:10BEC000A951970F016E040E032201C0ACF403C008
:10BED000ADF4036AA951970FE96E040E0320EA6ED0
:10BEE000EFCFAEF4AEC4AFF4000150DFADC4EAFF53
:10BEF000ACC4E9FF01C0EFFF0401A92B0101D9D7B0
:10BF00000401A96BA951030837E395C4E9FF96C45E
:10BF1000EAFFEF34026EEC34036E0236033602366B
:10BF2000033602360336F00E02160250ED52EF6E63
:10BF300003C0ECFF96C403F096C4EAFF95C4E9FF82
:10BF4000ECCFAFF4ED52EFCFAEF4A951AA25036ABE
:10BF5000970FE96E040E0320EA6EEF500F0BAE113F
:10BF6000AFC403F096C4EAFF95C4E9FFAFC4ECFF89
:10BF7000ED52EF6EA92BC6D7010E016E0001000C29
:10BF80000401A76BA86B020EA96F900EAA6F95C44F
:10BF9000E9FF96C4EAFFEF6A040EEA6E970EE96EB7
:10BFA0000801A16BA36B100EA26F000175EC30F0BD
:10BFB00001014D39006E0F0E001600500C0805E10E
:10BFC000050E0401A96FFE0EAA6F020E0401AB6FED
:10BFD000C80E0801A86F0001DDEC28F00401AB2FAA
:10BFE000F7D70001A8B13BD00401A7510F08D8B082
:10BFF00002D0000134D0000184EC37F001C0A8F475
:10C000000A0E0801A86F0001DDEC28F0010139A536
:10C010000DD0A8C4A9F8570E0801AA6F0001ACEC16
:10C0200037F0200E09EC2CF007D001010A0E0801B0
:10C03000A86F0001DDEC28F00401AA51A85D04E11D
:10C04000A76BA8C497F40AD0A72B036AA751970F30
:10C05000E96E040E0320EA6EA8C4EFFFC2D7020EF9
:10C060000401A925A75D03E2000E016E7CD0010149
:10C070004D39006E0F0E001600500C083EE1036AA9
:10C080000401A951970F016E040E032201C0ABF405
:10C0900003C0ACF4036AA951970FE96E040E0320A4
:10C0A000EA6EEFCFADF4ADC4AFF400016FDEACC407
:10C0B000EAFFABC4E9FF01C0EFFF010E0401A925AF
:10C0C000036A970F016E040E032201C0ABF403C094
:10C0D000ACF4010EA925036A970FE96E040E032044
:10C0E000EA6EEFCFADF4ADC4AFF400014FDEACC4E7
:10C0F000EAFFABC4E9FF01C0EFFF96C403F00401FF
:10C10000036AA951970FE96E040E0320EA6EEFCF80
:10C11000ADF496C4EAFF95C4E9FFADC4EFFF95C442
:10C12000E9FF96C4EAFFEF38006EF00E001600C07B
:10C13000EFFF96C403F096C4EAFF95C4E9FFEFCF82
:10C14000ADF4010EA925036A970FE96E040E0320D2
:10C15000EA6EEF500F0BAD1196C4EAFF95C4E9FFEC
:10C16000EF6E010E016E0001000C0401926B936BE7
:10C17000946B00017CEC3AF001014D39006E0F0E1A
:10C18000001600500C0816E0080E0401F26FF36B65
:10C19000000133EC4AF0040E0401966F930E956F84
:10C1A000000103DE012C04D094C458F193C457F16C
:10C1B00016D00101080E0401F26FF36B000123ECAD
:10C1C00041F0040E0401966F920E956F0001D8DEC7
:10C1D000012C05D0040192510101586B576F0001E9
:10C1E000000C04017D510608D8A478D00001A8995C
:10C1F000E5EF3FF001C007F47CEC3AF00401073DA5
:10C2000001D05AD0010139A510D00401926B92518E
:10C2100000015DEC0FF00401922B000109EC2CF001
:10C22000160E0401925DF3E10101040EEA6E7E0E2A
:10C23000E96EF2CF92F4F29E000E000178EC0FF05E
:10C240000A000900F550EE6E0009FBE1040192BFFF
:10C25000F28E040E08017A6F7E0E796F0001C3EC36
:10C2600030F0A88904010751300A000103E0010AF7
:10C2700008E00ED0010138B703D038953887448ED6
:10C280000001010138B503D038973885448E06D0B7
:10C29000010138510C0B02E13885448E040E040173
:10C2A000926FFA0E0801A86F0001DDEC28F004017E
:10C2B000922FF7D765D108D0010138510C0B05E05A
:10C2C0000001A88904015CD10101330E0401F26F61
:10C2D000010EF36F000123EC41F00401040EEA6E3D
:10C2E0007E0EE96E0801A16BA36B140EA26F000114
:10C2F00075EC30F0330E0401F26FF36B000123ECA8
:10C3000041F0F5EF46F00152D8A47DD00401F26B64
:10C31000F36B000133EC4AF0070E0501D76FD00E26
:10C32000D66F0001B5EC47F001523CE10401F26B1D
:10C33000F36B000133EC4AF0070E0501D76FD00E06
:10C34000D66F0001B5EC47F001522CE1040EEA6E05
:10C350007E0EE96EF2CF92F4F29E000E90EC0FF09A
:10C360000A000900F550EE6E0009FBE1040192BFDE
:10C37000F28E7D5130098E6F040E08017A6F7E0EA9
:10C38000796F0001C3EC30F0040E0401926FFA0ED5
:10C390000801A86F0001DDEC28F00401922FF7D707
:10C3A000EFD000017DC492F45FEF50F001014D53D6
:10C3B00002E10401E5D00D0E0401F26FF36B000100
:10C3C00033EC4AF04E0E0501D76F200ED66F0001F8
:10C3D000B5EC47F0010138A306D07DC492F400010A
:10C3E00078DC10D00101310E0401F26FF36B000113
:10C3F00033EC4AF04E0E0501D76F200ED66F0001C8
:10C40000B5EC47F070D001014D6BC00E4D13040E1A
:10C41000EA6E7E0EE96EF2CF92F4F29E000E0001FB
:10C42000A8EC0FF00A000900F550EE6E0009FBE1E0
:10C43000040192BFF28E7D5130098E6F040E080107
:10C440007A6F7E0E796F0001C3EC30F0010139A5DF
:10C450000FD00401926B92510001C0EC0FF0040167
:10C46000922B000109EC2CF0100E0401925DF3E117
:10C4700000017CEC3AF00D0E0401F26FF36B000149
:10C4800023EC41F01F0E0501F86F400EF76F00011D
:10C490001AEC40F07CEC3AF01A0E0401EF6FF06BEE
:10C4A00000011BEC50F0030E0501F86FE80EF76F6A
:10C4B00000011AEC40F0010138A306D07DC492F4CB
:10C4C000000107DC10D00101310E0401F26FF36BA3
:10C4D000000123EC41F0170E0501F86F700EF76FA5
:10C4E00000011AEC40F001014D83110E0401EF6FC1
:10C4F000010EF06F00011BEC50F001014D871B0E87
:10C500000401EF6F010EF06F00011BEC50F0010110
:10C510004D85150E0401EF6F010EF06F00011BEC4D
:10C5200050F001014D91100E0401EF6F010EF06FFC
:10C5300000011BEC50F0036A01018A51250F016EC6
:10C54000000E03220150380FE96E010E0320EA6E3F
:10C550004DC1EFFF000109DED89001018A35036A61
:10C560003A0F016E000E03220150380FE96E010EE2
:10C570000320EA6E58C1ECFFED5257C1EFFF0401F2
:10C58000000121EF63F0010EEA6E5D0EE96E080115
:10C59000A16BA36B070EA26F000175EC30F0CFEC1E
:10C5A00037F0010139A50FD004017D6B7D510001E9
:10C5B00028EC0FF004017D2B000109EC2CF0200E7B
:10C5C00004017D5DF3E1010E04017C6F7C510608DE
:10C5D0003BE3010139A522D004017D6B7D510001AF
:10C5E00048EC0FF004017D2B000109EC2CF0050E46
:10C5F00004017D5DF3E17CC47FF81F0E0801806FAC
:10C600000001FDEC37F03A0E09EC2CF0200E09EC9D
:10C610002CF0200E09EC2CF007D00101320E08019D
:10C62000A86F0001DDEC28F07CC499F4B7EC3DF074
:10C630000A0E0801A86F0001DDEC28F07CC47DF42F
:10C64000D0D504017C2BC2D70001000C040EEA6E89
:10C650009B0EE96E0801A16BA36B130EA26F000184
:10C6600075EC30F0040EEA6EAE0EE96E0801A16BB7
:10C67000A36B130EA26F000175EC30F00E015B6B23
:10C6800099C45AFE5D6B120E5C6F0001A2EC34F08F
:10C6900002C003F00150E40F016E010E032201C03D
:10C6A000C1F403C0C2F4040E0801A26F9B0EA16F77
:10C6B00003C0A4F801C0A3F8120EA56F000184EC1A
:10C6C00030F00C0E04019B6F036A03015E515F0F93
:10C6D000E96E030E0320EA6EEF2C03D03E0E040138
:10C6E0009C6F040E0801A26F9B0EA16F0001ECEC81
:10C6F00029F0050E0801A86F0001DDEC28F00E01FD
:10C700005B6B9AC45AFE5D6B120E5C6F0001A2EC6B
:10C7100034F002C003F00150E40F016E010E032259
:10C7200001C0C1F403C0C2F4040E0801A26FAE0E32
:10C73000A16F03C0A4F801C0A3F8120EA56F0001F9
:10C7400084EC30F00A0E0401AE6F036A03015E51FF
:10C750005F0FE96E030E0320EA6EEF50020803E15B
:10C760003E0E0401AF6F040E0801A26FAE0EA16F62
:10C770000001ECEC29F0000C04017C6B7C6B7C511B
:10C78000020821E3036A7C515F0FE96E030E032068
:10C79000EA6EEF6A036A7C51640F016E030E032296
:10C7A00003C07EF4036A7C516E0FE96E030E032012
:10C7B000EA6EEFCF7FF47EC4EAFF01C0E9FF7FC4D9
:10C7C000EFFF7C2BDCD703015E6B0001A893A895DB
:10C7D000A8970401036B03C406F406C405F4036AB6
:10C7E00003015E51640FE96E030E0320EA6EEFCF82
:10C7F0007DF4036A5E51640FE96E030E0320EA6E56
:10C80000010EEF2404017E6F7DC499F49A6F00013C
:10C810001DDF000C036A6451680FE96E000E0320EF
:10C82000EA6EEFCFE7F40401010E000164253F0B2F
:10C83000646F6451615D01E15B8E0401E7C401F046
:10C840000001000C036A6351680FE96E000E0320BB
:10C85000EA6EEFCF7DF40401010E000163253F0B6A
:10C86000636F6351615D01E15B8C04017DC401F084
:10C870000001000C04017C6B5BBE06D00001CADF26
:10C8800001C07CF40401F8D70001666B5BBC04D0E6
:10C89000D9DF01C07CF4FAD7000E9EBA010E000A5F
:10C8A00006E09EAAFED7AECF7CF40001F5D7666BFA
:10C8B0009D8A0A0E0801656F0001C8EC28F0C00EC1
:10C8C000F212A7EF67F00401786B796B7A6B7B6BE0
:10C8D000FA0E0801656F0001C8EC28F0FF0E040194
:10C8E000496F486F4A6F4D6B4C6F4B6F5B90589E12
:10C8F000456A446A476A466A4C6A5B925B945B96F7
:10C900005C6A5D6A5E6A5F6A7B6B7B510C080AE356
:10C91000036A7B51D70FE96E010E0320EA6EEF6ABE
:10C920007B2BF3D7010EEA6E380EE96E0801A16B7E
:10C93000A36B5C0EA26F000175EC30F004017B6B01
:10C940007B510108D8A086D07B51040DF3507D6B3C
:10C950007C6F0C0E7C25E96E040E7D21EA6EFF0EC5
:10C96000EC6EED52EF6E7B51040DF3507D6B7C6FDE
:10C97000020E7C25016E000E7D21036E01500C0F0E
:10C98000E96E040E0320EA6EEF6A7B51040DF3504A
:10C990007D6B7C6F180E7C25E96E040E7D21EA6E9E
:10C9A000FF0EEC6EED52EF6E7B51040DF3507D6B7C
:10C9B0007C6F020E7C25016E000E7D21036E0150FE
:10C9C000180FE96E040E0320EA6EEF6A7B51040D26
:10C9D000F3507D6B7C6F240E7C25E96E040E7D2167
:10C9E000EA6EFF0EEC6EED52EF6E7B51040DF350CC
:10C9F0007D6B7C6F020E7C25016E000E7D21036E27
:10CA00000150240FE96E040E0320EA6EEF6A7B5199
:10CA1000040DF3507D6B7C6F300E7C25E96E040EA7
:10CA20007D21EA6EFF0EEC6EED52EF6E7B51040D30
:10CA3000F3507D6B7C6F020E7C25016E000E7D2114
:10CA4000036E0150300FE96E040E0320EA6EEF6AA8
:10CA50007B2B76D70001666B0D0E676FEA6A680E56
:10CA6000E96E0801A16BA36B400EA26F000175EC8B
:10CA700030F0636B63C064F064C061F05B8E5B8C0C
:10CA8000EA6AA90EE96E0801A16BA36B780EA26F8A
:10CA9000000175EC30F0656B65C062F0A881040E92
:10CAA000EA6E640EE96EF2CF7CF4F29E000EB9ECF1
:10CAB00023F00A000900F550EE6E0009FBE10401C5
:10CAC0007CBFF28E040E08017A6F640E796F00014C
:10CAD000C3EC30F02BEF36F0040E04017C6FFA0E3D
:10CAE0000801656F0001C8EC28F004017C2FF7D71E
:10CAF00094948B940C0EBD6EC150C00B0C09C16E8A
:10CB0000C090C082C084C09EC280B098D190840E74
:10CB1000D56E950ECD6EB50EB16E000E766E000E12
:10CB2000776E9D80F28A070EB46E9750976E0D0E49
:10CB3000006E002EFED7B450A19CB56AF19EFA0E8D
:10CB40000801656F0001C8EC28F08CEC2AF0F19C1C
:10CB5000F288F19AF086F198F088F196F08AA38A2B
:10CB6000C00EF212196AF2BE198EF29E400E0E012C
:10CB7000616F626B000163EC24F019BEF28E02C09B
:10CB80008DF101C08CF18DC10DF48CC10CF48DC1FF
:10CB900011F48CC110F4196AF2BE198EF29E400E87
:10CBA0000E01616F626B000163EC24F019BEF28E1E
:10CBB00002C079F401C078F4196AF2BE198EF29EAF
:10CBC000440E0E01616F626B000163EC24F019BE2C
:10CBD000F28E02C079F401C078F4196AF2BE198E9F
:10CBE000F29E420E0E01616F626B000163EC24F055
:10CBF00019BEF28E02C079F401C078F4196AF2BE4F
:10CC0000198EF29E460E0E01616F626B000163EC9D
:10CC100024F019BEF28E02C079F401C078F4040E3B
:10CC2000EA6E640EE96EF2CF7CF4F29E000E47ECE1
:10CC300023F00A000900F550EE6E0009FBE1040143
:10CC40007CBFF28E040E08017A6F640E796F0001CA
:10CC5000C3EC30F098DC010139A912D0196AF2BE98
:10CC6000198EF29E880E0E016A6F0A0E6B6F020E0D
:10CC70006C6F0001F0EC25F019BEF28E11D00101AD
:10CC8000196AF2BE198EF29E880E0E016A6F0A0EA4
:10CC90006B6F030E6C6F0001F0EC25F019BEF28E85
:10CCA000640E0801656F0001C8EC28F0010139AB82
:10CCB00012D0196AF2BE198EF29E880E0E016A6FAA
:10CCC0000A0E6B6F050E6C6F0001F0EC25F019BEBB
:10CCD000F28E11D00101196AF2BE198EF29E880EF1
:10CCE0000E016A6F0A0E6B6F060E6C6F0001F0EC9E
:10CCF00025F019BEF28E0A0E0801656F0001C8EC1E
:10CD000028F0010139A312D0196AF2BE198EF29EE1
:10CD1000880E0E016A6F0A0E6B6F080E6C6F0001B1
:10CD2000F0EC25F019BEF28E11D00101196AF2BEA5
:10CD3000198EF29E880E0E016A6F0A0E6B6F070E37
:10CD40006C6F0001F0EC25F019BEF28E196AF2BE8C
:10CD5000198EF29E880E0E016A6F0A0E6B6F010E1D
:10CD60006C6F0001F0EC25F019BEF28E640E080124
:10CD7000656F0001C8EC28F001013AAB02D09D8A32
:10CD800001D09D9A0001F8DC640E0801656F000176
:10CD9000C8EC28F0196AF2BE198EF29E880E0E01B8
:10CDA0006A6F0B0E6B6F47C16CFE0001F0EC25F053
:10CDB00019BEF28E640E0801656F0001C8EC28F000
:10CDC000196AF2BE198EF29E880E0E016A6F060E67
:10CDD0006B6F46C16CFE0001F0EC25F019BEF28EBF
:10CDE000640E0801656F0001C8EC28F0196AF2BEF4
:10CDF000198EF29E880E0E01676F060E686F000195
:10CE00001DEC24F019BEF28E01C07AF40A0E08015E
:10CE1000656F0001C8EC28F0196AF2BE198EF29E07
:10CE2000880E0E016A6F030E6B6F45C16CFE000128
:10CE3000F0EC25F019BEF28E640E0801656F00015A
:10CE4000C8EC28F0196AF2BE198EF29E880E0E0107
:10CE5000676F030E686F00011DEC24F019BEF28E9F
:10CE600001C07AF40A0E0801656F0001C8EC28F0D1
:10CE7000010139A105D0FA0E04014A1704D00101BD
:10CE8000FC0E04014A174A9F196AF2BE198EF29EDF
:10CE9000480E0E016A6F010E6B6F4AC46CFE0001F2
:10CEA000F0EC25F019BEF28E196AF2BE198EF29ED0
:10CEB000880E0E016A6F6B6B800E6C6F0001F0ECD8
:10CEC00025F019BEF28E640E0801656F0001C8ECF2
:10CED00028F0196AF2BE198EF29E880E0E01676F55
:10CEE000686B00011DEC24F019BEF28E01C07AF4CB
:10CEF0000A0E0801656F0001C8EC28F0448A3BC1A6
:10CF00008EF1498A498401018A6B8B6B036A3B511C
:10CF1000250F016E000E03220150380FE96E010E3D
:10CF20000320EA6EEF50F00B06E03BC190F14A801F
:10CF30003CC191F14A82050E0801656F0001C8EC01
:10CF400028F001013ABB01D09D9A000193D474EFFF
:10CF5000F0F001018B530CE008016B517F0B06E1EF
:10CF600069517F0B03E16A517F0B01E0468C01019F
:10CF70004D39006E0F0E00160050FF0FF40F19E22E
:10CF80000C0F0001DBEF67F069C86CF86AC86DF838
:10CF90006BC86EF886EC3AF001010BD069C86CF8EA
:10CFA0006AC86DF86BC86EF8C2EC3BF0010101D0A5
:10CFB00001010001000CF2CF0EF0F29EE824F76AA6
:10CFC000F736E10FF66ECF0EF722000EF86EFB6E0D
:10CFD0000A00F550FA6E0800F5500EBEF28EF96E9A
:10CFE00088CF88CF88CF88CF88CF88CF88CF88CF89
:10CFF00088CF88CF88CF9CCF0401646B656B666B4C
:10D00000140E676F180E686F070E696F6A6B050E56
:10D010006B6F060E6C6F120E6D6F01014D39006E55
:10D020000F0E00160050020A000119E0070A20E066
:10D03000010A27E00E0A2EE0020A2CE0010A2AE08B
:10D040000E0A28E00C0A26E0070A2DE0020A34E066
:10D050000F0A3BE0070A39E0050A41E04AD0120E08
:10D060000401686F0D0E676F070E696F6A6B43D01E
:10D070000C0E0401686F0A0E676F070E696F6A6B0A
:10D080003AD0100E0401686F0C0E676F070E696FBF
:10D090006A6B31D0180E0401686F140E676F070EAB
:10D0A000696F6A6B28D0180E0401686F080E676FED
:10D0B000070E696F6A6B1FD0140E0401686F0C0EA7
:10D0C000676F070E696F6A6B16D0180E0401686FE0
:10D0D000140E676F070E696F020E6A6F0CD0100E88
:10D0E0000401686F0A0E676F070E696F6A6B03D0E1
:10D0F0000001C8D1040168510101485D02E248C144
:10D1000068F4040167510101495D02E249C167F415
:10D11000196AF2BE198EF29E7F0E0E01616F68C40D
:10D1200062FE0001CAEC24F019BEF28E01C06BF45D
:10D13000196AF2BE198EF29E7F0E0E01616F67C4EE
:10D1400062FE0001CAEC24F019BEF28E01C06CF43C
:10D15000196AF2BE198EF29E7F0E0E01616F69C4CC
:10D1600062FE0001CAEC24F019BEF28E01C06DF41B
:10D1700001014D39006E0F0E001600500A08D8B498
:10D18000F2D0D8904A31FF0A800F37533AE1365D2A
:10D1900038E2800ED880365504016E6FD8900101B8
:10D1A0004A3104016E5D6F6F196AF2BE198EF29EEC
:10D1B000E8CF61FE6BC462FE0001CAEC24F019BE28
:10D1C000F28E01C065F404016551685D03E268C434
:10D1D00065F404D0655302E1010E656F3FC100F0B4
:10D1E00001018A51016E04E0D8900032012EFCD773
:10D1F00000A003D00401659F02D00401658F3ED0DA
:10D200000101D8904A317F0F375303E1365D37E093
:10D2100036E3800E365D04016E6FD89001014A310D
:10D2200004016E5D6F6F196AF2BE198EF29EE8CF2F
:10D2300061FE6BC462FE0001CAEC24F019BEF28EDE
:10D2400001C065F404016551685D03E268C465F4DA
:10D2500004D0655302E1010E656F3FC100F001018A
:10D260008A51016E04E0D8900032012EFCD700A054
:10D2700003D00401658F02D00401659F01017F0E78
:10D28000D8804A55355336E1345D34E2800ED8807B
:10D290003455D8804A5504016F6F196AF2BE198E51
:10D2A000F29EE8CF61FE6CC462FE0001CAEC24F07D
:10D2B00019BEF28E01C064F404016451675D03E29B
:10D2C00067C464F404D0645302E1010E646F40C18A
:10D2D00000F001018A51016E04E0D8900032012E65
:10D2E000FCD700A003D00401648F02D00401649F26
:10D2F00039D001017F0E4A25355303E1345D33E017
:10D3000032E3800E345DD8804A5504016F6F196A8C
:10D31000F2BE198EF29EE8CF61FE6CC462FE00017F
:10D32000CAEC24F019BEF28E01C064F40401645109
:10D33000675D03E267C464F404D0645302E1010E44
:10D34000646F40C100F001018A51016E04E0D89081
:10D350000032012EFCD700A003D00401649F02D04C
:10D360000401648F0101D8904A31FF0A800F3353C2
:10D3700033E1325D31E2800ED880325504016E6FA8
:10D38000D89001014A3104016E5D6F6F196AF2BED7
:10D39000198EF29EE8CF61FE6DC462FE0001CAECF8
:10D3A00024F019BEF28E01C066F404016651695D75
:10D3B00003E269C466F405D066516A5D02E36AC49B
:10D3C00066F4668701013AA503D00401668F02D096
:10D3D0000401669F37D00101D8904A317F0F335343
:10D3E00003E1325D30E02FE3800E325D04016E6FA9
:10D3F000D89001014A3104016E5D6F6F196AF2BE67
:10D40000198EF29EE8CF61FE6DC462FE0001CAEC87
:10D4100024F019BEF28E01C066F404016651695D04
:10D4200003E269C466F405D066516A5D02E36AC42A
:10D4300066F4668701013AA503D00401669F02D015
:10D440000401668F010122510401665D0DE10101B5
:10D4500023510401655D08E1010124510401645D6B
:10D4600003E100010FD0040166C422F165C423F179
:10D4700064C424F165C469F864C46AF866C46BF8CE
:10D48000000167DD7BEFF0F00401666B6791679345
:10D49000196AF2BE198EF29E460E0E01616F626B22
:10D4A000000163EC24F019BEF28E02C065F401C0E5
:10D4B00064F4FF0E0401641B651B65C435F464C489
:10D4C00034F44AA107D064518008D8A4C4D065536D
:10D4D000D8A4C1D064C400F06551036E05E10052C8
:10D4E0000001D8B479D00401035006E1010E005CBC
:10D4F0000001D8B474D00401200E035C05E1005291
:10D500000001D8B475D00401035006E1020E005C9E
:10D510000001D8B476D00401020E035C05E100528C
:10D520000001D8B46ED00401040E035C05E1005282
:10D530000001D8B466D00401080E035C05E1005276
:10D540000001D8B45ED00401400E035C05E1005236
:10D550000001D8B456D00401800E035C04E10052EF
:10D5600000014FE00401035005E1400E005C0001A2
:10D5700050E00401035005E1200E005C00014FE083
:10D580000401035005E1800E005C000150E004013D
:10D59000035005E1040E005C000149E00401035062
:10D5A00005E1080E005C000142E00401035005E1C2
:10D5B000100E005C00013BE00401010E035C04E17D
:10D5C0000052000134E00401100E035C04E100523B
:10D5D00000012DE004012DD05B945B963BD004014B
:10D5E0004AB303D067815B8401D06783000132D0E6
:10D5F00004014AB303D067815B8601D067830001D1
:10D6000029D004014AB302D0678101D067830001A9
:10D6100021D0606B5B980401678100011BD0010180
:10D620008F6B906B916B04016781000113D0040133
:10D63000678158B406D045BA04D058BE02D05BA06A
:10D6400007D05B90589E459A58A402D044805886D3
:10D65000000100D0040167A105D066C436F4368FFE
:10D660005B9A04D031C435F430C434F40001D9EFEE
:10D670009EF00401836B825100082EE2825106085D
:10D680002BE3196AF2BE198EF29E880E0E01676FA7
:10D69000686B00011DEC24F019BEF28E01C083F40A
:10D6A0000A0E0801656F0001C8EC28F0196AF2BE85
:10D6B000198EF29E880E0E016A6F6B6B82C46CFE2F
:10D6C0000001F0EC25F019BEF28E640E0801656FC2
:10D6D0000001C8EC28F004010001000C0401816B7A
:10D6E000196AF2BE198EF29E880E0E01676F686B82
:10D6F00000011DEC24F019BEF28E01C081F40A0E67
:10D700000801656F0001C8EC28F00401805306E1B0
:10D7100089C182F40001ADDF11D00401818F196A43
:10D72000F2BE198EF29E880E0E016A6F6B6B81C479
:10D730006CFE0001F0EC25F019BEF28E000C040125
:10D74000986B010E986F985106081BE398C499F4E2
:10D750000001B7EC3DF00401972D09D00E0EEF6FDC
:10D76000010EF06F00011BEC50F008D004010D0E0B
:10D77000EF6F010EF06F00011BEC50F00401982BCD
:10D78000E2D70001FDEF6CF00401976B976B9751A6
:10D79000020821E3036A97515F0FE96E030E03202D
:10D7A000EA6EEF6A036A9751640F016E030E03225B
:10D7B00003C099F4036A97516E0FE96E030E0320BC
:10D7C000EA6EEFCF9AF499C4EAFF01C0E9FF9AC468
:10D7D000EFFF972BDCD7986B000164EC2CF0030172
:10D7E0005E6B0001A893A895A8970401036B03C47E
:10D7F00006F406C405F4036A03015E51640FE96E82
:10D80000030E0320EA6EEFCF98F498C499F4140E37
:10D8100004019A6F000126EC63F0FEEF6CF0040146
:10D82000816B826B802D21D04AA11ED0040EEA6E3E
:10D83000830EE96EF2CF97F4F29E000E0001D1EC58
:10D8400023F00A000900F550EE6E0009FBE1040127
:10D8500097BFF28E040E08017A6F830E796F000174
:10D86000C3EC30F0FF000401CAD08053D8A4C7D065
:10D870004AB1C5D003015E6B040EEA6E830EE96EF9
:10D88000200E0801A16FA36B140EA26F000175ECAE
:10D8900030F0036A03015E515F0FE96E030E03204F
:10D8A000EA6E010EEF6E040EEA6E830EE96EF2CFA1
:10D8B00097F4F29E000E000180EC22F00A000900AD
:10D8C000F550EE6E0009FBE1040197BFF28E040EE5
:10D8D0000801A26F830EA16F0001ECEC29F0040E89
:10D8E000EA6E830EE96EF2CF97F4F29E000EE9EC39
:10D8F00023F00A000900F550EE6E0009FBE1040177
:10D9000097BFF28E040E0801A26F830EA16F000173
:10D91000ECEC29F00401826B800E816F196AF2BE73
:10D92000198EF29E880E0E016A6F6B6B81C46CFEBD
:10D930000001F0EC25F019BEF28E640E0801656F4F
:10D940000001C8EC28F00401826B800E816F196A17
:10D95000F2BE198EF29E880E0E016A6F010E6B6F79
:10D9600081C46CFE0001F0EC25F019BEF28E640E4D
:10D970000801656F0001C8EC28F0FF0E0401496F33
:10D98000486F4A6F4C6F4B6F196AF2BE198EF29E48
:10D99000480E0E016A6F010E6B6F4AC46CFE0001E7
:10D9A000F0EC25F019BEF28E196AF2BE198EF29EC5
:10D9B0004C0E0E01636F646B49C466FE48C465FE7D
:10D9C00000011CEC26F019BEF28E196AF2BE198E07
:10D9D000F29E4A0E0E01636F646B4CC466FE4BC42C
:10D9E00065FE00011CEC26F019BEF28EBE6A9D9009
:10D9F000010E0401976F0001A2D6C6D604010001F2
:10DA0000000C030E0301645DF00FD8B0EAD0100FD4
:10DA10000001F4EF6DF0040103530CE1448C6EC37C
:10DA200064F3036A03015E515F0FE96E030E032086
:10DA3000EA6EEF6A0301D5D0040103531BE1196AB2
:10DA4000F2BE198EF29E880E0E016A6F0A0E6B6F7F
:10DA5000010E6C6F0001F0EC25F019BEF28E6EC362
:10DA600064F3036A03015E515F0FE96E030E032046
:10DA7000EA6EEF6A0301B5D00401035101013B5D79
:10DA800003E003C43BF1448E0301ABD00401035116
:10DA900001013C5D03E003C43CF1448E0301A1D0CD
:10DAA000040103510101435D03E003C443F1448ECB
:10DAB000030197D00401035101013E5D03E003C45B
:10DAC0003EF1448E03018DD00401035305E10101B1
:10DAD0003A97448E06D00401032D03D001013A8702
:10DAE000448E03017ED00401035101013D5D03E03A
:10DAF00003C43DF1448E030174D00401035305E1D6
:10DB000001013A93448E06D00401032D03D0010194
:10DB10003A83448E030165D0040103510101445D41
:10DB200004E003C444F1448E07D04451030DF3CF05
:10DB300080F4040180C4BEFF030153D004010353E9
:10DB400005E101013A95448E06D00401032D03D06E
:10DB500001013A85448E030144D00401032D05D010
:10DB600001013A81448E06D00401035303E101010F
:10DB70003A91448E030135D00401035306E10101BB
:10DB80003A99448A448E07D00401032D04D0010140
:10DB90003A89448A448E030124D0040103510101CF
:10DBA000485D03E003C448F1448E03011AD0040128
:10DBB00003510101495D03E003C449F1448E0301AF
:10DBC00010D00401035305E101013A8F448E06D0C1
:10DBD0000401032D03D001013A9F448E030101D0BB
:10DBE0000301030110EF71F0F2CF0EF0F29EE82472
:10DBF000F76AF736130FF66EDC0EF722000EF86E9A
:10DC0000FB6E0A00F550FA6E0800F5500EBEF28E5B
:10DC1000F96E38DA16DA78DA8CDA9ADBAEDBA0DA6B
:10DC2000B4DAC8DAE6DAFADA3CDB5ADB78DBC2DBF4
:10DC300018DB036A03015E515F0FE96E030E0320D8
:10DC4000EA6EEF5002081EE1036A5E51640FE96E4E
:10DC5000030E0320EA6E010EEF5C0401966F036A67
:10DC600003015E51640FE96E030E0320EA6EEFCFED
:10DC700097F496C499F497C49AF4000126EC63F0E3
:10DC80001BD00301036A5E51640FE96E030E03208B
:10DC9000EA6EEFCF96F4036A5E51640FE96E030EED
:10DCA0000320EA6E010EEF240401976F96C499F4E5
:10DCB0009A6F000126EC63F0000C0401806B816B0D
:10DCC000010E0301655DF60FD8B047D10A0F0001C0
:10DCD000B0EF6FF00401035305E101013A8B458E6B
:10DCE00006D00401032D04D001013A9B458E0401A6
:10DCF000448E030132D10401035304E101013A8D42
:10DD000005D00401032D03D001013A9D0401448E86
:10DD1000030123D10401035301E1458203011DD115
:10DD2000040103532AE1040EEA6E820EE96E080133
:10DD3000A16BA36B140EA26F000175EC30F0040E02
:10DD4000EA6E820EE96EF2CF96F4F29E000EC7ECF8
:10DD50000DF00A000900F550EE6E0009FBE1040128
:10DD600096BFF28E040E08017A6F820E796F000161
:10DD7000C3EC30F03BEC32F05CDF0301EED0040189
:10DD8000032D03D00101398702D001013997448E58
:10DD90000301E3D00401032D14D001013989196A6C
:10DDA000F2BE198EF29E880E0E016A6F0A0E6B6F1C
:10DDB000020E6C6F0001F0EC25F019BEF28E13D04C
:10DDC000040101013999196AF2BE198EF29E880E7A
:10DDD0000E016A6F0A0E6B6F030E6C6F0001F0ECA0
:10DDE00025F019BEF28E448E0301B7D00401032D35
:10DDF00041D001013983196AF2BE198EF29E880E54
:10DE00000E016A6F0A0E6B6F080E6C6F0001F0EC6A
:10DE100025F019BEF28E410E0401816F500E806F05
:10DE2000196AF2BE198EF29EA00E0E01636F646B2A
:10DE300081C466FE80C465FE00011CEC26F019BE9C
:10DE4000F28E200E0401816F4C0E806F196AF2BEB3
:10DE5000198EF29EA00E0E01636F020E646F81C4D4
:10DE600066FE80C465FE00011CEC26F019BEF28E31
:10DE700040D0040101013993196AF2BE198EF29E55
:10DE8000880E0E016A6F0A0E6B6F070E6C6F000131
:10DE9000F0EC25F019BEF28E540E0401816F4E0E87
:10DEA000806F196AF2BE198EF29EA00E0E01636F8A
:10DEB000646B81C466FE80C465FE00011CEC26F024
:10DEC00019BEF28E430E0401816F530E806F196AE2
:10DED000F2BE198EF29EA00E0E01636F020E646FE9
:10DEE00081C466FE80C465FE00011CEC26F019BEEC
:10DEF000F28E448E0401032D03D00101388302D039
:10DF000001013893448E030128D00401032D03D06E
:10DF10000101388902D001013899448E03011DD0D6
:10DF20000401032D07D00101388538970001A88925
:10DF300010D004010351020807E101013895388728
:10DF40000001A88906D00401010138953897000125
:10DF5000A899448E030101D00301030110EF71F071
:10DF6000F2CF0EF0F29EE824F76AF7368B0FF66ECA
:10DF7000DF0EF722000EF86EFB6E0A00F550FA6E07
:10DF80000800F5500EBEF28EF96ED4DCF6DC14DD1E
:10DF900020DD7EDD94DDECDDF4DE0ADF20DF030131
:10DFA0006651010A000105E0030A24E0010A43E08A
:10DFB00063D004010451035D1BE003C445F103C4B5
:10DFC00004F4448E196AF2BE198EF29E880E0E0178
:10DFD0006A6F030E6B6F04C46CFE0001F0EC25F059
:10DFE00019BEF28E640E0801A86F0001DDEC28F066
:10DFF000000142D004010451035D1BE003C446F15B
:10E0000003C404F4448E196AF2BE198EF29E880E7F
:10E010000E016A6F060E6B6F04C46CFE0001F0EC1B
:10E0200025F019BEF28E640E0801A86F0001DDEC28
:10E0300028F0000121D004010451035D1BE003C45A
:10E0400047F103C404F4448E196AF2BE198EF29E9D
:10E05000880E0E016A6F0B0E6B6F04C46CFE00011C
:10E06000F0EC25F019BEF28E640E0801A86F0001D5
:10E07000DDEC28F0000100D00DEF71F00401806BA1
:10E08000036A03015E51640FE96E030E0320EA6E1A
:10E09000010EEF5CF90FD8B079D0070F0001C9EF7E
:10E0A00070F00401802B00010401802B00010401A9
:10E0B000802B00010401802B00010401802B000152
:10E0C0000401802B0001040103532FE103015E5181
:10E0D000030815E10401805304E101013F6B0ED0F8
:10E0E0000401010E006E8051016E04E0D8900036EC
:10E0F000012EFCD70050FF0A01013F1714D0040184
:10E10000805304E10101406B0ED00401010E006E4A
:10E110008051016E04E0D8900036012EFCD70050EB
:10E12000FF0A010140172ED0040103015E510308CC
:10E1300015E10401805305E1FF0E01013F6F0DD091
:10E140000401010E006E8051016E04E0D89000368B
:10E15000012EFCD7005001013F1314D0040180535D
:10E1600005E1FF0E0101406F0DD00401010E006EAC
:10E170008051016E04E0D8900036012EFCD700508B
:10E1800001014013448E030101D00301030110EF8C
:10E1900071F0F2CF0EF0F29EE824F76AF736BD0F69
:10E1A000F66EE10EF722000EF86EFB6E0A00F550D7
:10E1B000FA6E0800F5500EBEF28EF96EC6E0C0E0B1
:10E1C000BAE0B4E0AEE0A8E0A2E0A893A895A897D2
:10E1D0000401036B03C406F406C405F4FF0E036FC9
:10E1E00003015E530BE16451120808E1010144513F
:10E1F000030DF3CF81F4040181C4BEFF000119DDDA
:10E20000000C03015E51FB0F0BE2050F000114EF40
:10E2100071F001EF6DF051D5C2D6030101D02ED7B8
:10E220000001D3DF22EF79F0F2CF0EF0F29EE82466
:10E23000F76AF736530FF66EE20EF722000EF86E0D
:10E24000FB6E0A00F550FA6E0800F5500EBEF28E15
:10E25000F96E12E216E218E21EE21EE2A8B33CD00A
:10E2600003015E5324E1036A5E515F0FE96E030E02
:10E270000320EA6EEF6A036A5E51640F016E030EBB
:10E280000322040103C081F4036A03015E516E0F8F
:10E29000E96E030E0320EA6EEFCF82F4040181C41D
:10E2A000EAFF01C0E9FF82C4EFFF13D00301036A54
:10E2B0005E515F0FE96E030E0320EA6E020EEF6EF1
:10E2C000036A5E51640FE96E030E0320EA6E010ECD
:10E2D000EF6E0001AEDC01D078DF000C0301645169
:10E2E000020A000131E0110A4BE0170A65E0070A53
:10E2F00063E0120AD8B479D01A0AD8B4AAD0060AB0
:10E30000D8B4C3D0030AD8B4DCD01E0AD8B40DD117
:10E31000170AD8B43ED10F0AD8B43BD10D0AD8B4ED
:10E320004DD1030AD8B454D10F0AD8B45BD1030A33
:10E33000D8B461D1060AD8B468D11E0AD8B46FD156
:10E340001D0AD8B475D1A8D1020E0401986F00013E
:10E3500064EC2CF0036A03015E51640FE96E030E56
:10E360000320EA6E010EEF6E036A5E515F0FE96EE5
:10E37000030E0320EA6E020EEF6E00016FDF90D1F4
:10E38000010E0401986F000164EC2CF0036A030194
:10E390005E51640FE96E030E0320EA6E010EEF6E0C
:10E3A000036A5E515F0FE96E030E0320EA6E020EF0
:10E3B000EF6E000153DF74D1030EEA6E730EE96E47
:10E3C000F2CF80F4F29E000ED8EC0BF00A000900A8
:10E3D000F550EE6E0009FBE1040180BFF28E056B83
:10E3E000036B03C406F400015BD1030EEA6E730EE7
:10E3F000E96EF2CF80F4F29E000EEDEC0BF00A0015
:10E400000900F550EE6E0009FBE1040180BFF28EB9
:10E41000030EEA6E850EE96EF2CF80F4F29E000ED6
:10E42000000102EC0CF00A000900F550EE6E000944
:10E43000FBE1040180BFF28E036B01013ABF03D000
:10E440000401032B0101010E0401056F066B00019D
:10E4500027D1030E0401986F000164EC2CF0036ACD
:10E4600003015E51640FE96E030E0320EA6E010E94
:10E47000EF6E036A5E515F0FE96E030E0320EA6ED2
:10E48000020EEF6E0001EADE0BD1040E0401986F5C
:10E49000000164EC2CF0036A03015E51640FE96E25
:10E4A000030E0320EA6E010EEF6E036A5E515F0FEA
:10E4B000E96E030E0320EA6E020EEF6E0001CEDE5F
:10E4C000EFD0030EEA6E730EE96EF2CF80F4F29E87
:10E4D000000E17EC0CF00A000900F550EE6E000972
:10E4E000FBE1040180BFF28E030EEA6E850EE96E39
:10E4F000F2CF80F4F29E000E00012DEC0CF00A0029
:10E500000900F550EE6E0009FBE1040180BFF28EB8
:10E51000036B01013AA503D00401032B0101010E95
:10E520000401056F066B0001BBD0030EEA6E730E8B
:10E53000E96EF2CF80F4F29E000E43EC0CF00A007C
:10E540000900F550EE6E0009FBE1040180BFF28E78
:10E55000030EEA6E850EE96EF2CF80F4F29E000E95
:10E56000000159EC0CF00A000900F550EE6E0009AC
:10E57000FBE1040180BFF28E010E056F036B010108
:10E580003AA903D00401032B01010401066B000129
:10E5900087D0A885180E0401056F010E066F0301D0
:10E5A0006451070A000103E00F0A04E006D048C1E5
:10E5B00003F403D049C103F400D072D0A885060E3D
:10E5C0000401056F3BC103F4010E066F000168D022
:10E5D000A8850C0E0401056F3CC103F4010E066F03
:10E5E00000015ED0A8853C0E0401056F43C103F411
:10E5F000066B000155D0A885180E0401056F010EA9
:10E60000066F3EC103F400014BD0A885140E04012F
:10E61000056F010E066F3DC103F4000141D0A885CE
:10E62000320E0401056F066B44C103F4000138D0BB
:10E63000030EEA6E730EE96EF2CF80F4F29E000EC6
:10E640006FEC0CF00A000900F550EE6E0009FBE1DA
:10E65000040180BFF28E030EEA6E850EE96EF2CFE2
:10E6600080F4F29E000E000186EC0CF00A00090016
:10E67000F550EE6E0009FBE1040180BFF28E010E41
:10E68000056F036B01013AA103D00401032B0101C3
:10E690000401066B000104D0A893A895A89700D0A8
:10E6A00039EF79F003016551030A00011CE0070A04
:10E6B0001AE0010A30E0030A61E0010AD8B491D0FF
:10E6C000060AD8B4C1D0030AD8B4BED00A0AD8B456
:10E6D0000CD1010AD8B43CD1030AD8B46CD1010AD8
:10E6E000D8B4B8D1BED1030EEA6E730EE96EF2CF84
:10E6F00080F4F29E000ED8EC0BF00A000900F550F1
:10E70000EE6E0009FBE1040180BFF28E056B036B26
:10E7100003C406F4ABD1030EEA6E730EE96EF2CFBA
:10E7200080F4F29E000E9DEC0CF00A000900F550FA
:10E73000EE6E0009FBE1040180BFF28E030EEA6E6B
:10E74000850EE96EF2CF80F4F29E000E0001B2EC6D
:10E750000CF00A000900F550EE6E0009FBE104011F
:10E7600080BFF28E010E056F066B036B010139A7A6
:10E7700003D00401032B0101040178D1030EEA6EDA
:10E78000730EE96EF2CF80F4F29E000EC7EC0CF02F
:10E790000A000900F550EE6E0009FBE1040180BF9C
:10E7A000F28E030EEA6E850EE96EF2CF80F4F29ED1
:10E7B000000E0001DEEC0CF00A000900F550EE6ED0
:10E7C0000009FBE1040180BFF28E010E056F066BAC
:10E7D000036B010139A903D00401032B01010401DA
:10E7E00045D1030EEA6E730EE96EF2CF80F4F29E0D
:10E7F000000EF5EC0CF00A000900F550EE6E000971
:10E80000FBE1040180BFF28E030EEA6E850EE96E15
:10E81000F2CF80F4F29E000E00010AEC0DF00A0027
:10E820000900F550EE6E0009FBE1040180BFF28E95
:10E83000010E056F066B036B010139A303D00401C0
:10E84000032B0101040112D1030EEA6E730EE96E6F
:10E85000F2CF80F4F29E000EEDEC0BF00A000900FE
:10E86000F550EE6E0009FBE1040180BFF28E030E4D
:10E87000EA6E850EE96EF2CF80F4F29E000E000182
:10E8800002EC0CF00A000900F550EE6E0009FBE105
:10E89000040180BFF28E036A03015E51640FE96ECA
:10E8A000030E0320EA6EEF50010A000103E0030AA1
:10E8B0000AE012D00401036B01013ABB03D004014A
:10E8C000032B01010DD00401036B01013ABD03D0FC
:10E8D0000401032B010104D00401036B010100D0EA
:10E8E000010E0401056F066BC1D0030EEA6E730EB4
:10E8F000E96EF2CF80F4F29E000E1FEC0DF00A00DC
:10E900000900F550EE6E0009FBE1040180BFF28EB4
:10E91000030EEA6E850EE96EF2CF80F4F29E000ED1
:10E92000000137EC0DF00A000900F550EE6E000909
:10E93000FBE1040180BFF28E010E056F066B036BD5
:10E94000010138A303D00401032B010104018ED07F
:10E95000030EEA6E730EE96EF2CF80F4F29E000EA3
:10E960004FEC0DF00A000900F550EE6E0009FBE1D6
:10E97000040180BFF28E030EEA6E850EE96EF2CFBF
:10E9800080F4F29E000E000167EC0DF00A00090011
:10E99000F550EE6E0009FBE1040180BFF28E010E1E
:10E9A000056F066B036B010138A903D00401032B2B
:10E9B000010104015BD0030EEA6E730EE96EF2CF23
:10E9C00080F4F29E000E7FEC0DF00A000900F55075
:10E9D000EE6E0009FBE1040180BFF28E030EEA6EC9
:10E9E000850EE96EF2CF80F4F29E000E000197ECE6
:10E9F0000DF00A000900F550EE6E0009FBE104017C
:10EA000080BFF28E030EEA6E970EE96EF2CF80F4AD
:10EA1000F29E000E0001AFEC0DF00A000900F55067
:10EA2000EE6E0009FBE1040180BFF28E020E056F5D
:10EA3000066B010138A505D0010E0401036F09D052
:10EA4000010138A704D0020E0401036F02D00401B3
:10EA5000036B0CD00401986B000164EC2CF0E5EC26
:10EA600070F0A893A895A897040100D0000139EF91
:10EA700079F003016651010A00010AE0030AD8B4E3
:10EA8000B8D0010AD8B4CCD0070AD8B4E0D0E6D0C8
:10EA9000030EEA6E730EE96EF2CF80F4F29E000E62
:10EAA000DFEC0DF00A000900F550EE6E0009FBE105
:10EAB000040180BFF28E030EEA6E850EE96EF2CF7E
:10EAC00080F4F29E000E0001F7EC0DF00A00090040
:10EAD000F550EE6E0009FBE1040180BFF28E030EDB
:10EAE000EA6E970EE96EF2CF80F4F29E000E0001FE
:10EAF0000FEC0EF00A000900F550EE6E0009FBE184
:10EB0000040180BFF28E030EEA6EA90EE96EF2CF09
:10EB100080F4F29E000E000127EC0EF00A000900BE
:10EB2000F550EE6E0009FBE1040180BFF28E030E8A
:10EB3000EA6EBB0EE96EF2CF80F4F29E000E000189
:10EB40003FEC0EF00A000900F550EE6E0009FBE103
:10EB5000040180BFF28E030EEA6ECD0EE96EF2CF95
:10EB600080F4F29E000E000157EC0EF00A0009003E
:10EB7000F550EE6E0009FBE1040180BFF28E030E3A
:10EB8000EA6EDF0EE96EF2CF80F4F29E000E000115
:10EB90006FEC0EF00A000900F550EE6E0009FBE183
:10EBA000040180BFF28E030EEA6EF10EE96EF2CF21
:10EBB00080F4F29E000E000187EC0EF00A000900BE
:10EBC000F550EE6E0009FBE1040180BFF28E070EE6
:10EBD000056F066B45C104F404C403F40651035DDC
:10EBE00003E30351055D02E206C404F404C403F424
:10EBF0003AD0A8850401066B280E056F46C104F4BF
:10EC000004C403F40651035D03E30351055D02E20E
:10EC100006C404F404C403F40001A887040123D04B
:10EC2000A8850401066B280E056F47C104F404C4CF
:10EC300003F40651035D03E30351055D02E206C4DC
:10EC400004F404C403F40001A88704010CD00401F7
:10EC5000986B000164EC2CF0E5EC70F0A893A8959B
:10EC6000A897040100D0000139EF79F00401806B0E
:10EC7000030EEA6E730EE96EF2CF81F4F29E000E7F
:10EC8000000117EC0CF00A000900F550EE6E0009C7
:10EC9000FBE1040181BFF28E030EEA6E850EE96E80
:10ECA000F2CF81F4F29E000E00012DEC0CF00A0070
:10ECB0000900F550EE6E0009FBE1040181BFF28E00
:10ECC000010E056F066B036A03015E51640FE96E66
:10ECD000030E0320EA6EEF50070A00010FE0010A5D
:10ECE00010E0030A11E0010A12E0070A13E0010A2A
:10ECF00014E0030A15E0090A3DE043D00401802B2B
:10ED000000010401802B00010401802B000104019B
:10ED1000802B00010401802B00010401802B0001E5
:10ED20000401805301E1802B03015E5103080FE1D0
:10ED30003FC100F004018051016E04E0D890003220
:10ED4000012EFCD7036B00B0032B11D003015E51E1
:10ED500004080DE140C100F004018051016E04E09F
:10ED6000D8900032012EFCD7036B00B0032B0001BA
:10ED7000A8830BD00401986B000164EC2CF0E5EC47
:10ED800070F0A893A895A89700D039EF79F0040106
:10ED9000AA51F00B006E003A0F0E00160050000151
:10EDA0000FE0010A41E0030AD8B48DD0010AD8B4BB
:10EDB000BFD0070AD8B407D1010AD8B435D165D17C
:10EDC0000401AA510F0B090815E3010EAB5D036A9C
:10EDD000AC25E96EAD510320EA6E300EEF6E036A8A
:10EDE000AB51AC25E96EAD510320EA6EAA51300952
:10EDF000EF6E19D0AA510F0B0F0815E3010EAB5D92
:10EE0000036AAC25E96EAD510320EA6E310EEF6E58
:10EE1000036AAB51AC25E96EAD510320EA6E0A0ED0
:10EE2000AA5D3009EF6E46D10401AA510F0B030809
:10EE300016E3010EAB5D036AAC25E96EAD5103200C
:10EE4000EA6E310EEF6E036AAB51AC25E96EAD513F
:10EE50000320EA6E0A0EAA5D3009EF6E33D0AA5184
:10EE60000F0B0D0816E3010EAB5D036AAC25E96ECE
:10EE7000AD510320EA6E320EEF6E036AAB51AC2542
:10EE8000E96EAD510320EA6E140EAA5D3009EF6EF3
:10EE900019D0AA510F0B0F0815E3010EAB5D036AE1
:10EEA000AC25E96EAD510320EA6E330EEF6E036AB6
:10EEB000AB51AC25E96EAD510320EA6E1E0EAA5D82
:10EEC0003009EF6EF7D00401AA510F0B070816E3C3
:10EED000010EAB5D036AAC25E96EAD510320EA6E0D
:10EEE000330EEF6E036AAB51AC25E96EAD510320D2
:10EEF000EA6E1E0EAA5D3009EF6E19D0AA510F0BF3
:10EF00000F0815E3010EAB5D036AAC25E96EAD5148
:10EF10000320EA6E340EEF6E036AAB51AC25E96E46
:10EF2000AD510320EA6E280EAA5D3009EF6EC2D003
:10EF30000401AA510F0B010816E3010EAB5D036A31
:10EF4000AC25E96EAD510320EA6E340EEF6E036A14
:10EF5000AB51AC25E96EAD510320EA6E280EAA5DD7
:10EF60003009EF6E2FD0AA510F0B0B0816E3010EDC
:10EF7000AB5D036AAC25E96EAD510320EA6E350E38
:10EF8000EF6E036AAB51AC25E96EAD510320EA6E1A
:10EF9000320EAA5D3009EF6E15D0010EAB5D036A2B
:10EFA000AC25E96EAD510320EA6E360EEF6E036AB2
:10EFB000AB51AC25E96EAD510320EA6E3C0EAA5D63
:10EFC0003009EF6E77D00401AA510F0B050816E344
:10EFD000010EAB5D036AAC25E96EAD510320EA6E0C
:10EFE000360EEF6E036AAB51AC25E96EAD510320CE
:10EFF000EA6E3C0EAA5D3009EF6E15D0010EAB5DD6
:10F00000036AAC25E96EAD510320EA6E370EEF6E50
:10F01000036AAB51AC25E96EAD510320EA6E460E92
:10F02000AA5D3009EF6E46D00401AA510F0B090802
:10F0300016E3010EAB5D036AAC25E96EAD5103200A
:10F04000EA6E380EEF6E036AAB51AC25E96EAD5136
:10F050000320EA6E500EAA5D3009EF6E15D0010E46
:10F06000AB5D036AAC25E96EAD510320EA6E390E43
:10F07000EF6E036AAB51AC25E96EAD510320EA6E29
:10F080005A0EAA5D3009EF6E15D0010E0401AB5D7A
:10F09000036AAC25E96EAD510320EA6E450EEF6EB2
:10F0A000036AAB51AC25E96EAD510320EA6E450E03
:10F0B000EF6E00D00001000C040EEA6E840EE96EC3
:10F0C0000801A16BA36B130EA26F000175EC30F069
:10F0D000040EEA6E970EE96E0801A16BA36B130E86
:10F0E000A26F000175EC30F0036A03015E51640FFA
:10F0F000E96E030E0320EA6E0E015B6BEFCF5AFE42
:10F100005D6B120E5C6F0001A2EC34F002C003F0E4
:10F110000150E40F016E010E032201C0AAF403C0E6
:10F12000ABF4040E0801A26F840EA16F03C0A4F813
:10F1300001C0A3F8120EA56F000184EC30F00C0E94
:10F140000401846F040E0801A26F840EA16F0001F8
:10F15000ECEC29F0050E0801A86F0001DDEC28F0A9
:10F16000A8B51CD004018351120DF350036A730F2C
:10F17000016E030E032201C0AAF403C0ABF4040E17
:10F180000801A26F970EA16F03C0A4F801C0A3F8F5
:10F19000120EA56F000184EC30F042D0A8B71CD04D
:10F1A000040EEA6E970EE96E200E0801A16FA36BA4
:10F1B000090EA26F000175EC30F083C4AAF4090EA9
:10F1C0000401AB6F040EAD6F970EAC6F0001DFDD75
:10F1D0000401A16B25D00001040EEA6E970EE96EC2
:10F1E000200E0801A16FA36B090EA26F000175EC40
:10F1F00030F083C4AAF4090E0401AB6F040EAD6FA6
:10F20000970EAC6F0001C3DD730E0401A26F650E93
:10F21000A36F630EA46FA56BA0C4A1F42E0EA06F04
:10F220000A0E0401976F3E0E986F040E0801A26F3C
:10F23000970EA16F0001ECEC29F0000CA8A303D0FD
:10F2400001EF71F01BD0A88303015E51000109E0BA
:10F25000010A09E0030A09E0010A08E0070A06E0DA
:10F2600006D06EEF71F052EF73F003D4FFD4A89381
:10F2700000D0A8A303D003C483F41EDF47EF84F0BB
:10F2800004010651035D03E1010E0525036F030729
:10F2900003015E530AE16451120807E104010351BE
:10F2A000030DF3CF83F483C4BEFF03C483F40001D2
:10F2B00003DF6AEF79F0040EEA6E800EE96E080152
:10F2C000A16BA36B030EA26F000175EC30F0A8A335
:10F2D00002D0D6D7FFD0036A03015E515F0FE96EFB
:10F2E000030E0320EA6EEF50000105E0010A31E051
:10F2F000030A4EE0EFD0036A03015E51640FE96E2A
:10F30000030E0320EA6E020EEF6E036A5E515F0F7A
:10F31000E96E030E0320EA6E010EEF6E036A5E5182
:10F32000640FE96E030E0320EA6EEFCF83F4036AE5
:10F330005E51640FE96E030E0320EA6E010EEF24A6
:10F340000401846F83C499F49A6F000126EC63F082
:10F35000C1D0036A03015E51640FE96E030E0320FE
:10F36000EA6EEF2A036A5E515F0FE96E030E032017
:10F37000EA6E020EEF6E030E0401806F816B040EC5
:10F380000801A26F800EA16F0001ECEC29F0A2D061
:10F39000036A03015E51640FE96E030E0320EA6EF7
:10F3A000EF2A036A5E51640FE96E030E0320EA6ED2
:10F3B000EFCF83F4036A5E51690FE96E030E0320F9
:10F3C000EA6EEF500401835D67E066E303015E537C
:10F3D00024E1036A5E515F0FE96E030E0320EA6EBB
:10F3E000EF6A036A5E51640F016E030E032204018B
:10F3F00003C084F4036A03015E516E0FE96E030ECD
:10F400000320EA6EEFCF85F4040184C4EAFF01C053
:10F41000E9FF85C4EFFF23D00301036A5E515F0F4C
:10F42000E96E030E0320EA6E020EEF6E036A5E5170
:10F43000640F016E030E0322040103C084F4036A07
:10F4400003015E516E0FE96E030E0320EA6E010E9A
:10F45000EF24040184C4EAFF01C0E9FFEF6E036AF0
:10F4600003015E516E0FE96E030E0320EA6EEFCFCB
:10F4700083F4036A5E516E0FE96E030E0320EA6E99
:10F48000010EEF240401846F83C499F49A6F000184
:10F4900026EC63F01ED00401036A03015E51640F81
:10F4A000E96E030E0320EA6E010EEF5C0401836F28
:10F4B000036A03015E51640FE96E030E0320EA6ED6
:10F4C000EFCF84F483C499F484C49AF4000126EC49
:10F4D00063F000D04CEF84F004010551035D03E1BB
:10F4E000010E065D036F032B03015E530AE16451B5
:10F4F000120807E104010351030DF3CF83F483C421
:10F50000BEFF03C483F40001D7DD96EF7AF0040E4A
:10F51000EA6E800EE96E0801A16BA36B030EA26F69
:10F52000000175EC30F0A8A302D0D6D772D1036ADF
:10F5300003015E515F0FE96E030E0320EA6EEF5088
:10F540000208D8A496D0036A5E51640FE96E030ED8
:10F550000320EA6EEF52D8B48CD0036A5E51640F78
:10F56000E96E030E0320EA6EEF065E534BE0036A7A
:10F570005E51640FE96E030E0320EA6EEF5242E122
:10F58000036A5E515F0FE96E030E0320EA6E020EFE
:10F59000EF6E036A5E51690FE96E030E0320EA6E97
:10F5A000010EEF5C0401836F036A03015E51690F72
:10F5B000E96E030E0320EA6EEFCF84F483C499F45E
:10F5C00084C49AF4000126EC63F0036A03015E51DF
:10F5D000640F016E030E0322040103C084F4036A66
:10F5E00003015E51690FE96E030E0320EA6EEFCF4F
:10F5F00085F4040184C4EAFF01C0E9FF85C4EFFF7C
:10F6000036D00301036A5E51640FE96E030E0320D6
:10F61000EA6EEF5216E1036A5E51640FE96E030E63
:10F620000320EA6EEF2A036A5E515F0FE96E030E54
:10F630000320EA6EEF6A010E0401806F816B0ED029
:10F640000301036A5E515F0FE96E030E0320EA6E49
:10F65000010EEF6E020E0401806F816B040E080133
:10F66000A26F800EA16F0001ECEC29F00401D1D053
:10F670000301036A5E51640FE96E030E0320EA6E14
:10F68000EFCF83F4036A5E516E0FE96E030E032021
:10F69000EA6EEF500401835DD8B47AD0D8A078D058
:10F6A000036A03015E51640FE96E030E0320EA6EE4
:10F6B000EF06036A5E51640FE96E030E0320EA6EE3
:10F6C000EF50010849E3036A5E51640FE96E030ECF
:10F6D0000320EA6EEF065E5311E1036A5E515F0F8D
:10F6E000E96E030E0320EA6EEF6A036A5E51640F4F
:10F6F000E96E030E0320EA6EEF6A12D0036A5E51D0
:10F70000640FE96E030E0320EA6E010EEF6E036ACA
:10F710005E515F0FE96E030E0320EA6E020EEF6E7C
:10F72000036A5E516E0FE96E030E0320EA6EEFCF9F
:10F7300083F4036A5E516E0FE96E030E0320EA6ED6
:10F74000010EEF240401846F83C499F49A6F0001C1
:10F7500026EC63F01BD00301036A5E51640FE96E6F
:10F76000030E0320EA6EEFCF83F4036A5E51640F49
:10F77000E96E030E0320EA6E010EEF240401846F8C
:10F7800083C499F49A6F000126EC63F042D004011F
:10F79000036A03015E515F0FE96E030E0320EA6EF8
:10F7A000020EEF6E036A5E51690FE96E030E0320CD
:10F7B000EA6E010EEF5C0401836F036A03015E5180
:10F7C000690FE96E030E0320EA6EEFCF84F483C461
:10F7D00099F484C49AF4000126EC63F0036A0301EF
:10F7E0005E51640F016E030E0322040103C084F412
:10F7F000036A03015E51690FE96E030E0320EA6E8E
:10F80000EFCF85F4040184C4EAFF01C0E9FF85C499
:10F81000EFFF040141EF89F00401666B6791196AFB
:10F82000F2BE198EF29E400E0E01616F626B0001F6
:10F8300063EC24F019BEF28E02C065F401C064F4DA
:10F8400001018C510401641B01018D510401651BF0
:10F8500065C411F464C410F458B40AD04AB102D09B
:10F860004AB306D0126B0DC411F40CC410F4C5D009
:10F8700064C400F06551036E05E100520001D8B484
:10F8800079D00401035006E1010E005C0001D8B4F8
:10F890008CD00401035006E1020E005C0001D8B4D4
:10F8A00084D00401035006E1040E005C0001D8B4CA
:10F8B0007CD00401035006E1080E005C0001D8B4BE
:10F8C00074D00401035006E1100E005C0001D8B4AE
:10F8D0006CD00401035006E1200E005C0001D8B496
:10F8E00064D00401035006E1400E005C0001D8B46E
:10F8F0005CD00401035005E1800E005C000155E07E
:10F900000401010E035C04E1005200014EE0040119
:10F91000020E035C04E10052000147E00401040E02
:10F92000035C04E10052000140E00401080E035CA6
:10F9300004E10052000139E00401100E035C04E10F
:10F940000052000132E00401200E035C04E1005289
:10F9500000012BE00401400E035C04E100520001B1
:10F9600024E00401800E035C04E1005200011DE06C
:10F97000040134D00101435317E004014AB302D01B
:10F98000010112D043C160F05B88686B68510001CF
:10F990009AEC21F00401682B000109EC2CF0190EFF
:10F9A0000401685DF3E101011BD05B9804016781EC
:10F9B00065C4A9F8570E0801AA6F0001ACEC37F036
:10F9C00064C4A9F8570E0801AA6F0001ACEC37F027
:10F9D0000D0E09EC2CF00A0E09EC2CF0010100D000
:10F9E000040167A105D066C412F4128F5B9A05D09A
:10F9F0000DC411F40CC410F4126B0001F7EF9EF06B
:10FA00000401666B020E676F686B696B010139A5B3
:10FA10004DD0040164C4E9FF65C4EAFFECCF6BF488
:10FA2000ED52EFCF6AF464C4E9FF65C4EAFFECCF9E
:10FA30006DF4ED52EFCF6CF4FF0E6C1B6D1B6E6B13
:10FA40006E510001AAEC1BF004016E2B000109ECC1
:10FA50002CF00C0E04016E5DF3E16BC4A9F8370EB7
:10FA60000801AA6F0001ACEC37F06AC4A9F8370EA0
:10FA70000801AA6F0001ACEC37F0200E09EC2CF065
:10FA80006DC4A9F8370E0801AA6F0001ACEC37F07D
:10FA90006CC4A9F8370E0801AA6F0001ACEC37F06E
:10FAA0000A0E09EC2CF00D0E09EC2CF0040164C4D4
:10FAB000E9FF65C4EAFFECCF03F0ED52EFCF68F445
:10FAC00003C069F468C400F06951036E06E1010ED9
:10FAD000005C0001D8B477D00401035006E1020EA7
:10FAE000005C0001D8B472D00401035006E1040E9A
:10FAF000005C0001D8B46DD00401035006E1080E8B
:10FB0000005C0001D8B468D00401035006E1100E77
:10FB1000005C0001D8B463D00401035006E1200E5C
:10FB2000005C0001D8B45ED00401010E035C05E165
:10FB300000520001D8B46DD00401020E035C05E14F
:10FB400000520001D8B468D00401040E035C05E142
:10FB500000520001D8B463D00401080E035C04E134
:10FB6000005200015FE00401100E035C04E100524A
:10FB700000015BE00401200E035C04E1005200017F
:10FB800057E00401035006E1800E005C0001D8B488
:10FB900081D00401035006E1400E005C0001D8B49E
:10FBA0007CD00401400E035C05E100520001D8B492
:10FBB00077D00401800E035C05E100520001D8B447
:10FBC00072D0040188D00401662B00010401662B69
:10FBD00000010401662B00010401662B00010401F1
:10FBE000662B00010401662B0101902D08D0040151
:10FBF00066510101915D03E18F2D01D008D0010E06
:10FC0000906F4A8066C491F14A828F6F498C0401DB
:10FC100062D00401662B00010401662B000104017F
:10FC2000662B00010401662B00010401662B000114
:10FC30000401662B01013AB114D09051020808E189
:10FC4000040166510101915D03E18F51020808E052
:10FC5000020E906F4A8066C491F14A828F6F498C80
:10FC600017D0902D09D0060E040166250101915D83
:10FC700003E18F2D01D00CD0010E906F4A80060E4B
:10FC8000040166250101916F4A82010E8F6F498C34
:10FC9000040121D00401672B00010401672B00013E
:10FCA0000401672B00010401672B67510101905D7E
:10FCB00007E1912D05D00401675101018F5D09E035
:10FCC00067C490F14A80010E916F4A8267C48FF138
:10FCD000498C040100D0000103EF9FF004016B6B1D
:10FCE0006A2D1AD06B6B6851F00B006E036A0350DB
:10FCF00005E1800E005C000109E00401035005E10C
:10FD0000400E005C000105E0040105D004016B2BEE
:10FD1000000104016B2B2DD0020E6B6F68C400F044
:10FD20006951036E05E1800E005C000117E00401DB
:10FD3000035005E1400E005C000113E00401800E59
:10FD4000035C04E1005200010FE00401400E035C7B
:10FD500004E1005200010BE004010BD004016B2B05
:10FD6000000104016B2B000104016B2B0001040155
:10FD70006B2B6BC401F00001000C0401666B6791F2
:10FD80006793196AF2BE198EF29E440E0E01616FDE
:10FD9000626B000163EC24F019BEF28E02C065F4C0
:10FDA00001C064F4FF0E0401641B651B65C41DF4EF
:10FDB00064C41CF44AA105D019C41DF418C41CF471
:10FDC000E7D064C400F06551036E05E10052000104
:10FDD000D8B47FD00401800E035C05E1005200011D
:10FDE000D8B487D00401400E035C05E10052000145
:10FDF000D8B47FD00401035006E1400E005C00013E
:10FE0000D8B477D00401035006E1800E005C0001F5
:10FE1000D8B46FD00401035006E1010E005C00016C
:10FE2000D8B4A1D00401035006E1020E005C000129
:10FE3000D8B499D00401035006E1040E005C00011F
:10FE4000D8B491D00401035006E1080E005C000113
:10FE5000D8B489D00401035006E1100E005C000103
:10FE6000D8B481D00401035006E1200E005C0001EB
:10FE7000D8B479D00401010E035C05E10052000101
:10FE8000D8B471D00401020E035C05E100520001F8
:10FE9000D8B469D00401040E035C05E100520001EE
:10FEA000D8B461D00401080E035C04E100520001E3
:10FEB0005AE00401100E035C04E10052000153E01B
:10FEC0000401200E035C04E1005200014CE0040137
:10FED0004CD004014AB309D058B406D058AE04D06F
:10FEE0005E50030801E2458A01D067835B90589E0B
:10FEF00044D004014AB335D0678158BE28D05BB0E6
:10FF000026D058B424D065C469F464C468F46A6B1C
:10FF10000001E4DE036A0150250F016E000E03228A
:10FF20000150380FE96E010E0320EA6EEF38006EC3
:10FF30000F0E0016005009E0588E5E6A030E040191
:10FF4000666FF28AD76AD66A000108D004015B9016
:10FF5000589E459A58A402D0448058860401668B66
:10FF600001D067830AD0040167815B90589E459A4F
:10FF700058A402D04480588600D067A105D066C43A
:10FF80001EF41E8F5B9A04D019C41DF418C41CF40F
:10FF9000000115EF9FF0780E04014A1301014DA5F1
:10FFA00003D004014A9701014DA103D004014A99ED
:10FFB00001014DA303D004014A9B01014DA703D0C9
:10FFC00004014A9D0101196AF2BE198EF29E480E83
:10FFD0000E016A6F010E6B6F4AC46CFE0001F0ECFB
:08FFE00025F019BEF28E000CA1
:020000040001F9
:1000000004017A6B7B6B7C6B7D6B7E6B7F91040E46
:10001000EA6E660EE96E0801A16BA36B140EA26F67
:10002000000175EC30F0010139A566EF80F00401A4
:1000300064C4E9FF65C4EAFFECCF81F4ED52EFCF71
:1000400080F464C4E9FF65C4EAFFECCF83F4ED52A9
:10005000EFCF82F4FF0E821B831B846B845100015F
:10006000A1EC1EF00401842B000109EC2CF00C0E15
:100070000401845DD8A42EEF80F081C4A9F8370E66
:100080000801AA6F0001ACEC37F080C4A9F8370E64
:100090000801AA6F0001ACEC37F0200E09EC2CF03F
:1000A00083C4A9F8370E0801AA6F0001ACEC37F041
:1000B00082C4A9F8370E0801AA6F0001ACEC37F032
:1000C0000A0E09EC2CF00D0E09EC2CF0040164C4AE
:1000D000E9FF65C4EAFFECCF03F0ED52EFCF7AF40D
:1000E00003C07BF464C4E9FF65C4EAFFEFCF00F00E
:1000F000E92AEF50E906036E0350D8A487EF80F099
:10010000020E005C0001D8B42EEF81F00401035010
:10011000D8A492EF80F0040E005C0001D8B4CFEFB9
:1001200081F004010350D8A49DEF80F0200E005C04
:100130000001D8B4A6EF82F004010350D8A4A8EFC0
:1001400080F0400E005C0001D8B429EF83F0040178
:100150000350D8A4B3EF80F0800E005C0001D8B447
:10016000ACEF83F00401010E035CD8A4BEEF80F075
:1001700000520001D8B445EF84F004010350D8A424
:10018000C9EF80F0080E005C0001D8B44AEF84F09B
:1001900004010350D8A4D4EF80F0100E005C0001DD
:1001A000D8B44FEF84F00401100E035CD8A4DFEF45
:1001B00080F000520001D8B451EF84F00401020E27
:1001C000035CD8A4EAEF80F000520001D8B456EFE7
:1001D00084F00401040E035CD8A4F5EF80F0005213
:1001E0000001D8B41BEF85F00401080E035CD8A40D
:1001F00000EF81F000520001D8B4DFEF85F0040178
:100200000350D8A40BEF81F0010E005C0001D8B4BC
:1002100080EF86F00401200E035CD8A416EF81F075
:1002200000520001D8B441EF87F00401400E035C96
:10023000D8A421EF81F000520001D8B404EF88F077
:100240000401800E035CD8A42CEF81F00052000161
:10025000D8B4A0EF88F0040141EF89F001014D51BD
:10026000F00BD8B4CCEF81F058B03AEF81F058A43D
:1002700048EF81F0588AA09258AC48EF81F0010E07
:100280000801656F0001C8EC28F001013CEF81F026
:1002900004014AB97DEF81F04A89040EEA6E660EC8
:1002A000E96EF2CF80F4F29E000E0001BBEC1EF06E
:1002B0000A000900F550EE6E0009D8A459EF81F04C
:1002C000040180BFF28E01014D9139A77AEF81F0D0
:1002D0000401806B80510001D3EC1EF00401802BDF
:1002E000000109EC2CF00A0E0401805DD8A46AEF2D
:1002F00081F00101ABEF81F004014A99040EEA6E2E
:10030000660EE96EF2CF80F4F29E000E0001E8EC7A
:100310001EF00A000900F550EE6E0009D8A48AEF1D
:1003200081F0040180BFF28E01014D8139A7ABEF4E
:1003300081F00401806B8051000100EC1FF004018A
:10034000802B000109EC2CF0090E0401805DD8A47B
:100350009BEF81F00101196AF2BE198EF29E480EE0
:100360000E016A6F010E6B6F4AC46CFE0001F0EC67
:1003700025F019BEF28E040E08017A6F660E796FB1
:100380000001C3EC30F0468058B0CAEF81F058A4A9
:10039000CCEF81F0589AA082040141EF89F004016A
:1003A0004ABF55EF82F001018953D8B44BEF82F078
:1003B00004014A8F196AF2BE198EF29E480E0E0190
:1003C0006A6F010E6B6F4AC46CFE0001F0EC25F001
:1003D00019BEF28E040EEA6E660EE96EF2CF80F45C
:1003E000F29E000E14EC1FF00A000900F550EE6EAC
:1003F0000009D8A4F5EF81F0040180BFF28E040E4D
:1004000008017A6F660E796F0001C3EC30F0A8A97D
:1004100019EF82F0010189510608D8B403D0000118
:1004200019EF82F008C482F4000139EC6BF01DEF83
:1004300082F089C182F439EC6BF00401806B000119
:100440006EEC6BF0010139A749EF82F00401806B7B
:100450008051000154EC1CF00401802B000109ECD8
:100460002CF0070E0401805DD8A428EF82F089C12A
:100470007FF81F0E0801806F0001FDEC37F00A0EB7
:1004800009EC2CF00D0E09EC2CF03E0E09EC2CF0D2
:10049000010152EF82F0010E0401806F00016EEC49
:1004A0006BF00101A3EF82F004014A9F196AF2BECA
:1004B000198EF29E480E0E016A6F010E6B6F4AC4D0
:1004C0006CFE0001F0EC25F019BEF28E040EEA6E0F
:1004D000660EE96EF2CF80F4F29E000E2CEC1FF057
:1004E0000A000900F550EE6E0009D8A471EF82F001
:1004F000040180BFF28E040E08017A6F660E796FD8
:100500000001C3EC30F089C182F439EC6BF0010ECC
:100510000401806F00016EEC6BF0010139A7A3EFBD
:1005200082F00401806B8051000144EC1FF0040153
:10053000802B000109EC2CF00B0E0401805DD8A487
:1005400093EF82F00101040141EF89F004014AB503
:10055000DDEF82F0060E4A134A93040EEA6E660E31
:10056000E96EF2CF80F4F29E000E000159EC1FF00C
:100570000A000900F550EE6E0009D8A4B9EF82F028
:10058000040180BFF28E0101399139A7DAEF82F0C0
:100590000401806B8051000171EC1FF00401802B7D
:1005A000000109EC2CF0110E0401805DD8A4CAEF03
:1005B00082F001010DEF83F00401060E4A134A9503
:1005C000040EEA6E660EE96EF2CF80F4F29E000E23
:1005D000000189EC1FF00A000900F550EE6E0009D9
:1005E000D8A4ECEF82F0040180BFF28E01013981C2
:1005F00039A70DEF83F00401806B80510001A1EC5D
:100600001FF00401802B000109EC2CF00F0E0401F7
:10061000805DD8A4FDEF82F00101196AF2BE198E47
:10062000F29E480E0E016A6F010E6B6F4AC46CFE9B
:100630000001F0EC25F019BEF28E040E08017A6F6D
:10064000660E796F0001C3EC30F0448E040141EF77
:1006500089F004014AB360EF83F0060E4A134A950D
:10066000040EEA6E660EE96EF2CF80F4F29E000E82
:10067000000189EC1FF00A000900F550EE6E000938
:10068000D8A43CEF83F0040180BFF28E01013981D0
:1006900039A75DEF83F00401806B80510001A1EC6C
:1006A0001FF00401802B000109EC2CF00F0E040157
:1006B000805DD8A44DEF83F0010190EF83F0040139
:1006C000060E4A134A93040EEA6E660EE96EF2CFE6
:1006D00080F4F29E000E000159EC1FF00A000900A0
:1006E000F550EE6E0009D8A46FEF83F0040180BFCF
:1006F000F28E0101399139A790EF83F00401806BEC
:100700008051000171EC1FF00401802B000109EC05
:100710002CF0110E0401805DD8A480EF83F001015C
:10072000196AF2BE198EF29E480E0E016A6F010E12
:100730006B6F4AC46CFE0001F0EC25F019BEF28E1E
:10074000040E08017A6F660E796F0001C3EC30F079
:10075000448E040141EF89F004014AB125EF84F091
:10076000020E6425E96E000E6521EA6EEFCF80F47B
:10077000000E80BD010E000AD8A404EF84F0196AAF
:10078000F2BE198EF29E460E0E01616F626B000181
:1007900063EC24F019BEF28E02C07DF401C07CF43B
:1007A000010E04017E6F7E516308D8A004EF84F02F
:1007B0007C51FF0A806F7D51FF0A816F8051800854
:1007C000D8A4E7EF83F08153D8B4E9EF83F041EF89
:1007D00089F00A0E0801656F0001C8EC28F0196A5B
:1007E000F2BE198EF29E460E0E01616F626B000121
:1007F00063EC24F019BEF28E02C07DF401C07CF4DB
:1008000004017E2BD3EF83F0010139A719EF84F0A7
:100810000401806B80510001B8EC1FF00401802BB3
:10082000000109EC2CF00C0E0401805DD8A40AEF45
:1008300084F00401806B00010FEC6CF08E909790B7
:10084000040141EF89F043EF84F0010139A73AEF49
:1008500084F00401806B80510001CEEC1FF0040194
:10086000802B000109EC2CF00B0E0401805DD8A454
:100870002BEF84F0010E0401806F00010FEC6CF08F
:10088000040141EF89F041EF89F01EEF79F0040196
:1008900041EF89F05BEF79F0040141EF89F087EFD8
:1008A0007AF02EEC71F0040141EF89F001014D5115
:1008B000F00BD8B418EF85F058B062EF84F058A46C
:1008C00070EF84F0588AA09258AC70EF84F0010E5B
:1008D0000801656F0001C8EC28F0010164EF84F0A5
:1008E00004014AB78EEF84F0140EEF6F010EF06F23
:1008F00000011BEC50F001014D95036A8A51250F50
:10090000016E000E03220150380F016E010E03220A
:1009100001C0E9FF03C0EAFFEF9404014A87196AA6
:10092000F2BE198EF29E480E0E016A6F010E6B6FB9
:100930004AC46CFE0001F0EC25F019BEF28E040EE4
:10094000EA6E660EE96EF2CF80F4F29E000EE3ECE2
:100950001FF00A000900F550EE6E0009D8A4AAEFB6
:1009600084F0040180BFF28E040E08017A6F660ED7
:10097000796F0001C3EC30F0010139A7D1EF84F0A9
:100980000401806B80510001FBEC1FF00401802BFF
:10099000000109EC2CF00C0E0401805DD8A4C2EF1C
:1009A00084F004017F910001B5EC60F0160E0401A3
:1009B000EF6F010EF06F00011BEC50F004017FB1EE
:1009C00010EF85F0196AF2BE198EF29E460E0E01E6
:1009D000616F626B000163EC24F019BEF28E02C0FD
:1009E0007DF401C07CF404017C51FF0A806F7D51CD
:1009F000FF0A816F8053D8A403EF85F0815102086C
:100A0000D8B406EF85F07F810EEF85F0160EEF6FFC
:100A1000010EF06F00011BEC50F00401DFEF84F0D9
:100A200058B016EF85F058A418EF85F0589AA082B8
:100A3000040141EF89F001014D51F00BD8B4DCEF16
:100A400085F058B027EF85F058A435EF85F0588A27
:100A5000A09258AC35EF85F0010E0801656F0001DA
:100A6000C8EC28F0010129EF85F004014AB753EFE3
:100A700085F0140EEF6F010EF06F00011BEC50F0CB
:100A800001014D95036A8A51250F016E000E032264
:100A90000150380F016E010E032201C0E9FF03C0AF
:100AA000EAFFEF9404014A87196AF2BE198EF29E9A
:100AB000480E0E016A6F010E6B6F4AC46CFE000196
:100AC000F0EC25F019BEF28E040EEA6E660EE96EA9
:100AD000F2CF80F4F29E000E11EC20F00A00090023
:100AE000F550EE6E0009D8A46FEF85F0040180BFC9
:100AF000F28E040E08017A6F660E796F0001C3EC66
:100B000030F0010139A796EF85F00401806B805128
:100B1000000129EC20F00401802B000109EC2CF0ED
:100B20000E0E0401805DD8A487EF85F00001B5ECBE
:100B300060F0170E0401EF6F010EF06F00011BEC67
:100B400050F004017F917FB1D4EF85F0196AF2BEB5
:100B5000198EF29E460E0E01616F626B000163EC0E
:100B600024F019BEF28E02C07DF401C07CF40401B1
:100B70007C51FF0A806F7D51FF0A816F8053D8A49A
:100B8000C7EF85F081510408D8B4CAEF85F07F81A2
:100B9000D2EF85F0170EEF6F010EF06F00011BEC26
:100BA00050F00401A3EF85F058B0DAEF85F058A4B7
:100BB000DCEF85F0589AA082040141EF89F0010131
:100BC0004D51F00BD8B47DEF86F058B0EBEF85F0C7
:100BD00058A4F9EF85F0588AA09258ACF9EF85F047
:100BE000010E0801656F0001C8EC28F00101EDEF6E
:100BF00085F004014AA72EEF86F04A97040EEA6EAC
:100C0000660EE96EF2CF80F4F29E000E000140EC19
:100C100020F00A000900F550EE6E0009D8A40AEF92
:100C200086F0040180BFF28E01014D8539A72BEFBC
:100C300086F00401806B8051000158EC20F0040123
:100C4000802B000109EC2CF00E0E0401805DD8A46D
:100C50001BEF86F001015CEF86F004014A87040E69
:100C6000EA6E660EE96EF2CF80F4F29E000E00018D
:100C70006FEC20F00A000900F550EE6E0009D8A4D0
:100C80003BEF86F0040180BFF28E01014D9539A73C
:100C90005CEF86F00401806B8051000187EC20F04E
:100CA0000401802B000109EC2CF0100E0401805D82
:100CB000D8A44CEF86F00101040E08017A6F660E8D
:100CC000796F0001C3EC30F0196AF2BE198EF29E02
:100CD000480E0E016A6F010E6B6F4AC46CFE000174
:100CE000F0EC25F019BEF28E468058B07BEF86F00E
:100CF00058A47DEF86F0589AA082040141EF89F054
:100D000001014D51F00BD8B43EEF87F058B08CEF95
:100D100086F058A49AEF86F0588AA09258AC9AEFC1
:100D200086F0010E0801656F0001C8EC28F0010192
:100D30008EEF86F004014ABDB8EF86F01C0EEF6F0F
:100D4000010EF06F00011BEC50F001014D97036A9A
:100D50008A51250F016E000E03220150380F016EDB
:100D6000010E032201C0E9FF03C0EAFFEF96040170
:100D70004A8D196AF2BE198EF29E480E0E016A6FF4
:100D8000010E6B6F4AC46CFE0001F0EC25F019BE39
:100D9000F28E040EEA6E660EE96EF2CF80F4F29ED9
:100DA000000E9FEC20F00A000900F550EE6E0009DD
:100DB000D8A4D4EF86F0040180BFF28E040E08019F
:100DC0007A6F660E796F0001C3EC30F0010139A72C
:100DD000FBEF86F00401806B80510001B7EC20F03E
:100DE0000401802B000109EC2CF00D0E0401805D44
:100DF000D8A4ECEF86F01E0E0401EF6F010EF06F29
:100E000000011BEC50F004017F917FB12FEF87F0C0
:100E1000420E006E002EFED70000196AF2BE198E37
:100E2000F29E460E0E01616F626B000163EC24F0CE
:100E300019BEF28E02C07DF401C07CF404017C5125
:100E4000FF0A806F7D51FF0A816F802D2CEF87F0A4
:100E50008153D8B42DEF87F07F8105EF87F01F0E07
:100E6000EF6F010EF06F00011BEC50F058B03CEF3B
:100E700087F058A43EEF87F0589AA082040141EF12
:100E800089F001014D51F00BD8B401EF88F058B052
:100E90004DEF87F058A45BEF87F0588AA09258ACCA
:100EA0005BEF87F0010E0801656F0001C8EC28F0C8
:100EB00001014FEF87F004014ABD79EF87F01C0E66
:100EC000EF6F010EF06F00011BEC50F001014D9728
:100ED000036A8A51250F016E000E03220150380F5C
:100EE000016E010E032201C0E9FF03C0EAFFEF9685
:100EF00004014A8D196AF2BE198EF29E480E0E0147
:100F00006A6F010E6B6F4AC46CFE0001F0EC25F0B5
:100F100019BEF28E040EEA6E660EE96EF2CF80F410
:100F2000F29E000ECDEC20F00A000900F550EE6EA6
:100F30000009D8A495EF87F0040180BFF28E040E5B
:100F400008017A6F660E796F0001C3EC30F0010181
:100F500039A7BCEF87F00401806B80510001E5ECFC
:100F600020F00401802B000109EC2CF00C0E040190
:100F7000805DD8A4ADEF87F01D0E0401EF6F010E68
:100F8000F06F00011BEC50F004017F917FB1F2EF94
:100F900087F0420E006E002EFED70000196AF2BEE6
:100FA000198EF29E460E0E01616F626B000163ECBA
:100FB00024F019BEF28E02C07DF401C07CF404015D
:100FC0007C51FF0A806F7D51FF0A816F8053D8A446
:100FD000EFEF87F081512008D8B4F0EF87F07F81E0
:100FE000C6EF87F01F0EEF6F010EF06F00011BECD4
:100FF00050F058B0FFEF87F058A401EF88F0589AEE
:10100000A082040141EF89F001014D51F00BD8B4E9
:101010009DEF88F058B010EF88F058A41EEF88F0CC
:10102000588AA09258AC1EEF88F0010E0801656F37
:101030000001C8EC28F0010112EF88F004014AAD6C
:101040003EEF88F04A9D040EEA6E660EE96EF2CF1E
:1010500080F4F29E000E0001FBEC20F00A00090073
:10106000F550EE6E0009D8A42FEF88F0040180BF80
:10107000F28E01014D8766EF88F004014A8D196AEE
:10108000F2BE198EF29E480E0E016A6F010E6B6F52
:101090004AC46CFE0001F0EC25F019BEF28E040E7D
:1010A000EA6E660EE96EF2CF80F4F29E000E13EC4B
:1010B00021F00A000900F550EE6E0009D8A45AEF9D
:1010C00088F0040180BFF28E01014D97196AF2BECB
:1010D000198EF29E480E0E016A6F010E6B6F4AC4A4
:1010E0006CFE0001F0EC25F019BEF28E040E080132
:1010F0007A6F660E796F0001C3EC30F04680010113
:1011000039A795EF88F00401806B805100012BEC2A
:1011100021F00401802B000109EC2CF00D0E0401DC
:10112000805DD8A485EF88F0010158B09BEF88F06E
:1011300058A49DEF88F0589AA082040141EF89F0ED
:1011400001014D51F00BD8B43EEF89F058B0ACEF2F
:1011500088F058A4BAEF88F0588AA09258ACBAEF39
:1011600088F0010E0801656F0001C8EC28F001014C
:10117000AEEF88F004014ABBEFEF88F04A8B040E13
:10118000EA6E660EE96EF2CF80F4F29E000E000168
:1011900041EC21F00A000900F550EE6E0009D8A4D8
:1011A000CBEF88F0040180BFF28E01014D9339A787
:1011B000ECEF88F00401806B8051000159EC21F0C4
:1011C0000401802B000109EC2CF00A0E0401805D63
:1011D000D8A4DCEF88F001011DEF89F004014A9BDF
:1011E000040EEA6E660EE96EF2CF80F4F29E000EF7
:1011F00000016EEC21F00A000900F550EE6E0009C6
:10120000D8A4FCEF88F0040180BFF28E01014D8369
:1012100039A71DEF89F00401806B8051000186EC35
:1012200021F00401802B000109EC2CF0090E0401CF
:10123000805DD8A40DEF89F00101040E08017A6FDA
:10124000660E796F0001C3EC30F0196AF2BE198E98
:10125000F29E480E0E016A6F010E6B6F4AC46CFE5F
:101260000001F0EC25F019BEF28E468058B03CEF3C
:1012700089F058A43EEF89F0589AA082040141EF0A
:1012800089F00001000C0401806B7F510008D8B088
:101290007CEF89F07F510608D8A07CEF89F0196AAD
:1012A000F2BE198EF29E880E0E01676F010E686FF6
:1012B00000011DEC24F019BEF28E01C080F40A0E6C
:1012C0000801656F0001C8EC28F0196AF2BE198E9A
:1012D000F29E880E0E016A6F010E6B6F7FC46CFE6A
:1012E0000001F0EC25F019BEF28E640E0801656F66
:1012F0000001C8EC28F00401000124EF8BF0040188
:10130000806B816B7F51010A0001D8B496EF89F0A0
:10131000030AD8B49DEF89F0010AD8B4A4EF89F08C
:10132000070AD8B4ABEF89F0B2EF89F07F0E040161
:10133000816FFF0E806FB8EF89F0BF0E0401816FDF
:10134000FF0E806FB8EF89F0FF0E0401816FBF0EB2
:10135000806FB8EF89F0FF0E0401816F7F0E806F00
:10136000B8EF89F0FF0E0401816F806FB8EF89F04C
:10137000196AF2BE198EF29E400E0E01636F646B05
:1013800081C466FE80C465FE00011CEC26F019BE17
:10139000F28EAEEF8CF00401666B676B020E686F25
:1013A0007D6B7E6B040EEA6E690EE96E0801A16B1F
:1013B000A36B140EA26F000175EC30F0010139A58A
:1013C00031EF8AF0040164C4E9FF65C4EAFFECCFA1
:1013D00080F4ED52EFCF7FF464C4E9FF65C4EAFF07
:1013E000ECCF82F4ED52EFCF81F4FF0E811B821B14
:1013F000836B83510001C4EC1BF00401832B0001BB
:1014000009EC2CF00C0E0401835DD8A4F9EF89F0EF
:1014100080C4A9F8370E0801AA6F0001ACEC37F0C0
:101420007FC4A9F8370E0801AA6F0001ACEC37F0B1
:10143000200E09EC2CF082C4A9F8370E0801AA6F1F
:101440000001ACEC37F081C4A9F8370E0801AA6F8F
:101450000001ACEC37F00A0E09EC2CF00D0E09EC93
:101460002CF0040164C4E9FF65C4EAFFECCF03F08B
:10147000ED52EFCF66F403C067F466C400F067C4B2
:1014800003F0200E675DD8A44CEF8AF000520001F3
:10149000D8B4F3EF8AF00401100E035CD8A457EF20
:1014A0008AF000520001D8B4F6EF8AF00401080E69
:1014B000035CD8A462EF8AF000520001D8B4F9EFBF
:1014C0008AF00401040E035CD8A46DEF8AF0005288
:1014D0000001D8B4FCEF8AF00401020E035CD8A42A
:1014E00078EF8AF000520001D8B4FFEF8AF00401CF
:1014F000010E035CD8A483EF8AF000520001D8B437
:1015000002EF8BF004010350D8A48EEF8AF0200E76
:10151000005C0001D8B4B5EF8BF004010350D8A4EF
:1015200099EF8AF0100E005C0001D8B4B8EF8BF090
:1015300004010350D8A4A4EF8AF0080E005C000157
:10154000D8B4BBEF8BF004010350D8A4AFEF8AF0FE
:10155000040E005C0001D8B4BEEF8BF00401035010
:10156000D8A4BAEF8AF0020E005C0001D8B4C1EF33
:101570008BF004010350D8A4C5EF8AF0010E005C83
:101580000001D8B4C4EF8BF004010350D8A4D0EF0D
:101590008AF0800E005C0001D8B4B1EF8CF0040139
:1015A0000350D8A4DBEF8AF0400E005C0001D8B4F1
:1015B000B4EF8CF00401800E035CD8A4E6EF8AF04F
:1015C00000520001D8B4B7EF8CF00401400E035C68
:1015D000D8A4F1EF8AF000520001D8B4BAEF8CF031
:1015E000040193EF8DF004017D2B000104017D2B9C
:1015F000000104017D2B000104017D2B0001040189
:101600007D2B000104017D2B3F0E4C136651FF0A18
:10161000006E6751FF0A036E00504B1703504C17C2
:10162000196AF2BE198EF29E4A0E0E01636F646B48
:101630004CC466FE4BC465FE00011CEC26F019BECE
:10164000F28E7DC47FF41FD67DC488F1A8A94AEF2D
:101650008BF004017D510608D8B403D000014AEF95
:101660008BF0040EEA6E690EE96EF2CF7FF4F29E03
:10167000000E0001DEEC1BF00A000900F550EE6ED2
:101680000009D8A43DEF8BF004017FBFF28E62EF1A
:101690008BF00001040EEA6E690EE96EF2CF7FF462
:1016A000F29E000EF6EC1BF00A000900F550EE6EFB
:1016B0000009D8A455EF8BF004017FBFF28E7D5155
:1016C0003009766F5BBA6DEF8BF0040E08017A6F0C
:1016D000690E796F0001C3EC30F0010139A794EF76
:1016E0008BF004017F6B7F5100010DEC1CF00401B5
:1016F0007F2B000109EC2CF00A0E04017F5DD8A4B9
:1017000073EF8BF07DC47FF81F0E0801806F00011E
:10171000FDEC37F00A0E09EC2CF00D0E09EC2CF064
:101720003E0E09EC2CF001013AAFB2EF8BF0036AE8
:1017300004017D51250F016E000E03220150380F68
:10174000E96E010E0320EA6EEF50F00BD8B4B3EF50
:101750008BF07D5101018A5DD8B4B2EF8BF07DC46E
:1017600090F14A80040193EF8DF004017E2B00017B
:1017700004017E2B000104017E2B000104017E2B5D
:10178000000104017E2B000104017E2B3F0E4B1350
:101790006651FF0A006E6751FF0A036E00504B1737
:1017A00003504C17196AF2BE198EF29E4A0E0E01B2
:1017B000636F646B4CC466FE4BC465FE00011CEC99
:1017C00026F019BEF28E04014A8F196AF2BE198EF4
:1017D000F29E480E0E016A6F010E6B6F4AC46CFEDA
:1017E0000001F0EC25F019BEF28EA8A930EF8CF0C4
:1017F00004017E510608D8B414EF8CF00101895120
:101800000608D8B403D0040114EF8CF07EC482F42F
:10181000000139EC6BF0010E04019B6F00019EEC9E
:101820003EF030EF8CF004017E510608D8A42BEF77
:101830008CF0010189510608D8A403D004012BEFD4
:101840008CF089C108F404019B6B00019EEC3EF012
:1018500030EF8CF004017EC482F4000139EC6BF0AF
:10186000A8B937EF8CF07EC482F439EC6BF07EC4FB
:1018700089F1A8A95DEF8CF0010189510608D8B45F
:1018800003D000015DEF8CF0040EEA6E690EE96E84
:10189000F2CF7FF4F29E000E000124EC1CF00A004F
:1018A0000900F550EE6E0009D8A450EF8CF0040149
:1018B0007FBFF28E75EF8CF00001040EEA6E690EA8
:1018C000E96EF2CF7FF4F29E000E3CEC1CF00A00B1
:1018D0000900F550EE6E0009D8A468EF8CF0040101
:1018E0007FBFF28E7E513009756F5BBA80EF8CF04E
:1018F000040E08017A6F690E796F0001C3EC30F0B5
:10190000010139A7A7EF8CF004017F6B7F51000123
:1019100054EC1CF004017F2B000109EC2CF0070EA5
:1019200004017F5DD8A486EF8CF07EC47FF81F0E83
:101930000801806F0001FDEC37F00A0E09EC2CF075
:101940000D0E09EC2CF03E0E09EC2CF001013AA929
:10195000AEEF8CF07EC47FF40001D1D4040193EF8C
:101960008DF00401682B00010401682B00010401C3
:10197000682B00010401682B036A6851250F016E72
:10198000000E03220150380FE96E010E0320EA6EAB
:10199000EF50F00BD8A4DCEF8CF0020E6425E96E5A
:1019A000000E6521EA6EEFCF7FF4000E7FBB010EC3
:1019B000000AD8A46FEF8DF0C00E4B134C13665184
:1019C000FF0A006E6751FF0A036E00504B17035069
:1019D0004C17196AF2BE198EF29E4A0E0E01636F01
:1019E000646B4CC466FE4BC465FE00011CEC26F023
:1019F00019BEF28ECF0E04014813FF0E4913196A67
:101A0000F2BE198EF29E4C0E0E01636F646B49C4D8
:101A100066FE48C465FE00011CEC26F019BEF28E7D
:101A200068C479F8C7EC54F068C499F4B7EC3DF099
:101A3000050E0801656F0001C8EC28F0CBEC7FF0C3
:101A4000040EEA6E690EE96EF2CF7FF4F29E000E8C
:101A50006AEC1CF00A000900F550EE6E0009D8A4EB
:101A60002BEF8DF004017FBFF28E68513009766F45
:101A70005BBA44EF8DF0040E08017A6F690E796F3E
:101A80000001C3EC30F004014680010139A76CEF7E
:101A90008DF004017F6B7F51000182EC1CF004018A
:101AA0007F2B000109EC2CF0070E04017F5DD8A408
:101AB0004BEF8DF068C47FF81F0E0801806F0001A6
:101AC000FDEC37F00A0E09EC2CF00D0E09EC2CF0B1
:101AD0003E0E09EC2CF0010190EF8DF00401040E94
:101AE000EA6E690EE96EF2CF7FF4F29E000E0001FD
:101AF00098EC1CF00A000900F550EE6E0009D8A41D
:101B00007BEF8DF004017FBFF28E68513009726F58
:101B1000040E08017A6F690E796F0001C3EC30F092
:101B2000040193EF8DF00001000C0401646B656B00
:101B3000666B67916793196AF2BE198EF29E420E28
:101B40000E01616F626B000163EC24F019BEF28E2E
:101B500002C065F401C064F4FF0E0401641B651B40
:101B600065C429F464C428F44AA1BDEF8DF025C4EE
:101B700029F424C428F4FBEF8EF064C400F065510E
:101B8000036ED8A4CAEF8DF000520001D8B47CEFE8
:101B90008EF004010350D8A4D5EF8DF0400E005C08
:101BA0000001D8B490EF8EF004010350D8A4E0EF08
:101BB0008DF0800E005C0001D8B490EF8EF004012F
:101BC0000350D8A4EBEF8DF0010E005C0001D8B4F7
:101BD000D6EF8EF004010350D8A4F6EF8DF0020E7C
:101BE000005C0001D8B4D6EF8EF004010350D8A4F5
:101BF00001EF8EF0040E005C0001D8B4D6EF8EF039
:101C000004010350D8A40CEF8EF0080E005C000114
:101C1000D8B4D6EF8EF00401010E035CD8A417EF00
:101C20008EF000520001D8B4D6EF8EF00401020EFF
:101C3000035CD8A422EF8EF000520001D8B4D6EF96
:101C40008EF00401040E035CD8A42DEF8EF0005238
:101C50000001D8B4D6EF8EF00401080E035CD8A4BE
:101C600038EF8EF000520001D8B4D6EF8EF00401A8
:101C7000100E035CD8A443EF8EF000520001D8B4DC
:101C8000D6EF8EF00401200E035CD8A44EEF8EF048
:101C900000520001D8B4D6EF8EF00401400E035C70
:101CA000D8A459EF8EF000520001D8B4D6EF8EF0D0
:101CB0000401800E035CD8A464EF8EF00052000192
:101CC000D8B4D6EF8EF004010350D8A46FEF8EF095
:101CD000200E005C0001D8B4E2EF8EF00401035046
:101CE000D8A47AEF8EF0100E005C0001D8B4E2EFB9
:101CF0008EF00401E4EF8EF004014AB38CEF8EF015
:101D000058B48CEF8EF05BA08CEF8EF05E50020822
:101D1000D8B08CEF8EF0458A5B90589EEEEF8EF037
:101D200004014AB3D3EF8EF0678158BEC7EF8EF03F
:101D30005BB0C7EF8EF058B4C7EF8EF065C469F49E
:101D400064C468F4010E6A6F00016EEC7EF0036AF1
:101D50000150250F016E000E03220150380FE96E6D
:101D6000010E0320EA6EEF38006E0F0E00160050D1
:101D7000D8B4C4EF8EF05B805E6A030E0401666F18
:101D8000F28AD76AD66A0001CFEF8EF004015B9029
:101D9000589E459A58A4CFEF8EF04480588604018F
:101DA000668BD4EF8EF06783EEEF8EF004014AB3BA
:101DB000DDEF8EF06781DEEF8EF067835B90589EDB
:101DC000EEEF8EF0040167815B90589E459A58A40F
:101DD000ECEF8EF044805886EEEF8EF067A1F7EFBF
:101DE0008EF066C42AF42A8F5B9AFBEF8EF025C42E
:101DF00029F424C428F4000133EF9FF004019A6B06
:101E00009B6B9C6B020E9D6F900E9E6F040EEA6E94
:101E10008A0EE96E0801A16BA36B100EA26F000180
:101E200075EC30F0040186C4E9FF87C4EAFFEE5286
:101E3000EE52EC6AED52EF6AED52EF6AED52EF6A44
:101E400088C4E9FF89C4EAFFEC6AED52EF6AFA0E32
:101E50000801A86F0001DDEC28F0A8B173EF8FF046
:101E600004019A510F08D8B003D0000173EF8FF02E
:101E7000000184EC37F001C09CF40A0E0801A86F41
:101E80000001DDEC28F0010139A555EF8FF09CC46D
:101E9000A9F8570E0801AA6F0001ACEC37F0200E2C
:101EA00009EC2CF05BEF8FF00101320E0801A86FF6
:101EB0000001DDEC28F004019E519C5DD8A466EF82
:101EC0008FF09A6B9CC48AF470EF8FF09A2B036AA0
:101ED0009A518A0FE96E040E0320EA6E9CC4EFFF4C
:101EE00000012DEF8FF0080E04019D259A5DD8B0FA
:101EF0007EEF8FF0000E016E3FEF90F0036A9D5170
:101F00008A0FE96E040E0320EA6EEFCF9FF4000EF5
:101F10009FB7010E0108D8A499EF8FF086C4E9FF9E
:101F200087C4EAFFFF0EEF6EEC6EEC6EEC6EA6EF70
:101F30008FF086C4E9FF87C4EAFFEE52EE52EC6AE6
:101F4000ED52EF6AED52EF6AED52EF6A9B6B9B51D7
:101F50000408D8A0FEEF8FF086C4E9FF87C4EAFF2B
:101F6000EF34006EEC34016EEC34026EEC34036E30
:101F700000360136023603360036013602360336A5
:101F80000036013602360336F00E0016ED52ED52E1
:101F9000ED5200C0EFFF01C0ECFF02C0ECFF03C038
:101FA000ECFF87C403F087C4EAFF86C4E9FFEFCFE4
:101FB000A1F4ECCFA2F4ECCFA3F4ECCFA4F49B51AA
:101FC0009D25036A8A0FE96E040E0320EA6EEF5026
:101FD0000F0BA111A2C401F0A3C402F0A4C403F02A
:101FE00087C4EAFF86C4E9FFEF6EA2C4ECFFA3C476
:101FF000ECFFA4C4ECFF9B2BA7EF8FF0050E9B6FAB
:102000009B510808D8A03DEF90F088C4E9FF89C42F
:10201000EAFFEF34026EEC34036E0236033602360A
:10202000033602360336F00E02160250ED52EF6E02
:1020300003C0ECFF89C403F089C4EAFF88C4E9FF48
:10204000ECCFA2F4ED52EFCFA1F49B519D25036A92
:102050008A0FE96E040E0320EA6EEF500F0BA111F8
:10206000A2C403F089C4EAFF88C4E9FFA2C4ECFF5C
:10207000ED52EF6E9B2B00EF90F0010E016E000110
:10208000AFEF91F00401986B996B9A6B020E9B6F06
:10209000900E9C6F86C4E9FF87C4EAFFEE52EE52B1
:1020A000EC6AED52EF6AED52EF6AED52EF6A010110
:1020B0004D39006E0F0E001600500C08D8A467EFC3
:1020C00090F0050E04019B6FFE0E9C6F0101040E43
:1020D000EA6E880EE96E0801A16BA36B100EA26F69
:1020E000000175EC30F0FA0E0801A86F0001DDEC7C
:1020F00028F0A8B1BFEF90F0040198510F08D8B0B4
:1021000003D00001BFEF90F0000184EC37F001C074
:1021100099F40A0E0801A86F0001DDEC28F0010116
:1021200039A5A1EF90F099C4A9F8570E0801AA6F3C
:102130000001ACEC37F0200E09EC2CF0A7EF90F08A
:1021400001010A0E0801A86F0001DDEC28F004016E
:102150009C51995DD8A4B2EF90F0986B99C488F423
:10216000BCEF90F0982B036A9851880FE96E040E2B
:102170000320EA6E99C4EFFF000179EF90F0070E9B
:1021800004019B25985DD8B0CAEF90F0000E016E57
:102190005EEF91F001014D39006E0F0E00160050F8
:1021A0000C08D8A403EF91F09BC49AF4070E040125
:1021B0009B259A5DD8B4E0EF90F0D8B004EF91F091
:1021C000036A9A51880F016E040E032201C09DF428
:1021D00003C09EF4036A9A51880FE96E040E03202F
:1021E000EA6EEFCF9FF49FC4AFF40001C6EC5EF03F
:1021F0009EC4EAFF9DC4E9FF01C0EFFF04019A2BD2
:102200000101D6EF90F004019A6B9A510708D8A00B
:102210005CEF91F086C4E9FF87C4EAFFEF34006EFB
:10222000EC34016EEC34026EEC34036E0036013691
:1022300002360336003601360236033600360136E2
:1022400002360336F00E0016ED52ED52ED5200C08C
:10225000EFFF01C0ECFF02C0ECFF03C0ECFF87C43E
:1022600003F087C4EAFF86C4E9FFEFCF9FF4ECCF09
:10227000A0F4ECCFA1F4ECCFA2F49A519B25036A11
:10228000880FE96E040E0320EA6EEF500F0B9F11CA
:10229000A0C401F0A1C402F0A2C403F087C4EAFF05
:1022A00086C4E9FFEF6EA0C4ECFFA1C4ECFFA2C49A
:1022B000ECFF9A2B05EF91F0010E016E0001D1EFBA
:1022C00091F004017E6B7F6B806B816B826B836B03
:1022D000846B858100017CEC3AF00401EF6B010E08
:1022E000F06F00011BEC50F001014D39006E0F0E34
:1022F000001600500A08D8B4E1EF91F000017CEC20
:102300003AF00A0E0401EF6FF06B00011BEC50F085
:1023100001014D39006E0F0E001600500808D8B4A8
